:020000040000FA
:100000000236920226D4C203A20322023F1CD2DA95
:10001000D2DB22025CB6EF25E025E0242CFE24038F
:10002000F8E220E60CEF25E025E0242EF8EDF2D3EF
:1000300022C322022BD2C2A20264330259DEAE07CF
:10004000AC03AF057401A807088002C333D8FCFADB
:10005000AF06FDAB0412475E0247A8025598900B0D
:10006000027402F0C294126490EF640160F8D2A4AA
:10007000D201126B057F0112660D7F011265FFC26E
:1000800001126B05438510224C4334434550322006
:10009000312E303800120976501A1265CEEF640402
:1000A00060030201311265C7EF641A600302013177
:1000B00012097C22120982500A9008B3E0FFC31390
:1000C00020E02D126A9FEF600D302E05122D9580D5
:1000D0001F1229F5801A126AA5EF70047F018002B1
:1000E0007F00BF0108E4FF12098812098E12639590
:1000F000123CF0900D3EE0B40108900BB8E0640CA7
:10010000702F120994402A302E19900BB8E0B4B425
:1001100012900BE9E0FF64046009EF6405600412CB
:10012000099A221209A05006124ABC124170120903
:100130009A22900BC9E004F0900BEAE020E14F1204
:10014000174A900BC9E030E00412175022900BC9F7
:10015000E030E10412175622900BC9E030E204129D
:10016000175C22900BC9E030E30412176222900B57
:10017000C9E030E40412176822900BC9E030E504AE
:1001800012176E22900BC9E030E603121774221288
:100190006AB1EF700A120B0240057FB0120AFC3000
:1001A0002E05123C7A8003123C04900BEEE0FEA375
:1001B000E0FF4E6010EF5403700B7890E6FF125A88
:1001C000621260D622125CA37878EEF608EFF6E6AB
:1001D000184660487A00799378937C007D007B0014
:1001E0007A0079787E007F02121B07E47892F67914
:1001F00094E77896667008900BECE004F08005E4D4
:10020000900BECF07893E6FF08E608CFF608EFF6DF
:100210007890E6FF125A621260D680097892E6C39F
:1002200094FF500106120982500F120B08500A78F1
:1002300090E6FF125A621260D622900556E0C394EF
:10024000BC506F1230A5900553E0702D9005E4E08E
:10025000FF9005E3E06F6021EF75F007A42457F5E8
:1002600082E43405F583E06403600EEF0475F01456
:10027000849005E4E5F0F080D3900553E07015908C
:1002800005E4E075F007A42457F582E43405F5830E
:10029000E0B4031E1235F39005E3E02414FFA3E05D
:1002A000FEC3EF9E75F01484E5F0D394064003126C
:1002B00035F3227E0A7FD0123A0DEF700302044F0D
:1002C000900AD0E0121F2002EC0102F002030B0A98
:1002D00003932004492803FA30040D31040D32043D
:1002E00017700423710432C20000044F1218D02288
:1002F000900AD1E0FF1218D6900AD3E0FFC2041290
:1003000018DC900AD4E0FF1218E222900AD1E0B47F
:100310000107A3E0FF1218E822900AD1E0B40A17FF
:10032000900B90E0B40108121276E4900B90F0E488
:100330009009E7F0C22222900AD1E064087019A364
:10034000E06007A3E06003D38001C39223D226902C
:100350000AD4E0FF1218EE22900AD1E0640D600387
:1003600002044F900AD0740AF0A3740DF0900BE8C9
:10037000E0900AD2F0900BE9E0900AD3F0900B00E5
:10038000E0900AD4F0E4A3F0A3F07E0A7FD0FD123F
:1003900034B322900AD1E024FE601C24FD602114B5
:1003A000604614604C2406600302044F900AD2E0B9
:1003B000FFD2041218DC22900AD2E0FF1218E222C7
:1003C000900A0CE05401FF900AD2E06F600312180B
:1003D000AC900A0CE030E0067E0E7F8180047E0E39
:1003E0007F40D20C120B5C22900AD2E0FF12114A1D
:1003F00022900AD2E0FF1218F422900AD1E0FFA363
:10040000E0FDA3E0FBA3E0F52F1218FA227B017AAE
:100410000A79D012190022900AD1E0FFA3E0FD1260
:10042000190622900AD1E0FFA3E0FDA3E0FB121918
:100430000C22900BE8E07017900AD1E0B40310A3EF
:10044000E0900A74F0121912229009B17401F0229E
:10045000900BBDE0FF131313541F30E014120C1C5B
:100460005004120C2222900BBFE0FEA3E0FF120CFE
:100470002822900B89E024FE602C14603E14601842
:1004800024037057900B897402F0120C2E900BBD50
:10049000E054F7F0120C3422900B88E014F0E07076
:1004A0005CA37402F022120C3A900B81E0FEA3E0F0
:1004B000FF120C40900B897403F022900B86E054DD
:1004C00001FF33333354F8FF900BBDE054F74FF086
:1004D0007F01120C46E4900B89F02278A6E6FF1209
:1004E0005FF478A6E6FF7DC87C001256E078A6E6A9
:1004F000FF7D0212001678A6E6FF12587E22900BAE
:10050000E8E0B40104120B3822900CECE014601205
:1005100014600F24FE601314600C2402700F120B81
:100520003E22120B4422120B4A22120B50227B0154
:100530007A0B79CA120B98500C900BCA7405F0A371
:10054000E0FF125A62900BEAE020E1031217D42276
:100550007B017A0B79CC120B98500C900BCC740A5F
:10056000F0A3E0FF125A621217DA900BEAE020E1E2
:10057000091217E01217E61217EC1217F21217F809
:100580007B017A0979E7120B981217FE22900BEA89
:10059000E020E11B12180412180A12181012181683
:1005A00012181C12182212182812182E121834228F
:1005B000900B00E0121F2005D00105FE0206770413
:1005C00006980506AC0606C50C061F0F000006DDE2
:1005D000D2A4302E107F9212234E40097D027F1844
:1005E000125A7B8010900B007402F0A3E0FF7D6430
:1005F0007C001256E0900B01E0FF12587E227F0132
:1006000012660D126498EF70107D0F7F01125A7BF5
:10061000900B01E0FF12587E22900B00740FF053F4
:10062000FB7F7D347FAE7E0012089E5007E4FF12F0
:10063000525E80057F0112525E120AD8D29F12626A
:100640006D7F01120ADEE4FF1265EAE4FF1265DC49
:100650007F011265F87F011265F17F321265D512B4
:100660006B8D7F011265DC7D047F13125A7B900B2A
:1006700001E0FF12587E22E4FF1265F1126B8E90AA
:100680000B007405F0A3E0FF7D147C001256E0908F
:100690000B01E0FF12587E221267FE5006900B00FD
:1006A0007406F0900B01E0FF12587E2212589C1243
:1006B0003554122E667F9212234E5021E4900B0C7B
:1006C000F043841022900B05E014F07008900B04A6
:1006D000E0900B00F0900B01E0FF12587E22900B8F
:1006E00000E024F870030207931470030207AC14AF
:1006F00070030207C524FA6074240960030207E24C
:10070000120AE4900BE9E0B40D0F7F011254FC7F54
:1007100001124A79120AEA802C900BE8E0B4011524
:10072000120AEA7D347FAE7E0012089E5017D2086E
:1007300012095880107D187FAE7E0012089E500569
:10074000C208120958E4FF1254FCE4FF124A79125D
:100750000AD8120AF0E4900553F0C29FFF1265DC3C
:10076000900B007410F0A3E0FF12587E22E4FF12F9
:100770000ADEC29412627843FB80900B007408F08A
:10078000A3E0FF7DC87C001256E0900B01E0FF1251
:10079000587E22900B007409F0A3E0FF7DC87C0016
:1007A0001256E0900B01E0FF12587E22900B00746D
:1007B0000AF0A3E0FF7DC87C001256E0900B01E038
:1007C000FF12587E22C2A4E4FF12525E7D347FAE37
:1007D0007E0012089E40057F0112525E900B00744D
:1007E0000BF022E5FB5407B40002E473C403C0E03D
:1007F000741AC0E0C082C083021A00E5FB5407B43B
:100800000102E473C403C0E0741AC0E0C082C08374
:10081000021A08E5FB5407B40202E473C403C0E003
:10082000741AC0E0C082C083021A10E5FB5407B4FA
:100830000302E473C403C0E0741AC0E0C082C08342
:10084000021A18E5FB5407B40402E473C403C0E0C1
:10085000741AC0E0C082C083021A20E5FB5407B4BA
:100860000502E473C403C0E0741AC0E0C082C08310
:10087000021A28E5FB5407B40602E473C403C0E07F
:10088000741AC0E0C082C083021A30EFC403901A09
:1008900000739090E10207E390C7D80207E390D776
:1008A0004E0207E390B2810207E390D7850207E387
:1008B00090C3B202082B908FF902081390F29502B0
:1008C00007E390E8F002081390F31F0207E390CDCE
:1008D0003402082B90A58C0207E390EC980207E302
:1008E00090D00602082B90A9390207E390D01B0292
:1008F000082B90CE9F02082B90AFFE02081390EEBB
:10090000420207FB90969102082B90C72F0207E343
:1009100090ED7D0207E390EC2302081390A54E02B0
:10092000082B90C9B502082B90C6E502082B90CC85
:10093000E802082B90F2A10207E390F29B0207E382
:1009400090D0450207E390F1F60207E390D86E02DB
:1009500007E390D0890207E390F0550207E3908403
:10096000A802085B90C20802082B90BA7A0207E33B
:1009700090EF580207FB90D04502082B90BC35023F
:10098000082B90D03702082B90D06102082B90D012
:100990006702082B90B9D402082B90F1340207E3C8
:1009A00090EA8E0207E390BAA502082B909380028A
:1009B000082B90C60602082B90D6FE02081390C69C
:1009C0009302082B90C77102081390D1D10207FB44
:1009D00090A0BD0207FB90B5C90207E390D8D902E9
:1009E00007E390C5AF02082B909C9C02082B90B2A5
:1009F000FB0207E390AC2902082B90EA5A0207E3B6
:100A000090D9880207FB90ED4102081390ACE802F0
:100A1000082B90DA120207E390C25202082B90B81A
:100A20004A02082B90B2A302082B90D10B02082B8C
:100A300090F0CD0207E390E7D70207E390F13F0281
:100A400007E390DF790207E390E7A402081390F22E
:100A5000720207E390ECB50207FB90937D02085BFE
:100A600090CC5802082B90E7600207E390BA090285
:100A7000082B90B3C002082B90AFFC0207E39091C3
:100A80002702082B90983602082B908FB102082B72
:100A900090D13702082B90A0F802082B90C0A70233
:100AA000082B909E8B02082B909FC802082B90C2A7
:100AB000BF02082B90ABC702082B90A81C02082B82
:100AC00090AFF302082B90B61A02082B90EADD02D1
:100AD00007FB90BA3D02082B90DFA30207E390EAE0
:100AE000FA0207FB909DE802082B90A2290207E377
:100AF00090F1760207E390EFFD0207E390F1280200
:100B000007E390D13E02082B90AD4602082B90D10E
:100B10003B02082B90ADFC02082B908EAE02085BC6
:100B2000908FE602085B90D05302082B90D8700299
:100B3000081390E9F402081390ED030207E390C94B
:100B4000BA0207E390C7840207E3908E3902082BAC
:100B500090DF0B02081390C79B02082B90BFC102C5
:100B600007FB908EC002081390F2B80207FB90D0EA
:100B70003002082B90B0E402082B90C12002082B11
:100B800090D1AF02081390927002085B90918D0291
:100B9000085B90F2AC0207FB90C96002082B90BE84
:100BA0000B0207FB9093A702085B90E0670207FB2C
:100BB00090CAA802082B908F3802085B908A88029E
:100BC000085B9086B902085B908C1702085B9087DF
:100BD0007702085B90936A02085B90D7660207FB76
:100BE00090CD6C0207FB909E420207FB90D2EE0272
:100BF00007FB90E92C02081390EF9E0207FB90F28E
:100C0000D60207FB90EA660207FB90E79C0207FB0F
:100C100090E9900207FB90E5AC0207FB90DFF7023A
:100C200007E390DD420207E390A0BC0207E390F1E6
:100C3000970207E390E3EB0207E390C62D0207E378
:100C400090E8B70207E390DECD0207E390F241029D
:100C500007E390BB930207FB90978D0207FB90B1CF
:100C6000320207FB90BD740207FB90AE5302082BC3
:100C700090B5FA0207FB909BAD0207FB90AE9D0278
:100C800007FB9098FC0207FB908CB002082B90A801
:100C9000300207FB90ADBB0207FB90B6B90207FB21
:100CA00090CD000207FB90D8F00207FB90C77F02AF
:100CB00007FB90CE400207FB90C1650207FB90C284
:100CC000750207FB90C58E0207FB90C2FB0207FB73
:100CD00090E0C80207E390E89C0207E390CD16027B
:100CE000082B90E1B90207E390932702085B90CFAD
:100CF000C60207E390DD150207E390E6000207E372
:100D000090E5DF0207E390E3320207E390D1990216
:100D100007E390BDFC02082B90B40602082B90CD8F
:100D20002502082B90938D02085B90800002085BDF
:100D300090935702085B90BED502082B90EC5602A8
:100D400007E39090B202085B90881D02085B9090C8
:100D50005B0207FB90D14802082B908E6602085B6D
:100D600090C2E302082B90C5D60207E390E37C0211
:100D700007E390DF9E02081390DFE602081390CE8F
:100D80002202082B90F2DA0207FB90D12702082BEF
:100D900090EBB30207E390D4D50207E390EEF6029E
:100DA00007E390CE1602082B90C32902082B90C9A6
:100DB0001D0207E390D9760207E390CB1902082BB6
:100DC00090B04402082B90A5CE02082B90AA3802BE
:100DD000082B90AEAA02082B90CFFF02082B90B8E8
:100DE000C002082B90EB830207E390CBB00207FB15
:100DF00090DB440207FB90E59B0207E390CF3502AE
:100E0000082B90C4DA02082B90ED410207E390DA38
:100E1000450207E390CD450207E390C5CC02082BBD
:100E200090ED690207E390EF160207E3908629022E
:100E3000082B90F2CA0207FB90C59202082B90C0C3
:100E40002B02082B90BC370207FB90DFCD0207E393
:100E500090D6A60207E390D6DE0207E390F2A7023F
:100E600007E390F2AD0207E390F2B30207E390F2DA
:100E7000B90207E390F2BF0207E390F2C50207E36D
:100E800090F2CB0207E390F2D10207E390F2D7028F
:100E900007E390C55602082B90C4BB02082B90E8CC
:100EA0002D0207E390C57402082B90A3050207FBEF
:100EB00090C8730207FB90E5010207FB90F14A021C
:100EC00007E390E16B0207E390CD8802082B90E2E4
:100ED000C30207E390B3EE0207E390AC8A02082B4B
:100EE00090D0EB02082B90D0EF02082B90D0F302A9
:100EF000082B90D0F702082B90D0FB02082B90E42F
:100F0000350207E390D0FF02082B90D10302082B93
:100F100090EC6C0207E390EAD102081390E14B02D7
:100F20000813909D4202082B909B3C02082B90AF27
:100F3000A202082B90CE5D02082B909BF402082B96
:100F40009093B302085B90B21302082B90CCC802B6
:100F5000082B90C29B02082B90D3250207E390CB6D
:100F60007302082B90B80E02082B90C63F02082B84
:100F700090D0D702082B90D0E302082B90D0DB0250
:100F8000082B90D0DF02082B90D0E702082B90CFDF
:100F90002C02082B9093CE02085B90D0450207FBF1
:100FA00090E9CE0207FB90E2540207FB90F2860222
:100FB00007FB908E600207FB9093E002085B90F0C5
:100FC000470207E390E9560207E390E6420207E38F
:100FD00090CA3002082B90DBD30207FB90C4780242
:100FE00007E390C82B0207E390A8A30207E390B49D
:100FF000650207E390BE9E0207FB90EFAF0207FB7E
:1010000090ED550207E390D5880207E390C15002A6
:1010100007E390BA110207E390C6DA0207E390A74C
:10102000720207E390A80C0207E390D4980207E34A
:1010300090DD6F0207E390BCDF0207E390DB3F0225
:1010400007E390C4D00207E39091DF02085B908F22
:10105000760207E390DE4C0207E390D9420207E3F1
:1010600090DBD00207E390B86B0207E390D3A402B1
:1010700007E390EE170207E390DE770207E3909113
:101080006402085B90E6C50207E390939B02085B4D
:1010900090A7370207FB90F17D0207FB90EC8102DD
:1010A00007FB90F1710207FB90EEC60207E390CABE
:1010B000560207E390F0E70207E390ED170207FB03
:1010C00090F0390207E390C8D802082B90F2520240
:1010D00007E390F18C0207E390F0A50207FB90EF85
:1010E000F00207FB90E9ED0207FB90ECCE0207FB54
:1010F00090F0870207FB90F0960207FB90F1CE027A
:1011000007E390F1DE0207FB90EFE00207FB90EBB4
:101110000B0207E390EB230207E390EB3B0207E3AC
:1011200090EB530207E390E9BE0207E390E9D8028F
:1011300007E390E9F20207E390EA0C0207E390EA82
:10114000260207E390E98A0207E39092430207E34D
:1011500090D10E0207FB90ED470207FB90D51802D5
:1011600007FB90F2A60207FB90EDF30207E390D98C
:10117000DE0207E3909DF20207E3909F810207E3FE
:1011800090F2540207FB90C8EB0207FB90CAA3023F
:1011900007E390A4380207E3909FFE0207E390F371
:1011A000390207E390F33A0207E3909FFF0207E357
:1011B00090F33B0207E390DB700207E390DC5D02F3
:1011C00007E390BFE20207E390AB8A0207E390EDEA
:1011D0002D0207E390E7F40207E39098C20207E3C9
:1011E00090E4590207E390E47D0207E390E4A10252
:1011F00007E390E4C50207E390E4E90207E390ED1A
:10120000E00207E390EFB20207E390AC1C0207E3B1
:101210009091B602085B90D2A40207E390E7BA026D
:1012200007E390910F02085B90904D02085B90EAF3
:10123000E202081390D06D02082B90F2940207FB93
:1012400090F1950207FB90EFC00207FB90DEB90218
:1012500007FB90F01E0207FB90C1EF0207FB90E135
:10126000110207FB90E7030207E390F0F40207E3A3
:1012700090DADD0207E390CC910207FB90EBA50228
:1012800007FB90EA2A0207FB90D5C30207E390D937
:101290000E0207E390C2C402081390994D0208138E
:1012A00090C65B02082B90C67702082B90CCB80240
:1012B000082B90C9CA02082B90CABB02082B90B415
:1012C0008E02082B90BC0502082B90CD9502082BAE
:1012D00090C89002082B90CB3D02082B90CE7E0246
:1012E000082B90CE8902082B90CE9402082B90BF39
:1012F0000002082B90BF2B02082B90CF7402082B02
:1013000090A33F02082B90BE2802082B90BF5602E4
:10131000082B90CAE102082B90CEE702082B90CF51
:10132000A802082B90CFB802082B90CFC802082B38
:1013300090CAF402082B90CEF102082B90CFB00295
:10134000082B90CFC002082B90CFD002082B90CE54
:10135000C902082B90C22D02082B90C74D02082B02
:1013600090D0AF02082B90D14302082B90C76702A0
:10137000082B90D14502082B90D11302082B90C462
:101380005902082B90CED302082B90BBA402082B45
:1013900090CB6102082B90D14202082B90C78102AA
:1013A000082B90CDC902082B90CACE02082B90942E
:1013B0008C02082B90C47A02082B90CB4F02082B8A
:1013C00090CF7D02082B90CEDD02082B90A8FB0267
:1013D000082B90D03E02082B90CC7802082B90A4CA
:1013E000CB02082B90CDD602082B90D0B502082B4B
:1013F00090B37902082B90C14702082B90B757028F
:10140000082B90C30602082B90C90602082B90CD2A
:10141000F002082B90C86002082B90D0A302082B82
:1014200090CA6C02082B90D11B02082B90C719029E
:10143000082B90C6FF02082B90C6CA02082B90BB4F
:101440004002082B90C7B502082B90CE4602082B0D
:1014500090CDFD02082B90C87802082B90D0A902ED
:10146000082B90CA8002082B90D11702082B90C736
:101470003302082B90CE3A02082B90D12302082B7E
:1014800090D11F02082B90C7CE02082B90D0BB0230
:10149000082B90D14602082B90CCA802082B90D0A4
:1014A0004C02082B90D14702082B90B55602082B0E
:1014B00090CC0302082B90B8FA02082B90C8EF02D8
:1014C000082B90CF5902082B90CF6202082B90CFA7
:1014D0005002082B90CF6B02082B90A44802082BD7
:1014E00090D14102082B90CB2B02082B90BCC0025C
:1014F000082B90CC8802082B90CC9802082B90CE19
:10150000B502082B90CF9802082B90CEBF02082B73
:1015100090CFA002082B90CA4402082B90B7190262
:10152000082B90D08B02082B90D07F02082B90D0F4
:101530009702082B90C41702082B90CA5802082B58
:1015400090D10F02082B90D07902082B90D09102F5
:10155000082B90D08502082B90D09D02082B90C4B8
:101560003802082B90CDA202082B90CDAF02082B99
:1015700090CDBC02082B90D14402082B90C7E70203
:10158000082B90CEFB02082B90D0C102082B90CFE5
:10159000D802082B90CFE002082B90CFF002082B46
:1015A00090CFE802082B90CC1402082B90CC250297
:1015B000082B90CC3602082B90CC4702082B90C900
:1015C0001D02082B90C8A802082B90C8C002082B47
:1015D0009092B302085B90DD2A02081390E1B702F3
:1015E00007FB90BE680207E390F10E0207E390F15B
:1015F000EC0207E390EC3F0207E390B6380207E302
:1016000090E5790207E390DD2E0207FB90EF7C0264
:1016100007FB90E2530207E390937C0207E390EF0D
:10162000560207E390EA740207E390CC670207E3EF
:1016300090F1A00207FB90AD400207E390F00F028B
:1016400007E390C03E0207E390ED2A02081390EFF3
:10165000C202081390C7C102081390EEA702081334
:1016600090DCFF02081390A22302081390BA4202F2
:1016700007FB90E4470207FB90DAFB0207FB90EFC1
:10168000AC02081390C0F702081390D6C8020813E2
:1016900090B4CF02081390EC0602081390F279027E
:1016A00007E390DCD402081390DAEE02081390EFFF
:1016B000A602081390AEE002081390E8CE0207FBE2
:1016C00090E9700207E390D5FC0207E390CB850216
:1016D000082B90CB9702082B90CBA902082B90BA2D
:1016E0007102082B90C16E02082B90C19502082B45
:1016F00090CBBB02082B90CBCD02082B90CBDF0206
:10170000082B90F00F0207FB90F1160207FB90C424
:10171000060207FB90DCB90207E3908E1702085B14
:1017200090ED4C02081390CA080207E390B7130229
:1017300007E390DA0302081390EBFA0207E390E262
:10174000EE0207FB90EAC00207FB90D12B02082BA8
:1017500090D12F02082B90D05A02082B90D133023F
:10176000082B90CF0F02082B90C5E902082B90C4DC
:101770009B02082B90C53702082B90F26A0207E300
:1017800090E82E0208139085A70207E390E11A0261
:1017900007E390F1890207FB90BE070207E390AFD1
:1017A000FF02081390A6310207E39097D20207E3E5
:1017B00090BF850207E390D7B60207FB90F1E202E3
:1017C00007E390F27F0207FB90E29E0207E390F2AC
:1017D000000207E390E5DD02081390C83002082BF1
:1017E00090E7E30207FB90EF6A0207FB908C9902F7
:1017F00007E390C1BC02082B9093BE02085B90C81F
:10180000CD0207E390E2B702081390E5F702081350
:1018100090F02D0207FB90E1800207FB90C8480280
:10182000082B90BBD502082B90EE580207FB908E38
:10183000F402085B90E2880207FB90EC9302081325
:1018400090C5D902081390EE160207FB90F22F0202
:1018500007E390EE1F02081390D49702081390EC50
:101860004B0207FB90CF110207FB90B1AD020813AA
:1018700090924A0207FB908D0402085B90E6A50255
:1018800007E390E22D0207E390E4770207FB90DE86
:10189000780207FB90D5B70208139098230208132B
:1018A00090DAB10207FB90C6880207FB90D635029A
:1018B00007E390DE370207FB90AEE90207E3909B57
:1018C000740207E39093DA02085B90BF270207E3F4
:1018D000908C9602085B90930C02085B90901A0221
:1018E000085B90913A02085B90929202085B909399
:1018F000C802085B9093D402085B90C7F90207FB0B
:10190000909CF90207FB9089FD02085B908FAF0263
:10191000085B90825002082B90F24A0207E390F293
:10192000380207E390DEF80207E390C6AF02082B07
:1019300090E6E40207E390F2800207E390F10102EF
:1019400007E390CE2E02082B90D07302082B90A4B0
:10195000E50207E390AAF70207E390E0F10207E34C
:1019600090C9DA0207FB90AF7F0207FB90D7F30222
:1019700007E390E2790207E390E1920207E390EF38
:10198000C502081390F2DD0207FB90C0DB0207FBE3
:1019900090E0D90207FB90B2090207FB90A41E0257
:1019A00007FB90CFDF0207FB90F1D40207FB8B2FE0
:1019B0008A3089317F781257C3787DE6547FF608E4
:1019C000E6547FF608E6547FFFF6787DE6AB2FAA53
:1019D00030A931121BB774012531F531E43530F5EA
:1019E0003008E6AB2FAA30A931121BB7740125319C
:1019F000F531E43530F530AB2FFAA931EF021BB7E2
:101A000053FBF843FB0022FF53FBF843FB0122FF8B
:101A100053FBF843FB0222FF53FBF843FB0322FF77
:101A200053FBF843FB0422FF53FBF843FB0522FF63
:101A300053FBF843FB0622E709F608DFFA8046E786
:101A400009F208DFFA803E88828C83E709F0A3DF81
:101A5000FA8032E309F608DFFA8078E309F208DF5A
:101A6000FA807088828C83E309F0A3DFFA806489AE
:101A7000828A83E0A3F608DFFA805889828A83E0AD
:101A8000A3F208DFFA804C80D280FA80C680D4802E
:101A90006980F28033801080A680EA809A80A880D6
:101AA000DA80E280CA803389828A83ECFAE493A3E5
:101AB000C8C582C8CCC583CCF0A3C8C582C8CCC574
:101AC00083CCDFE9DEE7800D89828A83E493A3F685
:101AD00008DFF9ECFAA9F0EDFB2289828A83ECFA9F
:101AE000E0A3C8C582C8CCC583CCF0A3C8C582C852
:101AF000CCC583CCDFEADEE880DB89828A83E4938D
:101B0000A3F208DFF980CC88F0EF60010E4E60C3CD
:101B100088F0ED2402B4040050B9F582EB2402B43D
:101B2000040050AF2323458223901A8773C2D53017
:101B3000F707B2D563F0FF05F030E70CB2D5F40437
:101B40008463F0FF05F080018430D502F40422BBE9
:101B5000010689828A83E0225002E722BBFE02E36B
:101B60002289828A83E49322BB010CE58229F582D3
:101B7000E5833AF583E0225006E92582F8E622BBA8
:101B8000FE06E92582F8E222E58229F582E5833A1C
:101B9000F583E49322BB010989828A83F8E028F067
:101BA00022500327F722BBFE05F8E328F3228A839D
:101BB0008982F8E4932822BB010689828A83F02275
:101BC0005002F722BBFE01F322F8BB010DE582298A
:101BD000F582E5833AF583E8F0225006E92582C8CC
:101BE000F622BBFE05E92582C8F222EF8DF0A4A8FB
:101BF000F0CF8CF0A428CE8DF0A42EFE22BC000BDA
:101C0000BE0029EF8DF084FFADF022E4CCF875F032
:101C100008EF2FFFEE33FEEC33FCEE9DEC98400511
:101C2000FCEE9DFE0FD5F0E9E4CEFD22EDF8F5F0D7
:101C3000EE8420D21CFEADF075F008EF2FFFED33DF
:101C4000FD4007985006D5F0F222C398FD0FD5F05D
:101C5000EA22C5F0F8A3E028F0C5F0F8E582158285
:101C600070021583E038F022BB010A89828A83E082
:101C7000F5F0A3E022500687F009E71922BBFE0722
:101C8000E3F5F009E3192289828A83E493F5F0747D
:101C9000019322BB0110E58229F582E5833AF583A1
:101CA000E0F5F0A3E0225009E92582F886F008E685
:101CB00022BBFE0AE92582F8E2F5F008E222E5837C
:101CC0002AF583E993F5F0A3E99322BB010DC582C0
:101CD00029C582C5833AC583021C525011C5822989
:101CE000F808E5F026F618F5F0E58236F622BBFE98
:101CF00011C58229F808E225F0F5F0F218E23582E4
:101D0000F222F8E58229F582E5832AF583740193AE
:101D100025F0F5F0E4933822BB010A89828A83F02A
:101D2000E5F0A3F0225006F709A7F01922BBFE0642
:101D3000F3E5F009F31922F8BB0111E58229F582D8
:101D4000E5833AF583E8F0E5F0A3F0225009E925B0
:101D500082C8F608A6F022BBFE09E92582C8F2E592
:101D6000F008F222EF2BFFEE3AFEED39FDEC38FCE5
:101D700022E88FF0A4CC8BF0A42CFCE98EF0A42CEC
:101D8000FC8AF0EDA42CFCEA8EF0A4CDA8F08BF038
:101D9000A42DCC3825F0FDE98FF0A42CCD35F0FC36
:101DA000EB8EF0A4FEA9F0EB8FF0A4CFC5F02ECD02
:101DB00039FEE43CFCEAA42DCE35F0FDE43CFC22E7
:101DC00075F008758200EF2FFFEE33FECD33CDCCDA
:101DD00033CCC58233C5829BED9AEC99E58298405D
:101DE0000CF582EE9BFEED9AFDEC99FC0FD5F0D63A
:101DF000E4CEFBE4CDFAE4CCF9A88222B800C1B964
:101E00000059BA002DEC8BF084CFCECDFCE5F0CBA1
:101E1000F97818EF2FFFEE33FEED33FDEC33FCEBDA
:101E200033FB10D703994004EB99FB0FD8E5E4F995
:101E3000FA227818EF2FFFEE33FEED33FDEC33FC82
:101E4000C933C910D7059BE99A4007EC9BFCE99A76
:101E5000F90FD8E0E4C9FAE4CCFB2275F010EF2FBB
:101E6000FFEE33FEED33FDCC33CCC833C810D707BB
:101E70009BEC9AE899400AED9BFDEC9AFCE899F8F6
:101E80000FD5F0DAE4CDFBE4CCFAE4C8F922EF5B3D
:101E9000FFEE5AFEED59FDEC58FC22E8600FECC352
:101EA00013FCED13FDEE13FEEF13FFD8F122E860F3
:101EB0000FEFC333FFEE33FEED33FDEC33FCD8F10F
:101EC00022E493F8740193F9740293FA740393FB78
:101ED00022F5F0C582A4C582C5F0C583A42583F58B
:101EE0008322A42582F582E5F03583F58322FAE684
:101EF000FB0808E6F925F0F618E6CA3AF622FAE6F3
:101F0000FB0808E625F0F9F618E63AFAF622E0FBB7
:101F1000A3E0FAA3E0F922EBF0A3EAF0A3E9F022B0
:101F2000D083D082F8E4937012740193700DA3A350
:101F300093F8740193F5828883E473740293686064
:101F4000EFA3A3A380DFD083D082F8E49370127450
:101F50000193700DA3A393F8740193F5828883E431
:101F600073740293B5F0067403936860E9A3A3A3A6
:101F7000A380D88A838982E473011F0E430C00007A
:101F80000000420C90006E410A9200410A99004103
:101F900005E3004105E40041062B0041062C004109
:101FA000055400C1B0C1B7C131430C45FF4D8E434C
:101FB0000C3FFF4D8E430C33FF3A8F430C48FF4CD0
:101FC000CE430C42FF4CCE430C3CFF4C8E430C21C5
:101FD000FF4CCE430C09FF4CCE430C2DFF4CCE439F
:101FE0000C57FF4CCE430C4EFF4CCE430C5AFF4CCB
:101FF000CE430C51FF4CCE430C5DFF4CCE430C54F2
:10200000FF4CCE430C36FF4D0E430C15FF4D0E43D7
:102010000C4BFF4D0E430C30FF4D0E430C39FF4D62
:102020000E430C18FF4D0E430C03FF4D4E430C06A0
:10203000FF4D4E430C0CFF4D4E430C0FFF4D4E43D6
:102040000C12FF4D4E430C1BFF4D4E430C1EFF4D1B
:102050004E430C24FF4D4E430C27FF4D4E430C2A9C
:10206000FF4D4E410CDA00410CE900410CE3004108
:102070000CC600410CCF00410CB700410CD500410B
:102080000CD800410CCA00410CD900410CCC0041D5
:102090000CDB00410CCE00410CDD00410CBF0041C7
:1020A0000CEA00410CD600410CDE00410CC100419D
:1020B0000CB500410CB600410CB800410CB9004110
:1020C0000CBA00410CCB00410CCD00410CD10041B9
:1020D0000CD300410CD400604A0789202020202026
:1020E0002020202020202020202020192020002017
:1020F000200D0820202020002020202020205820F3
:10210000000000000000001002000100000080003C
:1021100011000180400008010080800000400000A4
:10212000010000200C607E062E0000005DC00062F1
:102130006AAB0A6AA83437004000C000639301000C
:1021400080010080039080190C80080104000000C9
:1021500000000000C6000000000000101010100079
:1021600001F8000000000000002F0C00000000003B
:1021700000020000056000000000000000000000F8
:10218000000000000000000000000000000000004F
:1021900000000000000000000000000000600000DF
:1021A00000001FF8000100410A6E00410A6F014162
:1021B0000A7000410A6C40410A6D004109B6FF41B6
:1021C00009AFFF4109B7004109B4004109C5004EFC
:1021D00009CA8440849084B08100830084C086C092
:1021E0004109AD004109AE00410B0FFF410B0D004D
:1021F000410CED00410B5C06410B5D00410B5E01A3
:10220000410B5F01420B570600410AC6FF410D1CFE
:102210001F410D261F420BA6000042094E0000423E
:10222000095F0000410961004C09622D2D2D2D2D03
:102230002D2D2D2D2D2D0041094D0041094B004123
:102240000D2A00410BF42A410BF62A410BF50841F7
:102250000BF708410BC645410BC700410BC828418D
:102260000BC345410BC400410BC528410C721D41F5
:102270000C741D815D00815100815700815800431D
:102280000C75000000410CA100C1C4410CA000412C
:102290000D3C00420B930000410B9514410B980636
:1022A000410B9A004109250A4109270041093C00D8
:1022B00041094A004109190041091B00410B400036
:1022C000410CA200410CA300410D3E004108B700A3
:1022D0004108B8004108B900C12A4108E40060295A
:1022E000097E594F55522043484F4943453A2020D3
:1022F00020200355502F444F574E20204C45465424
:102300002F5249474854204B4559004209A7000025
:10231000410D3F00470AD700000000000000C12126
:10232000C122C123410ADE00410ADF00410ACF0079
:102330004109E5004109E6004109E700410D43FF7D
:10234000410C8F03420C8D000A410D450000BF80F7
:1023500005D2800223F9BF8105D2810223F9BF8211
:1023600005D2820223F9BF8305D2830223F9BF84F9
:1023700005D2840223F9BF8504D285807CBF9004F6
:10238000D2908075BF9104D291806EBF9204D29298
:102390008067BF9304D2938060BF9404D294805925
:1023A000BF9504D2958052BF9604D296804BBF97BA
:1023B00004D2978044BFA004D2A0803DBFA104D224
:1023C000A18036BFA204D2A2802FBFA304D2A380D3
:1023D00028BFA404D2A48021BFA504D2A5801ABF1F
:1023E000B004D2B08013BFB104D2B1800CBFB2042C
:1023F000D2B28005BFB302D2B3BF800630800302E1
:102400002492BF8106308103022492BF820630826B
:1024100003022492BF8303208378BF840320847245
:10242000BF850320856CBF9003209066BF91032079
:102430009160BF920320925ABF9303209354BF949C
:102440000320944EBF9503209548BF9603209642E3
:10245000BF970320973CBFA00320A036BFA1032055
:10246000A130BFA20320A22ABFA30320A324BFA49C
:102470000320A41EBFA50320A518BFB00320B012DF
:10248000BFB10320B10CBFB20320B206BFB3063008
:10249000B303D38001C3228B368A378938E53A5497
:1024A000079006B6F0900001121B68FF9006B6E098
:1024B000FEC374089EFCEFA804088002C333D8FC56
:1024C000FF900002121B68FCA806088002C313D804
:1024D000FC2F900002121BC9900001121B68FF9094
:1024E00006B6E0FEEFA806088002C313D8FCFF1270
:1024F0001B4FFCC374089EFEECA806088002C33381
:10250000D8FC2F900001121BC9121B4FFF9006B67A
:10251000E0FEEFA806088002C313D8FC121BB7E543
:102520003AC39410401CAB36AA37A938121B4F90FF
:102530000002121BC9900001E4121BC9E4121BB770
:102540008026E53AC39408401FAB36AA37A93890D5
:102550000001121B68900002121BC9121B4F900051
:1025600001121BC9E4121BB7ED5407FFC374089F87
:10257000FF74FFA807088002C313D8FC9006B6F0CA
:10258000EDC394104012AB36AA37A938121B4FFF87
:102590009006B6E05F021BB7EDC394084017AB3658
:1025A000E5382401F9E43537FA121B4FFF9006B6DF
:1025B000E05F021BB7AB36E5382402F9E43537FAA1
:1025C000121B4FFF9006B6E05F121BB7228F518D92
:1025D000528B53755A03900CA8E551F0E55A7002DE
:1025E000C1D3900CA8E07002C1D3E4F0155AE559AC
:1025F00064066005E559B4070585525B8003755B89
:1026000001E55860D7900CA8E070D1E55B60CD1271
:102610005D8FAF511248005006900CA8E551F0E5CF
:102620005964066006E55964077024AF57124800E4
:102630005008900CA8E551F080020557A854E6FF19
:102640001248005008900CA8E551F080020554E5AE
:10265000596403600BE55964046005E559B4050D40
:10266000AF571248005006900CA8E551F0E55964A8
:10267000026011E5596403600BE55964046005E5E7
:1026800059B4050FAD54AF521258D85006900CA84B
:10269000E551F0E559B4040FAD55AF531258D85079
:1026A00006900CA8E551F0E559B4050E755F01AB35
:1026B00056AD53AF5112433B8003126480E559B4C9
:1026C00007057F0A124BAE900CA8E06002C1051509
:1026D0005BC10522C0E0C0F0C083C082C0D075D00D
:1026E00010E58F540FAD8EF563EDF564E58F54F072
:1026F00075F010A4FFAD9BE5F0F565EF4DF566E5CF
:10270000EF20E573302439D3E56494C0E563940287
:102710005016E56694C0E5659402500712582105ED
:102720006980451251FB8040D3E56694C0E565940D
:10273000025004C2248005056912582105698028C9
:10274000D3E56494C0E5639402501AE56694C0E54D
:1027500065940250028001C340070569125821D2D6
:1027600024056980031251FBE569640C705D7FD11B
:102770007E0A12606E8054E5EF30E54CE569B40DD9
:102780000ED3E56494C0E56394025003202426E54B
:1027900069B40C0ED3E56494C0E563940250033031
:1027A0002413E569B40C21C3E56494C0E563940285
:1027B0004016302413E56B4480F567E56A6440F504
:1027C00068D2251251FB80031251FBD0D0D082D0A9
:1027D00083D0F0D0E032CDEFCDCCEECCEC25E024B0
:1027E000A0FF7BA08D507D01124E0E126262500A36
:1027F000900C61E04401F07F002278A0E6FF2222E5
:102800008F458C468D478B4874F62547F54774FFF6
:102810003546F546E549131313541FFFC374029F51
:10282000FB7A00AE46AF477C007D03121BEBEF2B1B
:10283000FFEA3EFEE5495407FDE545A8050880028C
:10284000C333D8FCF9E548A805088002C333D8FC97
:10285000FC742E2FF58274063EF583E0FBECF4FA4F
:10286000EB5AFBE95C4BF0C374089DFBE548A803F9
:10287000088002C313D8FCFC6027EF1F70011EE51F
:1028800045A803088002C313D8FCF9742E2FF582E3
:1028900074063EF583E0FDECF4FBED5BFDE95C4D79
:1028A000F0303956E4FF8547828546837403121E53
:1028B000D1E5822FF582E43583F583E582242EF578
:1028C00082E5833406F583E0FE74822FF8A6060FB6
:1028D000BF03D37B82E547240AF54EE43546F54D28
:1028E0007D037FB0124AFF9006F3EFF0900CE5E015
:1028F00070089006F3E0900CE5F02230780020207C
:1029000020003120002F003220003320003420002E
:102910000300210DDE050D310E32050E320E32059B
:102920000F330E320510350E320511360E320512F8
:10293000370E320100380E380100260E3E040039F1
:102940000E4404003A0E4404003B0E4404003C0EC6
:102950004404003D0E4404003E0E4404003F0E4477
:102960000200410E4A0200420E500200450E56057A
:10297000130A0E320514090E3205150B0E32020031
:10298000490E5C02004A0E6202004B0E68020046CD
:102990000E6E0200470E740200480E7A02004C0EC2
:1029A0008002004D0E8602004E0E8C0100610E92D8
:1029B0000100620E980300660E9E0100670EA404DB
:1029C00000680EAA0400690EB00300010EB60400F0
:1029D000680EAA0400690EB00300010EB62F0F1096
:1029E00011171718171817191A1B1C171D1E1F1F50
:1029F0001F172B432C900BBB7401F0E4900BB7F026
:102A0000126AABBF04047F0180027F00900BBCEF11
:102A1000F0900BBA7406F0126A9FEF121F202A4141
:102A2000012A5F032A7A042A9F052A37062A840787
:102A30002ABA0800002AE2900BB874DCF0120A6C83
:102A400022900BB87410F0900BE9E0FF640360086B
:102A5000EF64086003022AE8900BB87456F02290E5
:102A60000BB87411F0900BE9E0FF64036005EF64AC
:102A7000087075900BB87455F022900BB87452F032
:102A8000120A7222900BB87420F0900BE9E0FF64F8
:102A9000036005EF64087050900BB87450F02290FA
:102AA0000BB87421F0900BE9E0FF64036005EF645C
:102AB000087035900BB87451F022126A9FEF601BBA
:102AC0009008B5E030E714120982500F900BBCE07B
:102AD0006009126A9F900BB8EFF022900BB8740C4B
:102AE000F022900BB874FFF0228E2D8F2E8C2F8D3C
:102AF00030E49006ACF020390261D1125BB5EF6092
:102B0000047F0180027F00BF01089006AE740AF0C6
:102B100080069006AE7416F0126B7B9006ADEFF057
:102B20007F0F125F7C9006AEE0FF7E00C3E52E9F14
:102B3000E52D9E50048E2D8F2ED3E5309433E52F56
:102B400094004006752F0075303374F6252EF52E4F
:102B500074FF352DF52D74F62530F53074FF352FC3
:102B6000F52F852E31D3E5319530E4952F504C90DB
:102B700006ACE0704675F003E53190062E121EE2B9
:102B8000E07882F675F003E53190062F121EE2E040
:102B900008F675F003E531900630121EE2E008F603
:102BA0007B82E531240A754D00F54E7D037FB0121E
:102BB0004AFF9006ACEFF0053180AA900CE5E0707A
:102BC000089006ACE0900CE5F09006ADE0FF125FD7
:102BD0007C22C0E0C0F0C083C082C0D075D010E5B8
:102BE000D954F8FF131313541FB41A00400281AADA
:102BF000902BF625E073812A812F81348139813E23
:102C000081438148814D81528157815C8161816618
:102C1000816B81708175817A817F81848189818EC8
:102C200081938198819D81A281A71245DF807B12CB
:102C30005A9480761260888071125F31806C125FC6
:102C4000408067125D018062125F40805D125AAD64
:102C50008058125AC68053125F40804E125A4880E4
:102C600049125ADF8044126AC3803F125D13803AD2
:102C7000126AC38035125D138030126AC9802B122C
:102C80005D258026126AC98021125D25801C1200F4
:102C90000E8017126ACF8012125DF4800D126ACF77
:102CA000800812000E800312000ED0D0D082D08394
:102CB000D0F0D0E0328D2FEF90638D93FEB480057D
:102CC000D280022D81EEB48105D281022D81EEB435
:102CD0008205D282022D81EEB48305D283022D813A
:102CE000EEB48405D284022D81EEB48505D285022E
:102CF0002D81EEB49005D290022D81EEB49104D2D4
:102D000091807EEEB49204D2928076EEB49304D297
:102D100093806EEEB49404D2948066EEB49504D29F
:102D200095805EEEB49604D2968056EEB49704D2A7
:102D300097804EEEB4A004D2A08046EEB4A104D297
:102D4000A1803EEEB4A204D2A28036EEB4A304D297
:102D5000A3802EEEB4A404D2A48026EEB4A504D29F
:102D6000A5801EEEB4B004D2B08016EEB4B104D289
:102D7000B1800EEEB4B204D2B28006EEB4B302D289
:102D8000B3EF90639193FF1260A2EFD3952F4003AE
:102D9000D38001C322900BBB7401F0E4900BB7F019
:102DA000126AABBF04047F0180027F00900BBCEF6E
:102DB000F0900BBA7406F0126A9FEF14604414602E
:102DC0006714604914601F147079900BB87410F088
:102DD000900BE9E0FF64036005EF6408706B900BF3
:102DE000B87456F08063900BB87411F0900BE9E062
:102DF000FF64036005EF6408704F900BB87455F0E2
:102E00008047900BB87452F0120A72803C900BB855
:102E10007420F0900BE9E0FF64036004EFB408292C
:102E2000900BB87450F08021900BB87421F0900B87
:102E3000E9E0FF64036004EFB4080E900BB874512E
:102E4000F08006900BB874FFF0900BE8E0B4051525
:102E5000126A9FEF25E02494F582E43457F583E469
:102E600093900BB8F022E49006ACF0120934EFC056
:102E7000E012093ACDEFCDD0E0FF1209409006AD47
:102E8000EFF0D2011209469202900AE0E06012903F
:102E90000AE4E09006ADF09006AC7401F0C2028046
:102EA00053900BEAE030E24AA3E0FFF46040EFB455
:102EB000382CC202120934EFC0E07F0112094CCD58
:102EC000EFCDD0E0FF1209409006ADEFF09009B5CC
:102ED000E0C39403501E9006AC7401F08016900B72
:102EE000EBE09006ADF09006AC7401F08006C201F4
:102EF0008002C2019006ACE0B4010BA3E0FF12090E
:102F0000529009B5EFF0C208120958E4FF12095EA9
:102F1000E4900554F0120964A20192039006ADE01A
:102F2000F52C12096A120970900BEAE054FBF022AA
:102F3000CBEFCBCAEECA9006E77406F0E4900B3AEA
:102F4000F0C3EA648094805015EBF4FFEAF4FEEFDE
:102F500024019006E9F0E43E9006E8F0800890062F
:102F6000E8EAF0A3EBF09006E8E07002A3E070144A
:102F70009006E7E014F02434F582E4340BF5837412
:102F800030F080459006E8E0FEA3E0FFD39400EE29
:102F9000940040357C007D0A121BFDED2430FF902B
:102FA00006E7E014F02434F582E4340BF583EFF007
:102FB0009006E8E0FEA3E0FF7C007D0A121BFD9076
:102FC00006E8EEF0A3EFF080BBC3EA648094805083
:102FD000129006E7E014F02434F582E4340BF58314
:102FE000742DF09006E7E02434F9E4340BFA7B0109
:102FF00022900A99E0FF788EF6FF900A98E008F692
:10300000EF14603D1460571460631460782404600A
:1030100003023095900A95E5DAF0E024EF600A1497
:10302000600D14601024037012788E760180687829
:103030008E76028062788E760E805C788E760F8037
:1030400056900A95E024EF600904700A788E7604A1
:103050008004788E7605900A97E5DAF08039788ECC
:10306000760308A6DAE6F571757200802A788E7606
:103070000608A6DAE62572F572E43571F571E4907A
:103080000A96F08012788FA6DA900A97E0FFE6FDA4
:10309000123EAE8002C2DA788EE6900A99F008E617
:1030A000900A98F022900552E07003023144E4F057
:1030B0007B787D087F7D12508BEF600302313D905D
:1030C00006ADF0A3F09006ACF09006ACE0FFC39420
:1030D00008501574782FF8E6FFA3E48FF0121C5205
:1030E0009006ACE004F080E19006AEE070499006F6
:1030F000ACF09006ACE0FF2478F8E6FE90062BE0FA
:1031000075F007A424E5F582E43405F583E5822F04
:10311000F582E43583F583EEF09006ACE004F0E050
:10312000B407CF90062DE0FF125A6290062BE00400
:1031300075F00A84E5F0F0E4900556F0229005560B
:10314000E004F02290062CE0FF90062BE06F600870
:1031500090062DE0FF125A622278787C007D007B79
:10316000FF7A63799F7E007F05121B07787D7C00C4
:103170007D007BFF7A6379A47E007F05121B07D256
:103180003AD23978A57602D29F126490BF010678B0
:10319000A5E6B401F4BF0107900CC9E04440F01269
:1031A0006299E4F52C7B787D057FB01245928F2CD7
:1031B000900CE5E07003E52CF07B7D7D057FB0127F
:1031C00045928F2C900CE5E07003E52CF0787AE6C0
:1031D00054FBF67B787D057FB01245928F2C900CC6
:1031E000E5E07003E52CF07F6412602C1263A9EF18
:1031F0007007900CC9E04480F012628E7F01126269
:1032000083E4FF12628378A5762122D22F900BCF20
:103210007410F0A3E4F0A3F0A3F07B97753660750B
:10322000372F7D037FB0124B427897E6543FF64428
:1032300080F67B97754D60754E2F7D037FB0124AE7
:10324000FF7B97900BCFE0F536A3E0F5377D027F4B
:10325000B0124B42900BD3EFF0900BD2E025E0FF81
:10326000900BD1E033FE74292FF582745B3EF58319
:10327000E4937897667016742A2FF582745B3EF596
:1032800083E49308667006900BD3E06002C22F902F
:103290000BCFE475F001121C52900BD1E475F001D4
:1032A000121C52D3900BD0E0940B900BCFE09410F3
:1032B0005003202F8CA22F22EF121F2032F68032D3
:1032C000FC903302983308A0330EB03314B5331A90
:1032D000CC3320D33326D4332CD53332D63338DC19
:1032E000333EDD3344DE334ADF3350E43356E833D4
:1032F0005CFB00003361E580121BB722E590121BD6
:10330000B722E598121BB722E5A0121BB722E5B041
:10331000121BB722E5B5121BB722E5CC121BB72250
:10332000E5D3121BB722E5D4121BB722E5D5121B39
:10333000B722E5D6121BB722E5DC121BB722E5DD6A
:10334000121BB722E5DE121BB722E5DF121BB722E4
:10335000E5E4121BB722E5E8121BB722E5FB121BBE
:10336000B722E4F558F5597F03EF60391FA2AE92FA
:1033700015301502C2AED2DDE4900CA8F0C234D2F2
:1033800032301502D2AE7E647DB6EE600E30320B66
:10339000ED60031D80F41E7DB680EF2032CB900CD3
:1033A000A8E070C522EF7062A2AE9215301502C27D
:1033B000AE900CA7E0900CA8F0C235D2DFD2DEC2EE
:1033C000DDD2DCC2DBD2DA301502D2AEE4FB7D0600
:1033D0007F0112003EE4FB7D077F0112003E209733
:1033E00027C2DE209719E558C394085012C2967F71
:1033F00001124BBCD2967F01124BBC055880E4C22F
:10340000977F01124BBCD297D2DE227F0112525E0F
:10341000E49006ACF09006ACE0FFC394045011EFCA
:10342000906B3893FF1253809006ACE004F080E577
:103430007B027D017F0112003E7B02E4FD7F0312CF
:10344000003E7B027D027F0112003E7B037D04E48F
:10345000FF12003E7B027D057F0112003E7B02E4ED
:10346000FDFF12003E7B037D01E4FF12003E7B0363
:103470007D03E4FF12003E302E09D280D281D28338
:1034800075F6B47B037D047F0212003E202E037587
:10349000F634D2A5D2927B03E4FD7F0212003E7B7C
:1034A00003E4FDFF12003E7B037D047F0112003E1A
:1034B000D2A222ED605790062CE0FD90062BE06D25
:1034C000604B9005E4E0600414F080069005E4741D
:1034D00013F0E49006F0F09006F0E0FD2FF582E4A2
:1034E0003EF583E0FC9005E4E075F007A42457F571
:1034F00082E43405F583E5822DF582E43583F58396
:10350000ECF09006F0E004F0E0B407CB22E4900683
:10351000F0F09006F0E0FD2FF582E43EF583E0FC4C
:103520009005E3E075F007A42457F582E43405F52F
:1035300083E5822DF582E43583F583ECF09006F087
:10354000E004F0E0B407CB9005E3E00475F01484E8
:10355000E5F0F022E49006ACF0900BEAE04408F0CD
:1035600075FE557F01124A79E4FF1254FCA22150E6
:10357000028001C340091242289005547401F09062
:1035800006AC7401F0FF1265E31253201208B6E492
:10359000900AF6F0900AF7F0900AF6F0900AFEF022
:1035A0001208BC1208C21208C81208CE1208D4129F
:1035B00008DA1208E0900C83E04401F01208E612E9
:1035C00008EC1208F21208F81208FE120904120997
:1035D0000A12091012091612091C120922120928CE
:1035E000E49009E7F012092E900BEAE054F7F0544A
:1035F000FEF02220910302368B9005E4E0FF900557
:10360000E3E06F7003023691E49006ADF09006ACF3
:10361000F09006ACE0FF9005E4E075F007A42457B5
:10362000F582E43405F583E5822FF582E43583F5F0
:1036300083E0FE74782FF8EEF674782FF8E6FF90AA
:1036400006ADE02FF09006ACE004F0E0B407C290C5
:1036500006ADE0F404787FF67B787D087F7C124528
:1036600092EF70209005E4E00475F01484AFF0EF61
:10367000F09005E3E06F7006A3F09005E3F0E490AE
:103680000556F022900556E004F022900556E0041D
:10369000F02278FFE4F6D8FD9000007F007E10E471
:1036A000F0A3DFFCDEFA7581AE121A000236EA02E0
:1036B0003DD1E493A3F8E493A34003F68001F2081C
:1036C000DFF48029E493A3F85407240CC8C333C45F
:1036D000540F4420C8834004F456800146F6DFE4CA
:1036E000800B0102040810204080901F79E47E01C5
:1036F0009360BCA3FF543F30E509541FFEE493A33D
:1037000060010ECF54C025E060A840B8E493A3FA4E
:10371000E493A3F8E493A3C8C582C8CAC583CAF0DA
:10372000A3C8C582C8CAC583CADFE9DEE780BEA2D6
:10373000AF9202C2AFEF25E024FEFEF8E2FD30E7D3
:10374000030237C44480F2E51A700BE804F8E4F28F
:103750008F1A8F1B806EC8EEC8E2547FFDE51A25D4
:10376000E024FEF8E2547FFCEDD39C400AEE04F81E
:10377000E51AF28F1A804DE51B25E024FEF8E2548D
:103780007FFCEDD39C5012EE04F8E4F2E51B25E03B
:1037900024FFF8EFF2F51B802B851A2C852C2DE5E4
:1037A0002C25E024FFF8E2F52C25E024FEF8E25475
:1037B0007FC39D50E7EE04F8E52CF2E52D25E024CB
:1037C000FFF8EFF2A20292AF22A2AF922CC2AFEFAB
:1037D00025E024FEFEF8E2FD30E70302385E448077
:1037E000F2E51A700BE804F8E4F28F1A8F1B806E72
:1037F000C8EEC8E2547FFDE51A25E024FEF8E25445
:103800007FFCEDD39C400AEE04F8E51AF28F1A8093
:103810004DE51B25E024FEF8E2547FFCEDD39C50DF
:1038200012EE04F8E4F2E51B25E024FFF8EFF2F5D0
:103830001B802B851A6F856F70E56F25E024FFF8DC
:10384000E2F56F25E024FEF8E2547FC39D50E7EED9
:1038500004F8E56FF2E57025E024FFF8EFF2A22C02
:1038600092AF228F38E49006C0F0743CC231E4FB82
:103870007D067F0112003EE4FB7D077F0112003EC2
:1038800020972DC2DE20971F9006C0E0C3940850F9
:1038900016C2967F01124BBCD2967F01124BBC9090
:1038A00006C0E004F080DEC2977F01124BBCD297C5
:1038B000E5387004F5DB80038538DBD2AED2DFD289
:1038C000DEC2DDC2DCC2DBD2DAE4F5DEE5DF548045
:1038D000440FF5DF53DF7F43B502E4FB7D017F0238
:1038E00012003EE4FB7D027F0212003ED2A1D2A272
:1038F000E4900CA8F0228F2C900B02E0652C700352
:10390000023986E52C24FF92137D137FAE7E0012D0
:103910000898E52C64017029900B0004F090055381
:10392000F0900B01E0FF7D647C001256E0900B01EB
:10393000E0FF7D04120016900B01E0FF12587E801C
:103940003FE52C703B900B007407F07F0112095E7D
:103950007F607E01125162120AF65384EFE4900BED
:1039600003F0900B01E0FF7DC87C001256E0900B45
:1039700001E0FF7D05120016900B01E0FF12587E5A
:10398000900B02E52CF0221265489006ACEFF06433
:1039900001600FE0FF64036009EF64056004EFB4A9
:1039A0000704D2468002C246900D41E06401705A7D
:1039B000FB7A00792C1219AE900C87E0FF04FEE52B
:1039C0002CD39E5037EF14FFE52CC39F402EA3E06D
:1039D000FF04FEE52DD39E5023EF14FFE52DC39F7A
:1039E000401AA3E0FF04FEE52ED39E500FEF14FF14
:1039F000E52EC39F4006900D417402F0900C87E5C0
:103A00002CF0A3E52DF0A3E52EF074702290062C87
:103A1000E0FD90062BE06D6073E49006ACF090063C
:103A2000ACE0FD90062CE0F975F007A424E5F582E2
:103A3000E43405F583E5822DF582E43583F583E0F2
:103A4000FCEF2DF582E43EF583ECF0E975F007A478
:103A500024E5F582E43405F583E5822DF582E4352D
:103A600083F583E4F09006ACE004F0E0B407AF9097
:103A7000062CE00475F00A84AFF0EFF090062BE01E
:103A80006F7006A3F090062BF07F01227F0022FDCD
:103A900060FD6EFD7CFD8AFD97FDA5FDB3FDC0FDBB
:103AA000CEFDDCFDE9FDF7FE05FE13FE20FE2EFE39
:103AB0003CFE49FE57FE65FE72FE80FE8EFE9CFEB9
:103AC000A9FEB7FEC5FED2FEE0FEEEFEFBFF09FF3B
:103AD00017FF25FF32FF40FF4EFF5BFF69FF77FFB7
:103AE00084FF92FFA0FFAEFFBBFFC9FFD7FFE4FF3B
:103AF000F20000000D001B002900370044005200B6
:103B000060006D007B0089009600A400B200C090A8
:103B10000BE9E0FF64046004EFB40505E4FF12095B
:103B2000B8E4900A7EF01209BE1209C4D226900BA6
:103B3000D57401F01209CA1209707F021209D0125D
:103B400009D61209DC12093A9009B2E06F600790B9
:103B50000C83E04401F01209E24017900C83E0303E
:103B6000E0031209E81209EE900C83E030E0031242
:103B700009F4900C83E054FEF0E4900919F0120966
:103B8000FA120A00E4900AF7F0900AF6F022A2AFC7
:103B90009201C2AFAB1EE4F51EA20192AFEB6063CF
:103BA000E51D543FD39400405A7A01E51D543FFF70
:103BB000EAD39F504BEA25E025E0242CFE2403F8AD
:103BC000E2F930E638EE04F8E2FF1FEFD39400404C
:103BD00004EFF28028E930E70CC8EEC8E2FFE80401
:103BE000F8EFF2800DEE2403F8E954BFF2EE04F88A
:103BF000E4F2EE2402F8E2FF600312372F0A80ABF2
:103C00001B809A229006AC7408F09006ACE0FFD3BB
:103C10009400405CEF90578393FDE4FF122CB54075
:103C200047900BEEE0FEA3E0FF64014E700A9006A1
:103C3000ACE0900BEDF0801CD3EF9401EE940040CB
:103C40000E9006ACE0FD900BEDE06D60078021E486
:103C5000900BEDF0C3EF94FFEE94FF501C900BEE31
:103C6000E475F001121C52229006ACE014F0809A28
:103C7000E4900BEDF0A3F0A3F0229006AC7406F0F4
:103C80009006ACE0FFD39400405CEF90578C93FD1E
:103C9000E4FF122CB54047900BEEE0FEA3E0FF647A
:103CA000014E700A9006ACE0900BEDF0801CD3EF53
:103CB0009401EE9400400E9006ACE0FD900BEDE018
:103CC0006D60078021E4900BEDF0C3EF94FFEE945C
:103CD000FF501C900BEEE475F001121C522290066E
:103CE000ACE014F0809AE4900BEDF0A3F0A3F02286
:103CF0001209825033900BBBE07016900BB7E0FFB7
:103D00006009B4030C9008B4E07006900BB874FF1F
:103D1000F0900BBBE0B40110900BB8E0B4DC097478
:103D20003FF0900BB7741FF0900BB7E0FF60086492
:103D3000036004EFB40A0AEFB4030A9008B4E06029
:103D400004120AD222126A9FEF60159008B5E03083
:103D5000E70E1209825009900BBCE06003120AD2F0
:103D6000227F01126606E4900BE9F0900BE8F090D8
:103D70000BEAE04401F0125BF212340B7F60123860
:103D800063125DB1126002126AB7120A1812097644
:103D90005006E4900B02F022120A1E12005E12532B
:103DA00020120A24120A2A120A30120A36120A3C77
:103DB000120A42120A48120A4E120A54120A5A7D74
:103DC0003A7FAE7E0012089E922E120A60120A6698
:103DD00022126B0AC2AF53D0E51227FF12646012A1
:103DE0006B28125D6DD2AF126B341247F21265C0B0
:103DF00085811853D0E5E51E6003123B8EE51A60FD
:103E0000F2A2AF9200C2AFF519E51925E024FFF840
:103E1000E2F51AA20092AFE51925E024FEF8E2547B
:103E20007FF275F004E519904FAA121EE2E493FEAA
:103E3000740193CAEECAF9121F73E4F51980B42213
:103E4000CDEFCDCCEECC9006B37403F09006B474F5
:103E500030F0D3ED9400EC94004026ED540FFFF0C9
:103E6000FBECC4F854F0C868FCEDC4540F48FDEBFB
:103E7000940A5006E02430F080079006B4E024371E
:103E8000F09006B4E0FF9006B3E0243BF582E43402
:103E90000BF583EFF09006B3E0FF14F0EFD394003E
:103EA00050AAE4900B3FF07B017A0B793B22EF1292
:103EB0001F203EE9803EEC903EEF983EF2A03EF59A
:103EC000B03EF8B53EFBD33EFED43F01D53F04D60D
:103ED0003F07DC3F0ADD3F0DDE3F10DF3F13E43FCD
:103EE00016E83F19FB00003F1B8D80228D90228D2C
:103EF00098228DA0228DB0228DB5228DD3228DD413
:103F0000228DD5228DD6228DDC228DDD228DDE22E2
:103F10008DDF228DE4228DE8228DFB22C0E0C0F0EF
:103F2000C083C082C0D075D008C28C858C2A858A97
:103F30002B7407252BF52B74F8352AF52A852A8C46
:103F4000852B8AD28C051EE51D30E60930E7065325
:103F50001DBF12522D789D0806E618700106FFCE8F
:103F6000E6CEBE0317BFE414789D7600087600E520
:103F70001D30E70512522D8003431D40D0D0D08262
:103F8000D083D0F0D0E032EFC4335460FFE5E85482
:103F90009F4FF5E853E8F05398F0C2ECD2EB126A69
:103FA000D5A2EF92EBD2EA126AD5A2EF92EAD2E959
:103FB000126AD5A2EF92E9D2E8126AD5A2EF92E88E
:103FC000D29B126AD5A2EF929BD29A126AD5A2EF27
:103FD000929AD299126AD5A2EF9299D298126AD582
:103FE000A2EF9298E5E8C454F0FFE598540F4FFF14
:103FF000227D627F04125A147D627F05125A147D5D
:1040000064E4FF1244F0900B01EFF012589C120987
:10401000765006E4FF1238F6227D347FAE7E001221
:10402000089E50107D137FAE7E0012089EE433FF81
:104030001238F6227D3B7FAE7E0012089EC0D07DF6
:10404000137FAE7E0012089ED0F072F7E433FF12A9
:1040500038F6228F4F8D508B51755503900CA8E583
:104060004FF0E555604D900CA8E06047E4F0155521
:10407000E55460EE125D8FAF4F1248005006900C71
:10408000A8E54FF0E552FF1248005006900CA8E555
:104090004FF0AF531248005006900CA8E54FF0AD1A
:1040A00051AF501258D85006900CA8E54FF012644A
:1040B0008080AF22C2021200069202200252900BB0
:1040C000E9E0121F2040EF0040E10140E80340F624
:1040D0000440F60540FD06410B0841041000004174
:1040E00010120A8A92028028120A909202802112EB
:1040F0000A969202801A120A9C92028013120AA255
:104100009202800C120AA892028005120AAE920254
:10411000A2022278A5E664017055303A1B900C8FFC
:10412000E0FF2409FD124396900C8FE0240AF0E092
:10413000D3944C40037403F0303930900C8DE0FE82
:10414000A3E0FF2409FDE43EFC122AE9900C8DE473
:1041500075F00A121C52D3900C8EE09433900C8DA3
:10416000E094004006E4F0A3740AF078A5762122DA
:10417000C201120A7E40549009E7E07003D3800127
:10418000C35048900BBCE06005E4900907F0900B29
:10419000E8E014601924FD600E14601924057021F4
:1041A0001240B49201801A1252F0920180131254FC
:1041B0005E9201800C900B9EE030E705124E8792D4
:1041C00001200107120A845002D22622900A98E0A8
:1041D000788EF6A3E024FA601D24F8603524097077
:1041E0003B900A97E0FF7B007A00798E1232B87814
:1041F0008EE6F5DA8026900A96E02572F582E4359F
:1042000071F583E493788EF6F5DA900A96E004F07F
:10421000800A900A94E0FF788EF6F5DAC2DAD2DAF4
:10422000788EE6900A98F022E49006B6F09006B6F2
:10423000E0FFC394135018EF75F007A42457F582DC
:10424000E43405F583E4F09006B6E004F080DEE4A3
:104250009005E3F0A3F09006B6F09006B6E0FFC339
:1042600094095018EF75F007A424E5F582E43405AD
:10427000F583E4F09006B6E004F080DEE490062BCF
:10428000F0A3F022AE03EE20E00AEF25E0FFEEC33C
:1042900013FE80F21D1D1D74892DF582E43407F58F
:1042A00083E0FEEBF4FCEE5CFEEF5B4EF0303A2F69
:1042B00074892DF582E43407F583E07878F67B780D
:1042C000ED2403F5507D017F8A1245439006EEEF01
:1042D000F0900CE5E070089006EEE0900CE5F0221E
:1042E0008F388D398B3A753E03900CA8E538F0E590
:1042F0003E6047900CA8E06041E4F0153EE53D606B
:10430000EE125D8FAF381248005006900CA8E538C9
:10431000F0E53BFF1248005006900CA8E538F0AFDE
:104320003C1248005006900CA8E538F0755F01ABD0
:104330003AAD39AF3812433B80B5228F5C8D5D8B2F
:104340005E756003900CA8E55CF0E5606047900C3A
:10435000A8E06041E4F01560E55F60EE125D8FE576
:104360005C4401FF1248005008900CA8E55CF08006
:104370001FE55D601B12554AA85EA607055EE55D58
:1043800064016005125CC98003125DA0155D80E1C7
:1043900012648080B5228D2DE49006ACF0EFC394BA
:1043A0000350027F03E52DD3944C4003752D4C8FB1
:1043B0002EE52ED3952D502A9006ACE070247486FD
:1043C000252EF582E43407F583E07882F67B82853A
:1043D0002E507D017F8A1245439006ACEFF0052EEA
:1043E00080CF900CE5E070089006ACE0900CE5F012
:1043F00022900CDFEFF0900C48121F0E900CDFE0C3
:10440000F582758300121B68FF3395E0FEEF248070
:10441000FFE43EFE900CE9E0FD3395E0FCEF2DFF5C
:10442000EE3CFED3EF9498EE6480948040067E00CC
:104430007F98800FC3EF942CEE6480948050047EAC
:10444000007F2C025FB8900CD7EFF0900C42121F47
:104450000E900CD7E0F582758300121B68FF339530
:10446000E0FEEF2480FFE43EFE900CE3E0FD339598
:10447000E0FCEF2DFFEE3CFED3EF9498EE648094C9
:104480008040067E007F98800FC3EF942CEE6480FE
:10449000948050047E007F2C025E94900CB4EFF068
:1044A000900C3C121F0E900CB4E0F5827583001244
:1044B0001B68FF3395E0FEEF2480FFE43EFE900C86
:1044C000C6E0FD3395E0FCEF2DFFEE3CFED3EF940C
:1044D00080EE6480948040067E007F80800FC3EF72
:1044E000942CEE6480948050047E007F2C025E84C5
:1044F000CEEFCEE51D543FFFC394085043EF045464
:104500003FFFE51D54C04FF51D543FFF25E025E05A
:10451000242CFCBE80092403F8E24480F28008ECDD
:104520002403F8E2547FF2EC2403F8E254BFF2ECE7
:104530002402F8E4F2C8ECC8EDF2E804F8E4F22250
:104540007F00228F4D8D4E8B4FE4900CA8F03030C1
:1045500034125BDE501B854F54E4F555F5568550FB
:1045600057755801755903FBAD4EAF4D1225CD80DF
:1045700014854F54E4F555855056755703FBAD4EE1
:10458000AF4D124F38900CA8E0FFD394004002D2F8
:1045900031228F378D388B39E4900CA8F0303032CF
:1045A000125BDE501A853954E4F555F556F557750A
:1045B0005801755902FBAD38AF371225CD801385F0
:1045C0003954E4F555F556755702FBAD38AF37123F
:1045D0004F38900CA8E0FFD394004002D23122E47F
:1045E00090071EF0C2DEFB7D067F0112003EE4FB59
:1045F0007D077F0112003E20971F90071EE0C394A5
:10460000085016C2967F01124BBCD2967F01124B06
:10461000BC90071EE004F080DED2DE900CA7E09094
:104620000CA8F0C2DDD2DCC232D2DB228F518D5217
:104630008B53755603900CA8E551F0E55660399000
:104640000CA8E06033E4F01556E55560EE125D8F7E
:10465000AF511248005006900CA8E551F0AF54122B
:1046600048005006900CA8E551F0755F01AB53ADC2
:1046700052AF5112433B80C32201000000000200F0
:10468000000000000000000000000000000000002A
:1046900002020202020303030304030600000202F3
:1046A00002050200000000000000000101010101FC
:1046B00001000702020202020000030304030600D5
:1046C000000000000000EFC39D4007EFD39B5002A5
:1046D0008001C3400D300C05CFEBCF8034CFEDCF40
:1046E000802F300C17EF6B7010300D05CEEDCE80A3
:1046F00003CEEBCECFEECF80180F8015EF6D70108C
:10470000300D05CEEBCE8003CEEDCECFEECF8001C7
:104710001F228F458D46E54504FD7B82E4F5507FE1
:104720008A124E0E9006EFEFF074822545F8E6559A
:10473000469006EEF0E54620E0109006EEE0FFC35E
:1047400013F0E546C313F54680EB900CE5E07008E6
:104750009006EFE0900CE5F09006EEE0FF22EB64AF
:10476000036005EB6401701EEF14600E14600F14FB
:10477000601024037031ED429622ED429E22ED42FC
:10478000A622ED42BE22EF14600F146011146013D4
:1047900024037013EDF4529622EDF4529E22EDF4B0
:1047A00052A622EDF452BE22EB64036005EB6402D4
:1047B000701EEF14600E14600F146010240370312B
:1047C000ED429722ED429F22ED42A722ED42BF2209
:1047D000EF14600F14601114601324037013EDF4D0
:1047E000529722EDF4529F22EDF452A722EDF4529B
:1047F000BF22438901758CF8E4F58AD2A9D28C22B4
:104800008F61756280C216201623E562601F5561B4
:1048100024FF9217125F4FE562C313F562900C9567
:10482000E07002D2162016DF12003680DA3016024F
:10483000D322D2A11260959215120036900C95E009
:104840007002D322A21522900CB1EFF0900C2A1224
:104850001F0E900CB1E0F582758300121B682410C6
:10486000FF900CD4E02FFF3395E0FED3EF941CEEC5
:104870006480948040067E007F1C800FC3EF940408
:10488000EE6480948050047E007F04025ED4900C1D
:10489000B0EFF0900C27121F0E900CB0E0F582756F
:1048A0008300121B682410FF900CD3E02FFF339578
:1048B000E0FED3EF941CEE6480948040067E007F7F
:1048C0001C800FC3EF9404EE6480948050047E003B
:1048D0007F04025FE5900CAFEFF0900C24121F0EE6
:1048E000900CAFE0F582758300121B682410FF90D6
:1048F0000CD1E02FFF3395E0FED3EF941CEE6480E3
:10490000948040067E007F1C800FC3EF9404EE6409
:1049100080948050047E007F04025EB4900CAEEF61
:10492000F0900C1E121F0E900CAEE0F58275830005
:10493000121B682410FF900CCDE02FFF3395E0FE92
:10494000D3EF941CEE6480948040067E007F1C8030
:104950000FC3EF9404EE6480948050047E007F04C3
:10496000025EC4900CADEFF0900C1B121F0E900C69
:10497000ADE0F582758300121B682410FF900CCB0C
:10498000E02FFF3395E0FED3EF941CEE648094801B
:1049900040067E007F1C800FC3EF9404EE64809479
:1049A0008050047E007F04025FD6900B00E0640616
:1049B000703D900AFFE064017035126490EF702F33
:1049C000126498EF7023900B07E014F0E0700F90E2
:1049D0000C60E04410F07F01120988126B8CE4FF38
:1049E0001265DC7F011265DC22900B077403F02254
:1049F0008F308B318A328933E4F535E535C3953410
:104A00005030AB31AA32A93375F002E535A4F582F6
:104A100085F083121B6865307014E53575F002A4CB
:104A200029F9EA35F0FA900001121B68FF220535DA
:104A300080C97FFF22E47893F608F608F608F67638
:104A4000FF900BEDF0900BECF0900BEEF0A3F078F4
:104A500092F6900BEDF0A3F0A3F07D7F7F01125A48
:104A60001412596E7890EFF67D207F801244F07812
:104A700091EFF67D01120016228F35900BE9E0FFD1
:104A80009006BFF0E535C394115030E5356F602BCB
:104A9000AF351209A68F35C208900BE9E0F53690C4
:104AA00006BFE0F5371209AC900BE9E535F0D20806
:104AB000F5369006BFE0F5371209AC22900BB8E04E
:104AC00024F6501024BA602914602624FC601B14BC
:104AD00060188024900BB7E064036007900BB974F2
:104AE00001F022900BB97404F022900BB97402F01B
:104AF00022900BB97403F022900BB97404F0228F4A
:104B00004A8D4B8B4CE4900CA8F0303028125BDEC1
:104B10005014854D52854E53755401AB4CAD4BAF7F
:104B20004A124053800F854D52854E53AB4CAD4BCE
:104B3000AF4A125486900CA8E0FFD394004002D2F2
:104B400031228F338D348B35E4900CA8F030372828
:104B5000125BDE501485363B85373C753D01AB3525
:104B6000AD34AF331242E0800F85363B85373CAB26
:104B700035AD34AF33125350900CA8E0FFD39400FE
:104B80004002D23122AFF02275F0FD743230A20320
:104B900020A2F2D5E0F7D5F0F280EA75F0FD74328C
:104BA00020A20330A2DFD5E0F7D5F0F280D7EF23C3
:104BB00075F0FD0000D5F0FBD5E0F522EF0075F0B3
:104BC00003D5F0FDD5E0F722900CE0EFF0900C4B10
:104BD000121F0E900CE0E0F582758300121B682412
:104BE00010FF900CEAE02FFF3395E0FED3EF941F07
:104BF000EE6480948040067E007F1F800BC3EE64CD
:104C00008094805003E4FEFF025FC7900CC2EFF077
:104C1000900C30121F0E900CC2E0F58275830012CA
:104C20001B682410FF900CD6E02FFF3395E0FED3D5
:104C3000EF941FEE6480948040067E007F1F800BFF
:104C4000C3EE648094805003E4FEFF025EA48E33C2
:104C50008F348B358A368937E49006BEF07835E498
:104C600075F001121EEE121B4FFF0534E534AC3314
:104C70007002053314F5828C83EFF060089006BE55
:104C8000E004F080D8853482853383E4F022ACAE32
:104C9000B0B2B4B6B8BABCBEC0C1C2C3C4C5C6C740
:104CA000C8C9CACBCCCDCECFD0D1D2D3D4D5D6D70C
:104CB000D8D9DADBDCDDDEDFE0E1E2E3E4E5E6E7FC
:104CC000E8E9EAECEEF0F2F4F6F8FAFCFE00ACB635
:104CD000BABEC1C3C5C8C9CBCDCFD0D2D3D4D6D725
:104CE000D8DADBDCDDDEDFE0E1E2E4E4E5E6E7E8BC
:104CF000E9EAEBECEDEEEEEFF0F1F2F2F3F4F5F6BB
:104D0000F6F7F8F9F9FAFBFBFCFDFDFEFF00F0F009
:104D1000F1F1F2F2F3F3F4F4F5F5F6F6F7F7F8F84B
:104D2000F9F9FAFAFBFBFCFCFDFDFEFEFFFF0000BB
:104D3000010102020303040405050606070708082B
:104D400009090A0A0B0A0C0C0D0D0E0E0F0FF4F4D4
:104D5000F4F4F5F5F5F6F6F6F7F7F7F8F8F8F9F9EB
:104D6000F9FAFAFBFBFCFCFDFDFEFEFFFF00000173
:104D700001020203030404050506060607070808E6
:104D8000080909090A0A0A0B0B0B0C0C0C0C001081
:104D9000161B2023272A2D30323537393B3D404121
:104DA000434547494B4C4E505153545657595A5B03
:104DB0005D5E60616263656667686A6B6C6D6E708C
:104DC0007172737475767778797A7B7C7D7FE4F580
:104DD0002CC29F7B037D037F0212003EC2A353EED1
:104DE000EF052C43EE10052C53EEEF43EE047F64E9
:104DF00012602C43EE027B037D047F0212003ED240
:104E0000A47F6412602C12528FD29F0262A48F4D35
:104E10008D4E8B4FE4900CA8F0303722125BDE50A1
:104E200011855054755501AB4FAD4EAF4D12462C08
:104E3000800C855054AB4FAD4EAF4D1255BE900C0B
:104E4000A8E0FFD394004002D231228B2C8A2D8916
:104E50002ECEEDCE1254D59006B1EFF09006B1E013
:104E6000FFD394004020EF7A0024FFF582EA34FF5C
:104E7000F583AB2CAA2DA92E121B686E6008900634
:104E8000B1E014F080D622C202900BB8E0FF64B506
:104E90006009EF64B66004EFB4B4069009E7741ECD
:104EA000F0900BE9E024F2600A04700E120ABA9244
:104EB00002800C120AC092028005120AC69202A257
:104EC0000222900C93E0601014F0900C92E0F8E64F
:104ED000F5DAE004F0D2DB22303407D2DCC232D281
:104EE000DB22D234900C92E576F0900CA5E0900C89
:104EF00093F0203603024EC2D2DDD2DB22C2AFC213
:104F00009F43FB80C2A4E4900CEBF07FFA12602C6C
:104F1000900CEBE004F0E0C3940840EFD2A3E490DF
:104F20000CEBF07FFA12602C900CEBE004F0E0C385
:104F3000942840EF53FB7F22855475900CAAEDF026
:104F4000855576900CA5EBF0900CA7EFF0900CA98E
:104F5000E556F0E55764016005E557B40204D23325
:104F60008002C233E557B40504D2368002C236024D
:104F700033621263808F2FE52F64096017E52F6479
:104F8000026011E52F6406600BE52F64076005E5FC
:104F90002FB408151265B8BF010F126256EF30E248
:104FA00005752F0A8003E4F52FAF2F2201FF018F33
:104FB00002FF045003FF009504FF05B005FF06DE65
:104FC00006FF013207FF047208FF04FE09FF052EE9
:104FD0000AFF05500BFF058D0CFF023A0DFF02B3CF
:104FE0000EFF08928E4B8F4C900CA4E0602C789FA3
:104FF000EDF6C282E54B25E024A0FF7B9F854C5057
:105000007D01124543D28212642A126262500990D5
:105010000C61E04401F0C322D322C322AB07AA06ED
:10502000A90574F62BFB74FF3AFA7C007D03AF03ED
:10503000FE121BEBAA06AB07E4FFEF2BFDE43AFCE4
:10504000742E2DF58274063CF583E0A801F6090F55
:10505000BF03E722CCEFCCC9EDC9CAEBCACDEACD7C
:10506000A208920CA209920DAB2F1246C6CCEFCC2F
:10507000300714EC697010A208920CA209920DABD3
:105080002F1246C6CCEFCCCFECCF228F2C8D2D8BA0
:105090002EE4900CA8F030371C125BDE500E755FCA
:1050A00001AB2EAD2DAF2C12433B8009AB2EAD2DA5
:1050B000AF2C1256BE900CA8E0FFD394004002D251
:1050C00031220506360E320601370EE00601380E93
:1050D000E60601390EEC06013A0EF206013B0EF827
:1050E0000603150EFE0100170F040300190F0A0630
:1050F00002160F101957504F1A0300290F9A030078
:105100002B0FA002082C0FA605092D0FAC090134A6
:105110000FB20800330FB2A597A6A7A8A9AAABACF7
:10512000ADAEAFB0BCBDB5BEBFC0C1C2C3C48E2D95
:105130008F2EA2399201E4252EF52E7402352DF51D
:105140002DC239FF7549157B037D327C0012280082
:10515000A2019239AF2E75490D7BFF7D327C000292
:1051600028008E358F36A2399208E42536F536743C
:10517000043535F535C239FF7549087B077D237C39
:1051800000122800A2089239AF36E4F5497BFF7D72
:1051900023FC0228008D327B858E368F377D037F7E
:1051A000B0124B429006B3EFF0900CE5E07008901F
:1051B00006B3E0900CE5F0E4FF74852FF8E6A83222
:1051C000F605320FBF03F2228F2D7D7E7F087E0011
:1051D0001251957B007A00797E753A027D16122471
:1051E00097787EE6543FF6A82DF6052D787FE6A841
:1051F0002DF6052D7880E6A82DF6227F007E04127C
:1052000060477F567E091260547F007E0412606101
:105210007F567E0912606EE4F569FF7F02786AE4CA
:10522000F608DFFC53EFBF53EFDFD22422900C02CD
:10523000E004F0E0C3943C4024900C01E004F0E46E
:10524000A3F0900C01E0943C4013900C00E004F0BB
:10525000E4A3F0900C00E094184002E4F0223093B4
:1052600003D38001C39203E478A4F678A3F6BF02C7
:10527000087608A203B3929322BF030A78A4763F6C
:10528000A203B3929322EF7003C29322D29322E43B
:10529000900CEBF0E5AE20E016900CEBE0C394C868
:1052A000500D7FFA12602C900CEBE004F080E512B8
:1052B0005E04400B1262A4125E044003124EFD22F3
:1052C0008B518A5289531254D5EF2553F553E43547
:1052D00052F5527854E475F001121EEE121B4FFF86
:1052E0007851E475F001121EEEEF121BB770E42244
:1052F000C202200228900BE9E0601624FD600B2416
:10530000027015120A8A92028013120A9092028089
:105310000C120A9692028005120A8A9202A20222B6
:10532000E49006ADF09006ADE0FFC394075020EF87
:105330002411FF7E001227D69006ADE0249BF58253
:10534000E4340BF583EFF09006ADE004F080D62254
:10535000AC07E53B900CA9F0900CA6E53CF0D235EB
:105360008B75900CAAEDF0900CA7ECF0C233D236FE
:10537000900CA5EDF0857576E4900CAAF0023362EE
:105380008F2CE49006ADF09006ADE0FFC39408507A
:105390001CE52C2FFE5430FFC4540FFFEE540FFDBC
:1053A000E4FB12003E9006ADE004F080DA228B3E72
:1053B0008A3F8940AF441544EFD39400401C783EA7
:1053C000E475F001121EEE121B4FFF7841E475F0F8
:1053D00001121EEEEF121BB780DA2201007416CC08
:1053E00001007616D201007716D806007816DE0680
:1053F000007916E406007A16EA01007B16F0010037
:105400007C16F601007D16FC8B468A4789481254AB
:10541000D5EF2548F548E43547F5477846E475F07B
:1054200001121EEEED121BB7AB46AA47A948E412C3
:105430001BB7228E2C8F2DA2399201C239E52CFF89
:1054400075490C7B017D327C00122800A201923943
:10545000AF2D7549047BFF7D327C00022800C2021B
:10546000900BE9E024FD600F24F36012240F701309
:10547000120AB49202800C120A9092028005120A5B
:10548000A89202A20222AC07E552900CA9F0900C5F
:10549000A6E553F0D2358B75900CAAEDF0900CA7D1
:1054A000ECF0C233C236E4900CA5F0023362A2AF36
:1054B000922DC2AF741F2FFFF8E2FE547F6010EEF2
:1054C0004480F2547FFF1237C9A22D92AFD322A29B
:1054D0002D92AFC3228B578A588959E49006FCF06D
:1054E0007857E475F001121EEE121B4F600890060B
:1054F000FCE004F080EA9006FCE0FF228F30E5300B
:10550000C39406501D900BE8E0FF65306014C2089C
:105510008F311209B2900BE8E530F0D208F5311264
:1055200009B2227D637F0C125A147D407F801244A1
:10553000F0900555EFF07D0C120016C2BAD28AD257
:10554000AA12596E90062DEFF022E4F56175628083
:10555000D2A1E56260181260955008E5622561F5F8
:10556000618000E562C313F56212003680E4AF612A
:10557000228F2C7F011265E3E52C75F008A4FFAEA5
:10558000F012512EE52C547FFFE5D454804FF5D412
:1055900043D480E4FF0265E3C0E0C083C082C0D092
:1055A000900B0CE004F0E0D394014009C29F900BF3
:1055B0000BE04401F0D0D0D082D083D0E032900C08
:1055C000A9E554F08B75900CAAEDF0900CA7EFF0C4
:1055D000C233D236900CA5EDF0857576E4900CAA16
:1055E000F00233620A150B14486B7B6C716D396ED7
:1055F00039B548B6549671B47BB77272737376F549
:1056000052D12CAB798058DD59578B4B8A4C894D40
:105610007554FF75556375568B1252C0854E54856F
:105620004F55855056AB4BAA4CA94D1252C0221271
:105630006488125763126488BFB007900C62E0441C
:1056400002F01264A0126488BF8A07900C62E044E2
:1056500004F022900B0BE030E01C900C60E0444022
:10566000F0120AD8E4900553F07F0112095E12028D
:105670003A7FE0126A9922309303D38001C39201EA
:1056800078A3E6B40107E4F6A201B3929378A4E606
:10569000B40107763FA201B3929322000044108424
:1056A0000000931084000093108400009310840085
:1056B00000931084000093108400009310848B7575
:1056C000900CAAEDF0EF4401900CA7F0D233D23643
:1056D000900CA5EDF0857576E4900CAAF00233628B
:1056E000ED4C601BEF25E025E0242CF8EDF2EF25D2
:1056F000E025E0242FF8E230E60312587ED322C3DF
:10570000220600090F7006000A0F7606000B0F7CB8
:1057100006000C0F8203000E0F8801000D0F8E0F84
:1057200011108F34A23A9209C23A126A84E534C346
:1057300013FF126A8BA209923AE5341313543FFF08
:10574000026A928B388A39893A126B30A83AAC399E
:10575000AD387B017A0C79007E007F03121B0712A3
:105760006B2C227D787F097E00126B787878E6B406
:10577000FF0E08E6B4FF0908E6B4FF047F018002CB
:105780007F0022FFA993796049352106FFAA7F5B3C
:105790003F290E000001040205030704030501066A
:1057A0000807090000000FF000F00F0F000F0FFFB7
:1057B00000FF0F0000000FF000F00F0F000F0FFFB1
:1057C00000FF0FAB07E4F5507D0C7F8A124E0E9060
:1057D00006ADEFF0900CE5E070089006ADE0900C9F
:1057E000E5F0228B338A348935CFEDCFCEECCE1263
:1057F0002F308B548A558956AB33AA34A9351252AF
:10580000C0228F367B007A0079361208A49006C039
:10581000EFF0600AE0FF1208AAEF2463F536AF3616
:1058200022E569D39401400FE56994075009E569C1
:1058300090607B93426B22E56990607B93426A2281
:105840008F2CA2399201C2397B207D45124284A25D
:10585000019239E52CC313FF7B807D4B0242848F7C
:105860002CA2399201C2397B207D42124284A201CE
:105870009239E52CC313FF7B087D46024284EF2555
:10588000E025E0242CFFF8E2FE6010E804F8EEF2D8
:10589000C8EFC8E82403F8E24440F222900AFF74FB
:1058A00001F0900B067403F0A3F0A37414F0A3743A
:1058B0001EF0A37427F0E4A3F022E4FB7D05FF12A1
:1058C000003ED2857F077E001264781251FBC2250C
:1058D000D201125F22D2A8228F5C8D5DC214E55CDA
:1058E0006011A85DE6FF1248005002D214055D1554
:1058F0005C80EBA214228D308B317D821251957B1E
:10590000007A00798285313A7D081224977884E6FE
:105910005530FF22010101010100010101010100D7
:105920000101010101000101010101000101010169
:10593000010005051B0E3201001C0F1C03003F0F68
:10594000220600930D8403007E0F2801004E0F2EC7
:105950008D348B357D7812501C7B007A00797885E8
:10596000353A7D08122497787AE65534FF22E51CF3
:10597000C394105012051C741F251CFFF8E2547FBD
:10598000F25480F2AF1C227F00228E2C8F2DCFED9F
:10599000CF1258029006AEEFF0FDA2059213AF2D84
:1059A000AE2C1208982274862FF582E43407F58312
:1059B000E05DFFED20E00AEFC313FFEDC313FD80B0
:1059C000F22220030DEFC3952D50030F800FAF2E51
:1059D000800BEFD3952E40031F8002AF2D22C0E035
:1059E000C0F0C083C082C0D075D010120ACCD0D015
:1059F000D082D083D0F0D0E032900A937401F0C20C
:105A000082C2091264217F6012386343B502D2DA80
:105A100075FE5522EF25E024FEFFF8E2547FF25494
:105A200080FEED547F4EF2E804F8E4F2D322126BCC
:105A30003078007C0C7D017B007A0079327E007F1B
:105A400003121B07126B2C22900C93E014F0900CA5
:105A500092E0F8A6DAE004F0A3E0B40102C2DAD2E0
:105A6000DB22741F2FFFF8E2FE547F600CEE4480AF
:105A7000F2547FFF12372FD322C322900B04EDF094
:105A8000A3EFF0900B00740CF0A3E0FF7D647C00AA
:105A90001256E022900CAAE0900C93F0900C92E544
:105AA00075F0C2DD900CA7E0F5DAD2DB22900CA7EE
:105AB000E0900CA8F0D2DFD2DED2DDC2DCC2DBD2B5
:105AC000DAC234D2DB22D234900C92E576F0900C1C
:105AD000A5E0FF900C93F0BF0102C2DAD2DB229066
:105AE0000C93E014F0900C92E0F8A6DAE004F0D207
:105AF000DAD2DCC232D2DB2204042001091B2020CE
:105B0000B0B009B11B20B020B000B11B20000102D1
:105B1000058E348F35CFEDCF1258029006BFEFF0CF
:105B2000FDAF35AE3412089E22011807C007FE00F3
:105B300000002F0D6B07CF07FF071007FF0A8A062B
:105B4000BBA597A6A7A8A9AAABACADAEAFB0BCBD8C
:105B5000B4B5BEBFC0C1C2C3C400C001C102C2034C
:105B6000C304C405C706C60BF407D208D309D40A78
:105B7000F1E4900A93F07F60123863C2DAD282D2E5
:105B80000912642175FE0A228F3A8D3B125EE49061
:105B900006BFEFF06401FFF0AB3BAD3A025F5E126F
:105BA000093ABF0E03D38001C34009120A06120A44
:105BB0000C120A12221260E2500A900CE1E0540327
:105BC000F5388003E4F538AF3822900555E0FF1230
:105BD000587E9005537401F0E4900556F022E4FEDF
:105BE000EE90647093FD6008B50702D3220E80F03A
:105BF000C3227440E4F5771258BA7B037D037F011A
:105C000012003EC2932203006B0DEA04004B0DF01C
:105C10000400750DF00300490DF60502010E320572
:105C200003020E320504030E320507040E32020091
:105C3000430FD60400440D840400450D84060493EC
:105C40000D8400BC00C200C800CE00B600E700E82A
:105C500000E900EA0000201309EFC39546500A0F3F
:105C60008007EFD3954740011F22741F2FFFF8E2F2
:105C70005480FEED547F4EF2547FF2D322741F2FD6
:105C8000FFF8E2FE30E705547FF2D322C322C3229D
:105C9000E5D9B46009E4900A99F0900A98F0C2DA64
:105CA000D2DA2230250CC2A8AE67AF68C225D2A8CE
:105CB0008003E4FEFF22C0E0C083C08290055274DE
:105CC00001F0D082D083D0E032C217125F4FC2A25F
:105CD000D2A1900C95E06003126433223002089048
:105CE0000CD0E04402F022900CD0E054FDF022E40D
:105CF0007878F67B787D017F6512508B7878E6FFA7
:105D00002230350B900CA6E0F5DAD2DBC235221238
:105D10004EC222900CA8E5DBF0C234D2DA125C90BD
:105D2000D2DDD2DB22900CA8E5DBF0900C92E0F8FB
:105D3000A6DAD2DAD2DB2204060B0D0A0509131308
:105D40001307080C0E0F10111200F80101010801D1
:105D50000F012D0134013B01420149030305CC46EB
:105D6000072C2C322F111B332E472C2C43C2A9C2D7
:105D70008CE4F51EF51D789DF608F6D2B922CDEF1C
:105D8000CD90062DE0FF125C6A90062DE0FF22D236
:105D900017125F4FC2A1900C95E0600312003622EB
:105DA000D217125F4FD2A1900C95E060031200361B
:105DB000227448D23A126299E4FF1265DCC23AC2F8
:105DC00039228E388F39AF038D497B01AD39AC381C
:105DD0000228001265808F34126588EF25E0253493
:105DE000F534FF22123D617D7E7F03125A147F033A
:105DF000125F0422900CA8E5DBF0D2DDD2DA12416A
:105E0000CCD2DB22D201E5A45470C394305002C23C
:105E100001A20122000403030303020201010101A4
:105E20000000000074102FFF7549127B1F7D107C4D
:105E30000002280074102FFF7549097B1F7D117C1B
:105E40000002280074102FFF7549097B1F7D127C0A
:105E50000002280074102FFF75490A7B1F7D167CF5
:105E60000002280074102FFF7549057B1F7D167CEA
:105E70000002280074802FFF7549087BFF7D287C75
:105E80000002280074802FFF75490B7BFF7D237C67
:105E90000002280074802FFF7549087BFF7D247C59
:105EA0000002280074102FFF7549057B1F7D297C97
:105EB0000002280074102FFF75490A7B1F7D2C7C7F
:105EC0000002280074102FFF7549057B1F7D2C7C74
:105ED0000002280074102FFF7549057B1F7D2D7C63
:105EE000000228007401A805088002C333D8FCFD15
:105EF0001259A6220008040C020A060E0109050D1B
:105F0000030B070FCDEFCD7890E6FF125C6A789017
:105F1000E6FF227892E6D3940440047F0180027F5A
:105F2000002230010643EF80D28822C28853EF7FDF
:105F300022303303024EC2900CA9E0F5DAD2DB2204
:105F4000900CA7E0900CA8F0D2DCC232D2DB22A2E7
:105F50001792A1D2A2124B88900C95EFF0227401F7
:105F6000A803088002C333D8FCFB02428401F03F3F
:105F70007F01F2000001F30000010204EF547FFFF3
:105F8000E5DF54804FF5DF53DF7F2274102FFFE4ED
:105F9000F5497B1F7D16FC02280074102FFFE4F5E5
:105FA000497B1F7D17FC02280074802FFFE4F54910
:105FB0007BFF7D28FC02280074802FFFE4F5497BDD
:105FC000FF7D24FC02280074102FFFE4F5497B1F9D
:105FD0007D29FC02280074102FFFE4F5497B1F7D0A
:105FE0002CFC02280074102FFFE4F5497B1F7D2D47
:105FF000FC022800EF25E025E0242FF8E254BFF250
:10600000D322E4FB7D02FF12003ED209126421225A
:10601000900556E0C394BC4003D38001C322000224
:1060200001030102030405060708090AEFD39400DF
:1060300040077E66DEFE1F80F3221264681208B0FD
:10604000123FF1125BCA22E5EF54F84401F5EF8FDD
:10605000868E9522E5EF54F84402F5EF8F868E95F3
:1060600022E5EF54F84403F5EF8F868E9522E5EF95
:1060700054F84404F5EF8F868E9522408010080472
:106080000201201008040201C2DD900CA7E04401C7
:10609000F5DAD2DB22D2A2124B88900C95EFF0A257
:1060A000A122D238123F87900CABEFF0C238220009
:1060B0000102030400010203040201005387EFE41C
:1060C000FF1265DC1260C980FEC2DFD2DEC2DDC213
:1060D000DCC2DBD2DA2230930830A4057F021252F0
:1060E0005E22900CD0E030E103D38001C322010096
:1060F00001000001000001000000000102991101EF
:106100000001029911013200A000A3000035A5434F
:106110000000000F1E2D3C5A78B4F00000007549B5
:106120000E7B0F7D117C0002280075490E7B0F7DD0
:10613000127C0002280075490D7BFF7D147C000253
:1061400028007549057BFF7D147C000228007549F5
:10615000027B1F7D157C0002280075490D7B1F7D89
:10616000187C000228007B057D077F187E001259ED
:1061700050227549057B077D187C0002280075496F
:10618000087B1F7D187C000228007B107D1F7F1973
:106190007E00125950227549107B1F7D197C000228
:1061A00028007549087B1F7D197C0002280075496D
:1061B000047B0F7D1A7C0002280075490C7B0F7D43
:1061C0001B7C000228007549107B0F7D1B7C0002A0
:1061D00028007549147B0F7D1B7C0002280075493F
:1061E000047B0F7D1B7C000228007549087B0F7D16
:1061F0001B7C000228007549017B1F7D1D7C00026D
:10620000280075490E7B077D1E7C00022800754919
:10621000027B077D1F7C000228007549057B077DF6
:106220001F7C000228007549097B0F7D1F7C00023E
:1062300028007549017B077D327C000228007549E2
:10624000157B077D197C000228007B0A7D0F7F02E9
:106250007E001258F6227B027D1F7F157E001259A8
:106260005022900CA8E06003D38001C32274441232
:106270003159126ADB025571E478A5F6C23AC23987
:10628000C29F22AB077D077F157E00025DC27D3372
:106290007C007F0A7E00022AE9303A077D4C7F03AA
:1062A0001243962243FB4053FBBF7F6402602C6D78
:1062B0001400003F0020000000200102040810200C
:1062C0004001FF3F7FC8EFC8E6D39401400116228A
:1062D000E4F5497B037D15FC022800AB077D087FB0
:1062E000157E00025DC2AB077D097F157E00025D51
:1062F000C2E4FB7D1F7F18FE12595022E4F5497B52
:106300001F7D18FC022800E4F5497B1F7D19FC0263
:106310002800E4F5497B0F7D1AFC022800E4F549CA
:106320007B0F7D1BFC022800AB077D017F1C7E00DC
:10633000025DC2AB077D027F1C7E00025DC2AB071F
:106340007D037F1C7E00025DC2AB077D047F1C7E47
:1063500000025DC2AB077D057F1C7E00025DC2AB03
:10636000077D087F1C7E00025DC2E4F5497B037D4A
:106370001FFC022800E4F5497B077D22FC0228006F
:10638000E4FB7D1F7F01FE1258F6222000B3B0B15E
:10639000B200010203120982B39201120A7822604C
:1063A0002F840000602DFFC0807D147F017E0012CD
:1063B00064A82204004A0FF406024C0FFA03003FBF
:1063C0000F2207003C12347FA41262C57FA3026231
:1063D000C5900CE1E054FCF04FF022AB07E4FD7FE8
:1063E0001DFE025DC2AB07E4FD7F32FE025DC27D91
:1063F000127F017E001264A8227D0C7F017E0012B4
:1064000064A8227D0F7F017E001264A8227D057F93
:10641000017E001264A8227D067F017E001264A81E
:1064200022A209E433900CA4F022791478F9D8FE62
:10643000D9FA22124B9B900C95EFF0220003010237
:106440000800030808C2087D037F33025B88C20688
:10645000E4FD7F34025B88C2067D047F34025B88E2
:10646000E4F519F51AF51B227891E6FF12587E2201
:106470008687C0D6D7E4E20053EFF88F868E952248
:10648000C217125F4FD2A122900CE5E0FFE4F02288
:106490007D80E4FF124712227D807F021247122284
:1064A0007D0E7F0312471222AB057D011258F622A2
:1064B00002020002030200010102040810204080D1
:1064C0007FAE1262C5026B1E7D3F7F051259A62268
:1064D0007D3F7F101259A6227D3F7F121259A622BE
:1064E0007D3F7F141259A6227D3F7F151259A622A7
:1064F0007D3F7F171259A6227D3F7F181259A62291
:106500007D0F7F261259A6227DF07F261259A622E2
:10651000E4FD7F34125EE4227D037F34125EE422C8
:106520007D047F34125EE4227D077F361259A62255
:106530007D077F371259A6227DF07F3B1259A62294
:10654000E4FD7F43125EE4227D0FE4FF1247122236
:106550007D10E4FF124712227D20E4FF1247122231
:106560007D107F01124712227D207F0112471222E7
:106570007D017F02124712227D027F021247122202
:106580007D107F02124712227D207F0212471222C5
:106590007D407F02124712227D017F0312471222A3
:1065A0007DFF7F04124712227DFF7F0B12471222CC
:1065B00002020002030201007D017F2F125EE4222D
:1065C000126B2C12603A227893E6543FFF227894A3
:1065D000E6547FFF227B3F7D100242847B027D3D9B
:1065E000025F5E7B067D3E025F5E7B027D41025F55
:1065F0005EE4FB7D44025F5E7B017D44025F5E7B67
:10660000077D49025F5E7B047D4A025F5E7B057DFC
:106610004A025F5E7B7F7D030242847B7F7D0402B2
:1066200042847B3F7D050242847B3F7D060242849B
:106630007B3F7D070242847B3F7D080242847B3F93
:106640007D090242847B3F7D0A0242847B3F7D0BB1
:106650000242847B3F7D0C0242847B3F7D0D0242DF
:10666000847B3F7D0E0242847B3F7D0F0242847B10
:106670003F7D110242847B3F7D120242847B3F7D3D
:10668000130242847B3F7D140242847B3F7D1502CE
:1066900042847B3F7D170242847B3F7D1802428407
:1066A0007B3F7D190242847BC07D190242847B0FAF
:1066B0007D1A0242847B307D1A0242847B3F7D1B1F
:1066C0000242847B3F7D1C0242847B3F7D1D02424F
:1066D000847B3F7D1E0242847B3F7D200242847B7F
:1066E0003F7D210242847B3F7D220242847B077DE5
:1066F00023025F5E7B7F7D230242847B7F7D2402B9
:1067000042847B7F7D250242847B0F7D260242846A
:106710007BF07D260242847B3F7D270242847B3FC3
:106720007D280242847B067D28025F5E7B3F7D29B7
:10673000024284E4FB7D2F025F5E7B017D2F025FBE
:106740005E7B027D2F025F5EE4FB7D30025F5E7B3D
:10675000067D300242847B037D30025F5E7B047DD8
:1067600030025F5E7B057D30025F5E7B067D30021E
:106770005F5E7B077D310242847B037D31025F5E79
:106780007B047D31025F5E7B607D310242847B074A
:106790007D31025F5E7B027D32025F5E7B037D3274
:1067A000025F5E7B047D32025F5E7B057D32025FAD
:1067B0005E7B067D32025F5E7B077D330242847B17
:1067C000037D33025F5E7B307D330242847B067D36
:1067D00033025F5E7B077D33025F5EE4FB7D340244
:1067E0005F5E7B017D34025F5E7B027D34025F5E13
:1067F0007B037D34025F5E7B047D34025F5ED322C7
:106800007B057D34025F5E7B077D360242847B061A
:106810007D36025F5E7B077D370242847B387D37A1
:106820000242847B0F7D380242847BF07D38024235
:1068300084E4FB7D39025F5E7B067D390242847B06
:10684000037D39025F5E7B0F7D3A0242847B047DCB
:106850003A025F5E7B057D3A025F5EE4FB7D3B02B0
:106860005F5E7B017D3B025F5E7B027D3B025F5E84
:106870007B037D3B025F5E7BF07D3B024284E4FB59
:106880007D3C025F5E7B017D3C025F5E7B027D3C66
:10689000025F5E7B037D3C025F5E7B307D3C02429B
:1068A000847BC07D3C024284E4FB7D3D025F5E7BD5
:1068B000017D3D025F5E7B037D3D025F5E7B307D3F
:1068C0003D0242847B067D3D025F5E7B077D3D028B
:1068D0005F5EE4FB7D3E025F5E7B017D3E025F5EAC
:1068E0007B0C7D3E0242847B047D3E025F5E7B0525
:1068F0007D3E025F5E7B077D3F0242847B037D3FDE
:10690000025F5E7B047D3F025F5E7B607D3F0242F3
:1069100084E4FB7D40025F5E7B017D40025F5E7B25
:10692000027D40025F5E7B037D40025F5E7B047DF3
:1069300040025F5E7B057D40025F5E7B067D40021C
:106940005F5E7B077D40025F5EE4FB7D41025F5E30
:106950007B017D41025F5E7B057D41025F5E7B06C0
:106960007D41025F5E7B0F7D420242847B047D425B
:10697000025F5E7B077D42025F5EE4FB7D43025F58
:106980005E7B0E7D430242847B047D43025F5E7B1F
:10699000057D43025F5E7B067D43025F5E7B077D74
:1069A00043025F5E7B027D44025F5E7B037D4402A7
:1069B0005F5E7B047D44025F5E7B057D44025F5E1B
:1069C0007B067D44025F5E7B077D44025F5EE4FBE5
:1069D0007D45025F5E7B017D45025F5E7B0C7D45F0
:1069E0000242847B047D45025F5E7B067D45025F3B
:1069F0005E7B077D45025F5EE4FB7D46025F5E7B5A
:106A0000017D46025F5E7B027D46025F5E7B047D08
:106A100046025F5E7B057D46025F5E7B067D460229
:106A20005F5E7B077D46025F5E7B037D470242849B
:106A30007B0C7D470242847B307D470242847B078A
:106A40007D480242847B387D480242847B067D4833
:106A5000025F5E7B037D490242847B0C7D490242DA
:106A6000847B077D4A0242847B037D4A025F5E7B12
:106A7000077D4A025F5E7B067D4B025F5E7B787D11
:106A80002F0242847B047D39025F5E7B057D3902E3
:106A90005F5E7B067D39025F5E120AFC80FE2290FB
:106AA0000BEDE0FF22900BECE0FF22900BEFE0FFFC
:106AB00022900A93E0FF22E4900A93F022E49005EA
:106AC00056F022125C90D2DB22122FF1D2DB22127E
:106AD00041CCD2DB22D2EC20ECFD22E5D4547FFF66
:106AE00022C0300C03F00F00010203040501020470
:106AF0000810200808080C20007DFF124712227D94
:106B0000FF1259A622A201923A22744C024DCE00E5
:106B10000602010301020810047BFF0242847FA5E4
:106B20000262C50141434920E4F51C22431D802235
:106B3000531D7F22125DE4228090A0B0D7A50937B3
:106B4000D7A50447D7A51627D7A50827D7A50D256C
:106B50008686868ED7A5134701000000D7A50E10A4
:106B600003020303D7A51B1201003F7FD7A50236FE
:106B7000D7A50A46D7A50106025195AFDF220266C6
:106B8000D10267170268F50241130810222222225F
:106B900032FFFFFFFFFFFFFFFFFFFFFFFFFFFFFFD2
:106BA000FFFFFFFFFFFFFFFFFFFFFFFFFFFFFFFFF5
:106BB000FFFFFFFFFFFFFFFFFFFFFFFFFFFFFFFFE5
:106BC000FFFFFFFFFFFFFFFFFFFFFFFFFFFFFFFFD5
:106BD000FFFFFFFFFFFFFFFFFFFFFFFFFFFFFFFFC5
:10800000C0018891B4780320200A09D82C4081103F
:10801000000810037033030010100432F01003192D
:1080200004FF01FF03090309100410041B120E10C2
:1080300011111212191112030307800000000650DB
:10804000074107B60000003C193248715A5F000032
:10805000004F3B088220384A00022019321E2A3085
:108060005537320E3030E443320E2A30553732065F
:10807000282D50A832003030E443320E2A305541CA
:10808000320E2A305541320E2A305541320E1F4BE6
:10809000412D55013300660766AAAA02AA031E32C3
:1080A000D33B325353000002001B2F323835453585
:1080B0002F3B4BD33B325353D33B325353D33B32FF
:1080C0005353D33B32535300003F38353F3BB53514
:1080D000323B3838353238383B383238353F38352E
:1080E0003F3B000028FF96FF45193038200820103C
:1080F0002A3415451830382008201F2A2F150F075D
:108100000A000000C0C00A0AC0C0141E80801428E3
:108110008080142840401E3240401E3200001E3233
:10812000000000000101000002020A0A0202000031
:10813000002707EC00F60C13058303F600DD081397
:10814000064603F600DD0C0C07F3000605B900BD7A
:1081500002DD380000CA0303090987078B98470826
:1081600000000011078000001E0B8007003805800A
:1081700012003E3B801700AE08805200B63F805E82
:1081800000F536809D012B2580C701500580E20750
:10819000B10380E601551980E80497218101001A96
:1081A00004805A04D308815A0079258131009E0445
:1081B000815607C00F812207D1000000000003E8AC
:1081C0000004DB00C72005A3020C2007D10000003B
:1081D00001BF0101C0010321000320000394FF033C
:1081E00095FF03850004CC2004CD2004D13204CEB9
:1081F0003204D202016E0100373207BD0000010BCC
:1082000007B31F07B42500021E0005340004200731
:10821000CF0107D10000EE0100EE0000EF0100F0F9
:108220000100F00000F10100F10000F20100F20095
:1082300000F30100F40100F40004D30104D30004AE
:10824000D40104D50104D50004D60104D60004D716
:108250000104D70004D80104D90104D900000101A8
:10826000020203030405050607070808090A0A0BAA
:108270000C0C0D0E0E0F0F101111121313141515F7
:108280001616171818191A1A1B1C1C1D1D1E1F1F45
:108290002021212223232424252626272828292A91
:1082A0002A2B2B2C2D2D2E2F2F30313132323334DF
:1082B0003435363637383839393A3B3B3C3D3D3E2C
:1082C0003E3F00000101010201030001010202031F
:1082D000030405050607070808090A0A0B0C0C0D1C
:1082E0000E0E0F0F10111112131314151516161769
:1082F0001818191A1A1B1C1C1D1D1E1F1F202121B6
:108300002223232424252626272828292A2A2B2B02
:108310002C2D2D2E2F2F303131323233343435364F
:108320003637383839393A3B3B3C3D3D3E3E3F01DC
:108330000202010C030B0400030A0E0E10000000E1
:10834000000E0011123457082B2D1E11121427088D
:108350001B1D1EE49006C3F012F29BEF24FE604347
:1083600014606514602B240360030283EC9009BE43
:10837000E020E103D38001C340047F0280027F013B
:108380009006C3EFF09006C27404F09006C1F0802E
:10839000649006C37402F09006C27404F09006C1A3
:1083A000F080529009BEE020E203D38001C3400474
:1083B0007F0480027F039006C3EFF0E49006C2F0D2
:1083C0009006C17402F0802D9009BEE020E303D333
:1083D0008001C340047F0680027F059006C3EFF052
:1083E0009006C27403F09006C1F08009E49006C2C2
:1083F000F09006C1F012F29BEF601624FB50028051
:108400001E7FD17E041227D6EF543FFF1266A08054
:108410000E7F1D7E001227D6EF543FFF1266A090FC
:108420000BE8E0FF64046009EFB4050A120BA450E6
:108430000512E6E4800A9006C1E0FFE4FD128E0A10
:108440009006C2E0FF7D01128E0A7D02E4FF128ECB
:108450000A900AE0E0600C900AEBE07006FF1267F9
:108460007280057F02126772E4FF1267419006C3B3
:10847000E025E024CAF582E43409F583E0FFC45422
:1084800001FF126A0D9006C3E025E024CAF582E4DC
:108490003409F583E0FEA3E07803CEC313CE13D8EE
:1084A000F95401FF126988900B9CE030E4047F01CD
:1084B00080159006C3E025E024CAF582E43409F56E
:1084C00083E0A3E05407FF126981900B9CE030E445
:1084D000047F0180027F001269739006C3E025E0EB
:1084E00024CAF582E43409F583E0FEA3E07805CEE2
:1084F000C313CE13D8F95401FF1268319006C3E0BC
:1085000025E024CAF582E43409F583E0C4F854F088
:10851000C868A3E0C4540F485401FF12699D900637
:10852000C3E025E024CAF582E43409F583E0FEA324
:10853000E07806CEC313CE13D8F9EE5401FF1269CA
:10854000969006C3E025E024CAF582E43409F58359
:10855000E0FF13135403FF1268389006C3E025E0D0
:1085600024CAF582E43409F583E0FEA3E07806CE60
:10857000C313CE13D8F9540FFF126823900AE0E01A
:10858000600C900AEBE07006FF12682A800C9006DF
:10859000C3E090832F93FF12682A900B9CE030E495
:1085A000057F011269962212F29B9006BCEFF01231
:1085B000F2A19006BDEFF09006BCE0B40E047F017E
:1085C00080027F009006BEEFF09009B0E0121F20FD
:1085D00085EF01861802862B0386AB0486C00587CB
:1085E0006D06870D07872A08874009000087CA9013
:1085F00008B3E04404F012EEC61265689009AAEFD1
:10860000F0A3740FF09009B77401F09009B004F072
:10861000900BBDE054BFF02212F16B9006BEE070EB
:108620000312D2629009B07403F022900BBDE054A3
:10863000F7F09006BEE0600A9006BDE0FF12EDA5DF
:10864000803212F31B12E57992081294AF9009C0A0
:108650007406F09006BCE0701B900BBDE0FFC413E5
:10866000540730E0079009C0E02404F09006BDE014
:10867000FF12E253128353123B0F9006BEE06007D5
:108680009009B07406F022900A7DE04401F0E49075
:1086900009C5F012D2629009B07404F012F0F4909F
:1086A00009AF74FFF0E49009B7F0229009C0E0141C
:1086B000F0D3940640030287CA9009B07405F022F3
:1086C0009009C0E014F0E060030287CA9006BCE0A5
:1086D000FF6009B401179009B4E06011E4FF12686B
:1086E000627F011268B69009B07407F0229006BC50
:1086F000E0FF64026004EFB4030C7F011268B690DF
:1087000009B07407F0229009B07409F0229009AC06
:108710007402F0E4FF1268B69006BCE070057F01B9
:108720001268629009B07408F0229009ACE014F06D
:10873000E060030287CA9009B07409F0128B282206
:10874000126550EF6020126568BF01077F01EFC01E
:10875000E080057F00EFC0E012B3EECBEFCBD0E0BE
:10876000FF7D01120B8C9009B07406F022125B9F02
:1087700012CA56900BE8E06007900BE9E0B40E08CF
:10878000E4FBFD7F02120B209006BCE0600F900618
:10879000BEE060047F0180027F0012DECD12F29BFA
:1087A000EFC39401400B12F29BEFD394035002806D
:1087B00001C3500A900BBDE04408F04440F0E4903F
:1087C00009B0F09008B3E054FBF02212F29B90063F
:1087D000AEEFF09006B07411F09009C4E0FF5403BE
:1087E0009006B1F0EF13135403A3F0E4FF12C36D2E
:1087F000E4339006B3F07F0112C36DE4339006B406
:10880000F0E49006B6F09006B3E0600A7F0112DB58
:10881000FF9006B1EFF09006B4E0600A7F0212DB31
:10882000FF9006B2EFF09009C4E0FF30E703028941
:108830000A30E50302890A5403FE9006B1E0F96E9E
:108840006011EE70079006B004F08007E9700490A4
:1088500006B0F0EF13135403FE9006B2E0FD6E6015
:10886000179006B0E06401600FEE70057402F080AE
:1088700007ED70049006B0F09006B0E0705CEF3049
:10888000E658E97031ED702E9006B5F07F0312CEF8
:10889000F4900001121B68FB9006B5E0FD7F051205
:1088A0000B209006B67401F0120BAAE4900AABF00C
:1088B000FF12ED5580249006B1E060047F01800234
:1088C0007F029006B0EFF012F29B9006B0E06F705E
:1088D000097411F09009B47401F09006B0E0FF64DF
:1088E000016004EFB402239006B5EFF0FDE4FB7FD6
:1088F00005120B209006B67401F0120BAAE4900A40
:10890000ABF09006B0E0FF12D1DC12F29B9006B003
:10891000EFF09006AF7403F0BF01169009C4E05465
:1089200003FF9006B1E0FE6F60079006AFEEF080A7
:108930001E9006B0E0B402179009C4E0FF13135470
:1089400003FF9006B2E0FE6F60059006AFEEF09078
:1089500009C4E054FCFF9006B1E04FFF9009C4F059
:108960009006B2E0FE25E025E0FEEF54F34E9009BC
:10897000C4F09006AFE06403600F9006AEE0FF9095
:1089800006B0E06F700312D8D99009C4E054DFF04C
:1089900022900B5BE0121F2089B10189D20289E28B
:1089A0000389F5048A05058A61068AED0800008BB3
:1089B00027900C98E0FFA3E0900B60CFF0A3EFF0BE
:1089C000900B5B7402F0201903028B27D21A7405F6
:1089D000F022A21A92017F0A12BC17900B5B74035B
:1089E000F02212EAC05007900B5B7402F022900B49
:1089F0005B7404F022A21A92017F0A12BC17900B3A
:108A00005B7405F02212EAC050507B787536007511
:108A100037067D037FB0124B427878E6FDFF900B5E
:108A200057E4F0A3EFF0E0FE08E67A002400F0EA55
:108A30003E900B57F0ED30E711E0FEA3E0FFC3746A
:108A4000FF9FF074FF9E900B57F0A21A92017F0ACD
:108A500012BC17900B5B7406F022900B5B7404F051
:108A6000227B787536007537067D037FB0124B4246
:108A70007878E6FDFF900B59E4F0A3EFF0E0FE08F4
:108A8000E67A002400F0EA3E900B59F0ED30E71250
:108A9000E0FEA3E0FFC3E49FFFE49E900B59F0A328
:108AA000EFF0900B57E0FEA3E0FFD3900B5AE09F4E
:108AB000900B59E09E4017A21AB392017F0A12BC94
:108AC00017201903D21822900B5B7408F022900B28
:108AD00059E0FFA3E0900B57CFF0A3EFF0A21A925A
:108AE000017F0A12BC17900B5B7406F022900B8773
:108AF000E0FF12DA45900B87E004F0900B60E0FC99
:108B0000A3E0FDECC313FEED1325E0FFEE33FEED15
:108B10006F7002EC6E600AA21AB392017F0512BC5C
:108B200017900B5B7402F022E49006BFF012F29BE8
:108B30009006C0EFF09009B0E0FF64017003028C72
:108B40007BEF64037003028C7BEF64057003028C7F
:108B50007BEF64077003028C7BEF64087003028C68
:108B60007B9006C0E024FE6045147003028BEC2469
:108B7000026003028C287F0212C36D4003028C281E
:108B8000125DD3BF02047F0180027F009009BEE026
:108B900020E103D38001C340047E0180027E00EF08
:108BA0006E7003028C289006BF7401F0807A7F03F8
:108BB00012C36D5073126598BF010B12E2C35006C9
:108BC0007E007F0180047E007F009009BEE020E2ED
:108BD00003D38001C340047D0180027D00EF6D70EE
:108BE00001EE60449006BF7401F0803C7F0412C324
:108BF0006D5035126598BF010B12E2C350067E001E
:108C00007F0180047E007F009009BEE020E303D353
:108C10008001C340047D0180027D00EF6D7001EE94
:108C200060069006BF7401F09006BFE0604D9009A9
:108C3000BEE0FF9006C0E0FE7401C8EEC8088002E6
:108C4000C333D8FC6F9009BEF012F29B12C91D50BD
:108C50000C126548EF70069009BF7404F09006C0CE
:108C6000E0B401119009BEE020E103D38001C3B359
:108C700092081294AF128353120B927B017A0979F6
:108C8000BF120B98501212F29B12C91D500A7F019D
:108C90001268B6E4FF1268B622C201852C2C852D1D
:108CA0002DA2019201900D19E0603B125BB5EF64BB
:108CB000016006125BB5EF602A78ACE6B4012712BA
:108CC000A6D28F2DE52D6408601CE4900D19F0905C
:108CD0000D01E52DF078AA760178A9760178AB76BA
:108CE00001800312D837900D19E06002C10612A06E
:108CF00000125BB5EF64016008125BB5EF7002A172
:108D0000E112F301BF0C1578ADE664016002C10603
:108D1000FD7F06129EBC78AD7608C106900D0EE070
:108D2000FF900D24E0FD12BB4A8F2CEF9046799303
:108D3000900CFDF0900D01E0B4040DE52C700920BD
:108D40003C02D201D23C8007303C02D201C23C300E
:108D5000012CE4FF12CBD2EF6006E4FDFF128E0A75
:108D60007F0112CBD2EF60077D01E4FF128E0A7FF4
:108D70000212CBD2EF60077D02E4FF128E0A900D43
:108D800045E0652C6053E4FF12CBD2EF6034203C09
:108D90000A900CFDE0FFE4FD12B6A6AF2C12DDF444
:108DA0007F0112CBD2EF70087F0212CBD2EF60129C
:108DB000203C0A900CFDE0FF7D0612B6A6AF2C12F7
:108DC000DE20900CF7E0B40210E52C70077F011252
:108DD000C31380057F0212C313900D45E52CF0806C
:108DE00025125BB5EF6401601D125BB5EF701712C1
:108DF000F301BF0C1178ADE6B4010BE4FD7F061260
:108E00009EBC78AD760812ECAE228F348D35E535F8
:108E10007008900D08E534F08018E535B40108902D
:108E20000D1AE534F0800BE535B40206900D1BE514
:108E300034F0125BB5EF6401602C125BB5EF702665
:108E4000E5349060AF939006C6F0E5359060B99335
:108E50009006C7F0E53570079006C504F0806DE414
:108E60009006C5F08066125BB5EF64016006125B88
:108E7000B5EF6058E5349060B4939006C6F0E535E0
:108E80009060B9939006C7F0E5357022E53470160E
:108E9000303C0B9006C6F09006C504F0802E90067C
:108EA000C57402F080269006C57401F0801EE5347A
:108EB0007015303C0A9006C6F09006C5F0800D9003
:108EC00006C57403F08005E49006C5F0E49006C47E
:108ED000F0A3E014601F1460431460602403600278
:108EE000E1709006C6E0FFA3E0FD12CE1EE43390D1
:108EF00006C4F0807B9006C6E0FF7D0312CE1EE420
:108F0000339006C4F0E4FD7F0312B6A67D02E4FFB1
:108F100012B1087D037F0112B1088054900CFDE06E
:108F2000FFE4FD12B6A6E4339006C4F07D02E4FF30
:108F300012B1087D037F0112B1088034900CFDE06E
:108F4000FF7D0612B6A6E4339006C4F0E4FD7F0967
:108F500012B1087D017F0A12B1089006C4E06010CA
:108F60009006C7E0FD7F0512CE1EE4339006C4F0E4
:108F70009006C4E0FF22E49006B6F09006B6E075D5
:108F8000F005A424BCF582E43481F583C374019315
:108F900094D1E4939407506EE49006B2F0A3F0905D
:108FA00006B6E0FD75F005A424BEF582E43481F533
:108FB00083E493FE740193FF9006B2E0FAA3E0FB12
:108FC000C39FEA9E5037ED75F005A424BCF582E4FA
:108FD0003481F5837401932BFFE4933AFEED75F031
:108FE00005A424C0F582E43481F583E493FD124F97
:108FF000E49006B2E475F001121C5280A29006B60D
:10900000E004F0028F7BE49006B6F09006B6E0FF35
:1090100075F005A42462F582E43481F583E493FCC1
:10902000740193FDC394D1EC940750729006B4EC94
:10903000F0A3EDF0EF75F005A42465F582E434812A
:10904000F583E493FE7401938E2CF52DE49006B124
:10905000F09006B6E075F005A42464F582E434814E
:10906000F583E493FF9006B1E0C39F5028E0FDFF35
:109070009006B5E02FFF9006B4E03400FEE52D2DFC
:10908000F582E4352CF583E493FD124FE49006B1AC
:10909000E004F080BC9006B6E004F002900BE4908F
:1090A00006B6F09006B6E0FD75F003A424D0F58274
:1090B000E43481F583E493FE740193FFC394D1EE0D
:1090C0009407501CED75F003A424D2F582E434819A
:1090D000F583E493FD124FE49006B6E004F080C3FC
:1090E00022900A6EE0700302923424FE603A1470FB
:1090F0000302917824026003029242900A6C744049
:10910000F0F5D4126538900A6BEFF07F02126877A1
:10911000E4900A6DF0900A6FF0900A6E7402F0E429
:10912000FB7D017FFF120B20900A6DE004F01265B9
:1091300048BF020BE4900A6DF0A37403F0801B900B
:109140000A6DE0D394144012E4F0900A6BE0FF1231
:10915000687743D480E4900A6EF0E4FB7D027FFFE1
:10916000120B20900A7FE0FF7D287C001256E090D1
:109170000A7FE0FF12587E22900A6DE004F012652B
:10918000A89006EDEFF0900A6DE0C394FA5071904C
:1091900006EDE0FF94804017900A6CE0947F500F3A
:1091A000E004F0547FFEE5D454804EF5D48061EFA6
:1091B000C3947E5017900A6CE09400400FE014F0C6
:1091C000547FFFE5D454804FF5D48044900A6CE07E
:1091D000FFD3947F503AEFC394004034900A6BE081
:1091E000FF12687743D480900A6CE0FD7F057E0013
:1091F000124FE4900A6F7401F0E4900A6EF0801050
:10920000900A6BE0FF12687743D480E4900A6EF016
:10921000900A6CE0FD9006EDE0FB7FFF120B2090C2
:109220000A7FE0FF7D147C001256E0900A7FE0FF89
:1092300012587E22900A6FE0FB7D047FFF120B2004
:10924000D226228F349006C4E534F0900A01F01241
:10925000F29BEF640E60371209E240329006C4E0E0
:10926000602C900A0FE0FF9006C4E02FF0E0FFC3EF
:10927000648094805004E4F0800ED3EF648094E422
:1092800040069006C47464F09006C4E0F534E534FA
:109290007003029359900A16E0FFE534C39F50070C
:1092A000E49006C3F0802C900A17E0FFE534C39FDA
:1092B00050089006C37401F08019900A18E0FFE589
:1092C00034C39F50089006C37402F080069006C312
:1092D0007403F09006C3E0F925E0241AF582E43423
:1092E0000AF583E0FAA3E0FBE925E0241CF582E41B
:1092F000340AF583E0FEA3E0C39BFFEE9AFE7415EB
:1093000029F582E4340AF583E0F9C3E53499FD7C5C
:1093100000121BEB9006C3E02416F582E4340AF534
:1093200083E0C399FD121BFDEB2FFFEA3EFE900682
:10933000C1F0A3EFF02400FFEE34FCFE1251629066
:109340000A0DE054EFF054EFF0900A0CE0FF20E13A
:109350001920E01612F1EC80117F607E011251623B
:1093600012EFFD900A0DE04410F01209E2400C905B
:109370000A01E0FD7FF67E00124FE422900BE8E048
:1093800064016007900BE9E0B40D24900A0AE0A3A1
:10939000F0900A0DE020E3030294AB900B8AE064A6
:1093A0000470030294AB1295D012BE680294AB9085
:1093B0000BE8E064057028120BA45023900A0DE01E
:1093C00020E3030294AB900A097402F012B63890BD
:1093D0000A0CE030E10312BE6812F1810294AB90F6
:1093E0000BE8E0B40423900A0DE020E3030294AB01
:1093F000900A097402F012B638900A0CE030E103CA
:1094000012BE6812F1810294AB12F29BEF7040120F
:10941000F287503012D511900A0BE0FF6408601FEC
:10942000EF6409601A12CB3C4015900A0DE030E35E
:109430007AA3E06411600312BE681295D0806C12AA
:10944000DFA3806712DFA3900A0B7408F0805C90A2
:109450000A0DE030E355900A0BE0B4080E900A0ABA
:10946000E0FF12C03E900A0B7409F0900A097402E2
:10947000F0900A0CE030E406900A097401F012B68C
:1094800038900A0CE030E10612BE6812F18112CB6E
:109490003C50089006AF7401F08005E49006AFF0F0
:1094A0009006AFE024FF920312EE0512C57F22E47E
:1094B0009006C1F0A3F0A304F0E4A3F0A3F07D03B1
:1094C0007FEDFE12D3A49006C6EFF07D017FED7E06
:1094D0000012D3A49006C7EFF0E4A3F0A3F0A374A6
:1094E0001EF0A3E4F0A3741FF012F29B9006CDEFE0
:1094F000F0605E9006C17401F07D027FED7E001287
:10950000D3A49006C6EFF0E4FD7FEDFE12D3A49045
:1095100006C7EFF03008309006CDE0B4011E90068B
:10952000C27401F07465448860129006C97404F036
:10953000A374CCF0A37404F0A374CDF074654488D4
:1095400070059006C404F0E49006C3F09006C504CC
:10955000F09006C9E0FEA3E0FF1227D6EF543FFFCC
:109560001266929006CBE0FEA3E0FF1227D6EF54DE
:109570003FFF1266999006C8E0FF1269AB9006C1E2
:10958000E0FF12675D9006C2E0FF1268709006C3AC
:10959000E0FF12685B7D2A7FAE7E0012D74EE43377
:1095A000FF1268699006C4E0FF1268AF9006C5E03C
:1095B000FF1269579006C6E0FF126A309006C7E0B6
:1095C000D394024002E4F09006C7E0FF126A37220B
:1095D00012F1C3400B900A0EE0641270030296DC95
:1095E000900A127403F012F2EF9006B0EFF030E739
:1095F00006900A127408F09006B0E0547024E060FF
:109600000C24E0700F900A12E004F08007900A1218
:10961000E02402F01263EFBF010D9006B0E030E7E6
:1096200006900A127403F0900A12E0FFB40A219027
:109630000A09740BF0900A0CE0FE30E407E4900A8B
:1096400009F0803BEE30E537900A09740CF0802F6A
:10965000EFB40515900A097406F0900A0CE030E5A5
:109660001E900A097407F08016900A09EFF0900A1C
:109670000CE030E40AEF64036005E4900A09F0901E
:109680000A0EE064117048900A14E004F0E0B4039C
:109690000B12CB3C400612BE6812F181900A14E016
:1096A000640670359006B0E0FF20E30F30E70CE46D
:1096B000900A09F0900A0CE04410F0120BE0D22658
:1096C0007F017E0A120BDA900A0E7412F0800A9063
:1096D0000BD6E030E003120BE012B6381296E0220F
:1096E000900A0BE024FE604014600B24FD602414FB
:1096F000604A240670589006B1E4F0A37459F090C3
:1097000006B5E4F0A37454F09006B3E4F0A37457E4
:10971000F0803B9006B3E4F0A37457F09006B17468
:1097200004F0A374CEF080269006B3E4F0A374583E
:10973000F09006B1E4F0A3745AF080129006B1E400
:10974000F0A37455F09006B5E4F0A37455F0900AB8
:1097500009E0FF64036003EF70129006B1E0FEA31E
:10976000E0FF1227D6EF24F0FF12CF81900A09E024
:10977000FF64096013EF6408600EEF640A6009EF8C
:10978000640B6004EFB40C209006B3E0FEA3E0FF8E
:109790001227D612EAD99006B3E0FEA3E0FF122703
:1097A000D6EF24F0FF12D000900A09E0FF640460B5
:1097B0000EEF64056009EF64066004EFB4071290D1
:1097C00006B5E0FEA3E0FF1227D6EF24F0FF12D08B
:1097D00000229009AEE014605514700302988124B1
:1097E0000260030298C1900B9BE030E60B12F29BE3
:1097F000EF640E70030298C19009B0E06003029814
:10980000C112098250081209E250030298C190095E
:10981000ADE004F0E0D394C850030298C1E490098D
:10982000B1F0120BD4E49009ADF0A304F022900B38
:109830009BE030E60C12F29BBF0E06E49009AEF0FE
:10984000229009ADE004F0E0D394C84004A3740270
:10985000F09009B1E0601A7FCF7E071227D6EF6043
:1098600009E4FD7FCF7E07124FE4E49009ADF0A339
:10987000F012098240051209E25046E49009AEF068
:1098800022900B9BE030E60D9009B5E0B40E06E4A3
:109890009009AEF0227FCF7E071227D6EF700A1212
:1098A000098240051209E25006E49009AEF0227DDB
:1098B000017FCF7E07124FE4C2A27FB012F1288051
:1098C000FE228E348F351227D69006C4EFF0E53590
:1098D0002401FFE43534FE1227D69006C5EFF0E5EB
:1098E000352402FFE43534FE1227D69006C6EFF089
:1098F000E5352403FFE43534FE1227D69006C7EF82
:10990000F0E5352404FFE43534FE1227D69006C86E
:10991000EFF0E5352405FFE43534FE1227D6900636
:10992000C3EFF0E5352406FFE43534FE1227D69068
:1099300006C2EFF09006C4E0547FFF12E9BE900625
:10994000C5E0547FFF12E9D89006C6E0547FFF12AD
:10995000E9F29006C7E0547FFF12EA0C9006C8E0D7
:10996000547FFF12EA269006C2E0547FFF12E9A45A
:109970009006C3E0547FFF12E77E900A0CE0547F0C
:10998000F054BFF0900A2474FFF09006C4E030E772
:1099900017900B9DE030E309900A0CE04440F08002
:1099A00007900A0CE04480F012A9CF228F36E4F52C
:1099B00037853636853737853636125BB5EF640125
:1099C00070024190125BB5EF60024190E536146081
:1099D000270460024190900CEF7401F0E4900CF6C3
:1099E000F0126518900C69EFF07F011267F0E490B7
:1099F0000C6BF0900C6AF022900CEFE024FE6053A8
:109A000004600241901265708F37E53730E0047FC3
:109A10000180027F00900C6AE02FF0A3E004F09038
:109A20000C6AE0C394014015900CEF7402F0E4FF5F
:109A30001267F0E4900C6BF0900C6AF022900C6BC3
:109A4000E06402704B900C69E0FF1267F0E4900C48
:109A5000EFF0221265788F37900C6AE004F0A3E0F3
:109A600004F0900C6AE0C394004012E4900CEFF014
:109A7000900CF604F0900C69E0FF0267F0900C6B1C
:109A8000E0700D900C69E0FF1267F0E4900CEFF0CD
:109A9000227F011267A3E4FD7FAEFE12D74EE433AE
:109AA000FF1267F77D017FAE7E0012D74EE433FFD1
:109AB0001267DBE4FF1262DB7F5F7E001227D612A3
:109AC000F2F57F607E001227D61262267F3F7E006D
:109AD0001227D6125E247F407E001227D6125E34F3
:109AE0007F417E001227D612611E7F427E00122720
:109AF000D61261427F437E001227D6126136E4FF00
:109B00001263E57F477E001227D61262327F487EBD
:109B1000001227D6EF75F002A4FFAEF01254337F87
:109B2000497E001227D6FFEF75F008A4FFAEF012B1
:109B3000512E7F057E001227D6EF547F9006ADF0A0
:109B4000E0FE547FFDE5D454804DF5D443D480EE3F
:109B500075F008A4FFAEF012512E7F011267AA7FA4
:109B6000447E001227D6125E447F457E001227D61F
:109B700012612A2212F29BEF600E12F29BEF640E2A
:109B8000600612EC82029C41900A097403F0900A6C
:109B900012E024FB602B24FD603E14605414606AC4
:109BA00024066003029C41900A0CE06410FFF090D0
:109BB0000A097404F0EF20E403029C41E4F0029CE3
:109BC00041900A0CE06420FFF0900A097406F0EF5F
:109BD00030E56E7407F08069900A0CE06410F05470
:109BE000DFFFF0900A097408F0EF30E454E4F080ED
:109BF00050900A0CE06410F054DFFFF0900A0974F2
:109C000009F0EF30E43BE4F08037900A0CE0FF30DD
:109C1000E40B54CFF0900A09740BF08024EF20E598
:109C20001154EF900A0CF04420F0900A09740CF0E3
:109C3000800FEF4410900A0CF054DFF0E4900A0912
:109C4000F012B638900BE8E06401600312B77F228F
:109C50009006B6E4F0A374F8F0900BE8E0B4010AC3
:109C60009006B67401F0A3742DF0900A02E09006FD
:109C7000B8F0900A03E09006B9F0900A04E090066C
:109C8000BAF0900A05E09006BBF0900A10E090064A
:109C9000BCF0900B9DE030E314900A0CE0FF20E64E
:109CA0000330E7179006B8E04480F0800E900A0C6D
:109CB000E030E7079006B8E04480F09006B6E0FE9A
:109CC000A3E0FFA3E0FD124FE49006B7E02401FFFC
:109CD0009006B6E03400FE9006B9E0FD124FE49025
:109CE00006B7E02402FF9006B6E03400FE9006BA04
:109CF000E0FD124FE49006B7E02403FF9006B6E0C3
:109D00003400FE9006BBE0FD124FE49006B7E0245D
:109D100004FF9006B6E03400FE9006BCE0FD124F52
:109D2000E422900AC5E09006AFF0900AC4E09006E5
:109D3000B0F0900AC3E09006B1F012E89C40030234
:109D40009DF112F29BEF7003029DF112DC8B900AE1
:109D500079E0FF900AC7E06F7003029DF1EFF09089
:109D60000B9DE030E203029DF11264D89006ACEF47
:109D7000F01264D09006ADEFF01264C89006AEEF1A
:109D8000F0900A79E070319006ACE0FF9006AFE009
:109D9000FEC3EF9E9006ACF0A3E0FF9006B1E0FE9C
:109DA000C3EF9E9006ADF0A3E0FF9006B0E0FEC3C7
:109DB000EF9E9006AEF080219006AFE0FF9006ACDB
:109DC000E02FF09006B1E0FF9006ADE02FF0900696
:109DD000B0E0FF9006AEE02FF09006ACE0FF126618
:109DE000769006ADE0FF1265D59006AEE0FF1266F4
:109DF0002222900A0DE054BFF0E49006EDF020130B
:109E000003029EB3900A0DE04440F09006ED740109
:109E1000F07F797E001227D69006EEEFF0A3747AD9
:109E2000F0E4A3F09006EFE0FF7E0012E16BEFC4D8
:109E3000F8540FC8689006F2F0EEC454F04890064B
:109E4000F1F0E07878F6A3E008F69006F0E0FF90F5
:109E500006EEE02F08F67B78754D00754E207D03E9
:109E60007FB0124AFF9006EFE02402F0A3E004F076
:109E7000E0C3941040AE7F9C7E0012E16BEFC4F80B
:109E8000540FC8689006F2F0EEC454F0489006F102
:109E9000F0E07878F6A3E008F67F9A7E001227D6E5
:109EA000787AEFF67B78754D00754E207D037FB094
:109EB000124AFF9006EDE0FF126202228D338533D5
:109EC00033BF0620900C66121F0E900C64E0F582E2
:109ED000758300121B68FE900D05E06E60047F051F
:109EE00080027F03EF121F209F01009F30019F38E7
:109EF000029F60039F78049F7D059F3D0700009FA0
:109F000080D20912F0001262F1900C63EFF012613E
:109F100066900C65EFF0E4FF12DDF47D027F051220
:109F2000B6A67D037F0512B6A6E4FD7F0502B6A6A0
:109F3000E4900C64F002ACAEE4FF02ACC1900C63A0
:109F4000E0FF1262FC900C65E0FF1261727D027FFF
:109F50000612B6A67D037F0612B6A6C20902F0005D
:109F6000900C64E004F0900D00E0FF900C64E0C3FE
:109F70009F4002E4F002ACAEAF3302ACC112ACAE13
:109F800022200B07900AC2E054BFF0300A4D200B8C
:109F900008900ACEE0900ABEF07F0312BA11900B2F
:109FA0009DE0FF30E10A900ACBE0900ABFF0800804
:109FB000900AC1E0900ABFF0E4900AC1F0EF30E2ED
:109FC000347406F0900BA1E030E608900AC17405E5
:109FD000F08022900AC17406F0801A200B0F900ABC
:109FE000C2E054F7F0900ABEE0FF12BA11900ABF27
:109FF000E0900AC1F0900AC1E0FF12C205222222BD
:10A000009006AC7410F0852E2E125BB5EF640160E3
:10A0100008125BB5EF700201A8126403BF010F784C
:10A02000A9E6B4010D9006ACE04480F0800478A964
:10A03000760112640DBF011278AAE6B401109006F1
:10A04000ACE04440F054EFF0800478AA760112644A
:10A0500017BF011A78ABE664016007900D24E0B4E5
:10A0600004109006ACE04420F054EFF0800478AB8C
:10A0700076011263F9BF01079006ACE04401F012CB
:10A08000624A8F2EE52E30E3079006ACE04408F0DC
:10A09000E52E30E2079006ACE04404F0E52E30E116
:10A0A000079006ACE04402F09006ACE0FF900D0E85
:10A0B000E06F6002D23F900D0EEFF022900BBFEEEA
:10A0C000F0A3EFF012E663CCEECCCDEFCD900BBF5A
:10A0D000E0FEA3E0FF2D7879F6EE3C18F6900BBE7B
:10A0E000E0906B5093787AF612D155787BEFF618A2
:10A0F000E654BFF6900BBDE0FF540175F040A42676
:10A10000F6A3E0FE60046402702B787AE6441879C6
:10A110007CF7787D7660EEB40212EFC4540F30E025
:10A12000047F1080027F08EF787B46F67D787F06FB
:10A1300012EBCB80327878E6FF08E6787CCFF60821
:10A14000EFF6900BC1E0FEA3E0FFD3900BC0E09FC1
:10A15000900BBFE09E40097D787F0412EBCB800717
:10A160007D7A7F0412EBCB900BBFE0FFA3E0A3CF7F
:10A17000F0A3EFF022900A157401F0900A197464AC
:10A18000F0E49006ADF09006ADE0FFC39405505C9E
:10A19000EF25E02465FF7E0012E16B9006ADE0FD47
:10A1A00025E0241AF582E4340AF583EEF0A3EFF0FB
:10A1B000ED25E0241AF582E4340AF583E0FEA3E0FD
:10A1C000FFC3EE9400401DD3EF94C0EE94005014F2
:10A1D000ED25E0241AF582E4340AF583740775F05E
:10A1E000FF121C529006ADE004F0809A9006AD7408
:10A1F00001F09006ADE0FFC394045020EF246EFF01
:10A200007E001227D69006ADE02415F582E4340ACC
:10A21000F583EFF09006ADE004F080D67F3F12EEBC
:10A220005F7D01E4FF12DF4E2212F19712EEC6C2EB
:10A2300019900BE8E0B4011FE4FF1254FC900A7A75
:10A240007403F0C208120BF2900B5FE09006B9F0B5
:10A25000E4FF1268B68030C20812D7BC900B5FEFE3
:10A26000F07F011254FCE4900A7AF0D208120BF24B
:10A270007F01124A79120BF8D20812D7BC9006B9A6
:10A28000EFF07F011268B6900BE8E0B40103D380D1
:10A2900001C3920812F055E490044FF012EDB9900A
:10A2A00006B9E0FF12E332900BE8E0702D9006B99A
:10A2B000E0FF12D089EF601F7FC07E011227D69089
:10A2C00006B8EFF0E075F002A424C1FFE5F0340118
:10A2D000FE12E16B12E8B7120BFE22C2069006AC2A
:10A2E0007403F0E4A3F0900B9DE030E2259006ACFF
:10A2F0007407F0E4A3F0900BE8E0B40415900BA110
:10A30000E030E6089006AD7405F080069006AD7466
:10A3100006F0E4FF12BA119006AE7402F0900BA1A1
:10A32000E030E608D2069006AE7406F0900AC1E06E
:10A33000FF9006AEE0FD9006ADE0FB9006ACE014A9
:10A34000F52FA2069207A2059208D20912505412C4
:10A35000C205900AC1E0FD900ACBF0900B9DE03061
:10A36000E203D38001C3400D900BE8E070077F85C6
:10A370007E03124FE4900B9DE030E20D900BE8E07D
:10A38000FF900AC1E0FD12E8492212B3EE9006C523
:10A39000EFF0A374FFF0900A78E09006C7F0900AFF
:10A3A0000BE09006C8F01265489006C9EFF09006E1
:10A3B000C7E0FF60049006C9F012F29BEF601EE454
:10A3C0009006C6F09006C5E024FE60090470639014
:10A3D00006C6E004F09006C6E004F080559006C57D
:10A3E000E024FD602B04704A9006C8E0FFB4010829
:10A3F0009006C67404F0803AEFB403089006C67461
:10A4000006F0802EEFB4022A9006C67403F0802274
:10A410009006C8E0FFB406069006C67407F0EFB4D5
:10A4200001069006C67408F0EFB403069006C674E1
:10A4300005F09006C6E0FF228C348D357B017A064C
:10A4400079C97D0612D90E9006C9E09006C3F09036
:10A4500006CAE09006C4F09006CBE09006C5F090E6
:10A4600006CCE09006C6F0E5354534600CAF35AE5D
:10A47000341227D69006C6EFF09006CEE09006C7BD
:10A48000F030E30512F07F800312F08C900B9CE01B
:10A4900030E4047F0180027F00EF6401703112D24A
:10A4A000A49006C7E030E1097D107F0212EE938090
:10A4B000077D107F0212EE299006C7E030E0097D8B
:10A4C000017F0312EE9380077D017F0312EE299036
:10A4D0000CA1E0700F9006C7E030E20512EBE380BC
:10A4E0000312E7BA228F2F9009B5E09006B6F090DC
:10A4F00009B5E52FF0121F20A52B00A52B01A52BD8
:10A5000002A52B03A52604A52605A52606A56E07EC
:10A51000A56E08A56E09A5260AA5610EA56E0FA554
:10A5200026100000A571120BBC8046120BC25041D0
:10A53000E52F6003B40E117F0312CEF490000112D8
:10A540001B68FF12E0C88005AF2F12ED559006B6CC
:10A55000E0FFD39403401AEF940E501512F24A8094
:10A5600010900BE8E064016008120BC88003120B26
:10A57000CEE52FC39404500AE4FD7FBD7E07124F41
:10A58000E422AD2F7FBD7E07124FE422E4900A7DC6
:10A59000F07F1EFE1227D6EF543FFF1266927F1FF8
:10A5A0007E001227D6EF543FFF12669912E811126F
:10A5B000EB6B12F155E4FF12672CE4FF12673312C4
:10A5C000E90812ECC47D297FAE7E0012D74EE43339
:10A5D000FF1267B112E2E812E92212DEA212EED6F1
:10A5E00012E93C12ECD912ECEE12CE6612CD8E12AC
:10A5F000E09F12F16012EEE612F33E12ADD012B9F6
:10A600003F12EDF3E4900A7BF0900A7A7403F09025
:10A610000BA0E030E3047F0180027F00BF01111234
:10A620000B0E7F977E041227D6EF5403FF120B14F4
:10A6300022E49006ACF09009B0E060047F01800253
:10A640007F00EF7031900BE8E0FF600B6403600760
:10A65000900BE9E0B40E1F1265509006AEEFF0903B
:10A6600009AFE06F60109006AEE0FD9009AFF0E436
:10A67000FB7F10120B201265609006ADEFF0900981
:10A68000B6E06F604C9006ADE0B40111126568BF92
:10A6900001047F0180027F009006ACEFF09009B7C3
:10A6A000E0702E900BE8E0FF600B64036007900BF6
:10A6B000E9E0B40E1C9006ADE09009B6F0B40111CB
:10A6C00012B3EECBEFCB9006ACE0FFA3E0FD120B94
:10A6D0008C22124F72EF24E16042241EB41200401B
:10A6E00002E16C90A6E925E073E112E10DE117E1CA
:10A6F00021E126E12BE130E135E13AE13FE144E1BE
:10A7000049E14EE153E158E15DE162E167752E01F7
:10A71000805DE4F52E8058752E038053752E0880D9
:10A720004EE4F52E8049752E058044752E01803F3C
:10A73000752E0A803A752E0B8035752E0680307581
:10A740002E04802B752E028026752E0C8021752EEE
:10A7500003801C752E0D8017752E0E8012752E0F1E
:10A76000800D752E108008752E118003752E07AF91
:10A770002E22900A7DE04401F0E4FF12DECD900A23
:10A780007A7403F0C22778A6E6FF125FF412F25A39
:10A7900012EF46E4900CECF012F241900B81EEF0D7
:10A7A000A3EFF0900A78E0B4011512F241D3EF94D0
:10A7B000E4EE94064010900BBDE054FDF08007C21B
:10A7C0001CE4FF12673AE4FF120B3212F0F47F022E
:10A7D00012BA11900AF77401F0E4900AF6F0900AA8
:10A7E000FE7404F0E4FF12692D78A6E6FF7DC87CB4
:10A7F000001256E078A6E6FF7D0212001678A6E663
:10A80000FF12587E900BBDE04408F022CBEFCBCA7C
:10A81000EECACEECCECFEDCF7C007D0A121BEB7CD6
:10A82000027D71121BFDCCEECCCDEFCDEBC4F85404
:10A830000FC868FFEAC454F048FEED2F9006AFF051
:10A84000EC3E9006AEF0900BE8E0B4010E7C007D8B
:10A850000ACFEBCFCEEACE121BEB22900A78E0B4FF
:10A860000138CEEACECFEBCFEA702FEF24C46014CC
:10A8700024FD601C240870229006AE7403F0A374BB
:10A880007CF080169006AE7403F0A374C8F0800AC2
:10A890009006AE7403F0A374FCF09006AEE0FEA345
:10A8A000E0FF22900CECE0B4050E120B56C20C7FB8
:10A8B000407E18120B5C8014201B0512F01D500303
:10A8C000120B62C20C7F407E18120B5C900A7DE076
:10A8D0004401F0E4FF12DECD900A7A7403F0120B0B
:10A8E0006878A6E6FF125FF412F25A12EF46E4907F
:10A8F0000CECF0C21CFF12673A201B0812F01D403E
:10A9000003303B11120B6E5005120B74801D7F013A
:10A9100012E0C88016900B87E014FF12E0C8900B7D
:10A9200087E014FBE4FD7F05120B20E4FF12692D84
:10A93000E4FBFD7F0E120B202212DFA3C213129D37
:10A94000F212CAF0129A9112A175900A0F740AF0CD
:10A9500012DCE77FF77E001227D6900A08EFF0128C
:10A96000E98A7D397FAE7E0012D74E5005D2131290
:10A970009DF27F3D7E001227D6900A11EFF0E49001
:10A980000A0AF0FF12DECD900A097403F0900A1251
:10A99000F0900A0CE04401F0900A2474FFF07D105E
:10A9A0007FAE7E0012D74E4007900A0CE054FEF0B6
:10A9B0007FB17E0712E16B900A25EEF0A3EFF07FE6
:10A9C000527E0112E16B900A27EEF0A3EFF0229085
:10A9D00006C9E4F0A37472F0A3E4F0A3745CF0A3DE
:10A9E000E4F0A37461F012F29BEF600612F29BBFD9
:10A9F0000E0C120BA44007900BE8E0B4041F900665
:10AA0000C9E4F0A37474F0A3E4F0A3745DF012F24F
:10AA10009BBF02099006C9E4F0A37472F09006C9C6
:10AA2000E0FEA3E0FF1227D61266149006C9E0FEEE
:10AA3000A3E0FF1227D612661B9006CBE0FEA3E030
:10AA4000FF1227D6125F9A9006CDE0FEA3E0FF1218
:10AA500027D6125FA99006CDE0FEA3E0FF1227D60D
:10AA6000125E742212A38A9006C0EFF0F470030203
:10AA7000AAF6E0FF75F003A42417F582E43482F50A
:10AA800083E4939006C2F0EF75F003A42415F582D9
:10AA9000E43482F583E493FF7401939006C3CFF00E
:10AAA000A3EFF0900A7DE030E2349006C0E0FF753D
:10AAB000F003A4243BF582E43482F583E49390060A
:10AAC000C2F0EF75F003A42439F582E43482F583F3
:10AAD000E493FF7401939006C3CFF0A3EFF09006C8
:10AAE000C3E0FEA3E0FF9006C2E0FD12DC5D90062D
:10AAF000C1EFF01268462212DFA37F01124A7912D9
:10AB0000F1F6500B12F2E9C20812F05512F0F47F80
:10AB1000BF7E011227D69006B7EFF012D0899006BB
:10AB2000B8EFF070069009B4E060079006B8E0B4A2
:10AB30000E0F7FC07E011227D69006B7EFF012E20B
:10AB4000539006B8E014602314602814602D14603C
:10AB50001A2404702E9009B4E0B40108E4FD7F04C7
:10AB6000128E0A22E4FDFF128E0A22E4FD7F0412F7
:10AB70008E0A22E4FD7F02128E0A22E4FD7F031278
:10AB80008E0A22E4FDFF128E0A2212CAA39006B09A
:10AB9000EEF0A3EFF0E4A3F0EF2402FFE43EFE901A
:10ABA0000B0DE024FF92137D0712C7D89006B2E088
:10ABB000FF900A76E0FE5402FDC313FD25E025E078
:10ABC000FDEF4DFF9006B2F0EE5404FE1313543F18
:10ABD000FE33333354F84FF0E0FFEFC0E07F021252
:10ABE000D7F3EF5410FFC4540F25E0FED0E04E9091
:10ABF00006B2F0E0FFEFC0E07F0312D7F3EF54019D
:10AC0000FED0E04EFF9006B2F0FD9006B1E02405C4
:10AC1000FF9006B0E03400FE124FE4229006B0E44C
:10AC2000F0A374F8F0900BE8E0FFB4010A9006B0CE
:10AC30007401F0A3742DF09006B4E4F0A374FFF057
:10AC4000EFB4010A9006B47401F0A3742CF09006DE
:10AC5000B4E0FEA3E0FF900A0CE0A2E29213E4FD50
:10AC600012C7D8900BE8E06401603312B9A89006CF
:10AC7000B3EFF02456FFE43403FE1227D6EF54C09E
:10AC8000FF9006B2F0900A0FE0240A4FFF9006B240
:10AC9000F0FDA3E02456FFE43403FE124FE4900AD3
:10ACA00008E0FD7FF77E00124FE4129C5022900CCA
:10ACB00066121F0E900C64E0F582758300121B680B
:10ACC000FF8F34853434900D05E065346071E534D0
:10ACD00075F005A42414F582E43459F583E493FF58
:10ACE000126328E53475F005A42416F582E434597E
:10ACF000F583E493FF126333E53475F005A424155E
:10AD0000F582E43459F583E493FF126349E5347521
:10AD1000F005A42417F582E43459F583E493FF1277
:10AD20006354E53475F005A42418F582E43459F52C
:10AD300083E493FF12633E900D05E534F0D23D228B
:10AD4000900A0CE054BFF0E49006B4F09006B3F023
:10AD500030084E12EF06900A0CE04440F09006B323
:10AD60007409F0E4FD7F78FE12DC5D9006B4EFF02C
:10AD700012F29BEF600812F29BEF640E7023900BAF
:10AD8000E8E0B40505120BA44017900BE8E0B4040A
:10AD900003D38001C3400AE4FF1262FCE4FF1261A6
:10ADA0007212618A9006B5EFF09006B4E0FF12636C
:10ADB000759006B3E0FF12BDA512F29BEF60101272
:10ADC000F29BEF640E60089006B5E0FF12619622D8
:10ADD00012C0F512E88112EA4012F1A2E4FF1268F3
:10ADE000D9E4FF1268007F027E001227D6EF543F9D
:10ADF000FF12668B7F047E001227D6EF543FFF12AE
:10AE00006684E4FD7F38FE12DC5DEF5403FF1267B9
:10AE10004F7F251266457F1F1266307F1F126629FD
:10AE20007F081266227F2812665A7F1E1266537FA1
:10AE30000A12664C7F1912666F7F1A1266617F1EB6
:10AE40001265D57F251266687F2012663E7F20122C
:10AE500066377F1A1266767F1912667D229006ACDD
:10AE600074FFF0A37403F0E4A3F0900B9DE0FF30B7
:10AE7000E2099006AD7407F0E4A3F0EF30E16990C9
:10AE80000AC2E0FF20E36130E21912E2C35014125B
:10AE9000B4DC9006ACEFF07022900ACBE09006ACE8
:10AEA000F08018E4900ACAF0A3E09006ACF0900A93
:10AEB000C2E030E1069006AC74FFF09006AEE0FE12
:10AEC0009006ACE0FFC39E401FA3E0FEEF9E50182B
:10AED000900AC1E06F6011A3E020E00C12C205C22D
:10AEE0000C7F027E0A120B5C227F037E0012CEF4DE
:10AEF000121B4F9006ACF07F0312CEF490000112AB
:10AF00001B68FF9006ACE0FD12D0459006ADEFF057
:10AF10001209E250179006ADE0FFA2039208C209A1
:10AF2000AD2C12D4D59006ADEFF080159006ADE0B3
:10AF3000FFA2039208D209AD2C12D4D59006ADEF32
:10AF4000F07B017A0679AD12B2819006ACEFF06029
:10AF500014E0640E600F7F0312CEF4900001121B08
:10AF6000689006ADF09006ADE0FF9006ACE0FD12F3
:10AF7000D41E228F34853535853434E4900D0EF09F
:10AF8000125BB5EF64016006125BB5EF604C900D8B
:10AF9000197401F078AC7602900D017408F0E53474
:10AFA000B404057535018003E4F535900D23E0FF09
:10AFB000AD3512E410E534B409077F1F12614E80ED
:10AFC0000AE534906B1493FF12614EE4FF1262D0D5
:10AFD000E4FF1262837F01026283900D23E0FFE4AD
:10AFE000FD12E410900D197401F078AC763F900DCD
:10AFF00001E534F0FF12CCFB12F20A227B007A004A
:10B0000079009006AC121F171265C79006AFEFF0DB
:10B010001265CE9006B0EFF03001389006AFE02414
:10B02000FD70127BFF7A5579E49006AC121F1790E1
:10B0300006B17413F09006AC121F0EE94A6014E4D6
:10B040009006AFF0A3E0FFA3E0F53012C52890060C
:10B05000B0EFF0E4900BBBF09006AFE0900BB7F0D0
:10B060009006B0E0900BB8F0126AA5EF70047F0173
:10B0700080027F00900BBCEFF0126AA5900BBAEF34
:10B08000F0228F358B368A378938EF75F002A42489
:10B09000C1FFE5F03401FE12E16BAB36AA37A938E7
:10B0A000EE8FF0121D18AB36AA37A938121C68FFB4
:10B0B000AEF012D588400EAB36AA37A938740275A7
:10B0C000F0C4121D18E53524BCFFE43402FE12273B
:10B0D000D6AB36AA37A938900004EF121BC9AD359C
:10B0E0007F9A7E0212D74E40047F0180027F00EFDC
:10B0F0005401FFAB36E5382405F9E43537FA121B65
:10B100004F54FE4F121BB7228F368D37D20885362B
:10B1100036853737125BB5EF64016014125BB5EF0B
:10B12000700E125BB5EF6401605D125BB5EF705796
:10B13000E537B40800504E90B13D25E073214D2114
:10B1400054215B2162216921702177217EAF361263
:10B15000631D8033AF361261DE802CAF361263126E
:10B160008025AF361261AE801EAF361261EA8017BD
:10B17000AF361261BA8010AF361261C68009AF36A1
:10B180001261D28002C208A208229006AC7412F0AA
:10B19000E4A3F0900AC1E024FE6025146015146059
:10B1A0001F240370279006AD74F6F09006AC740C63
:10B1B000F080199006AD74F6F0E49006ACF0800CC7
:10B1C0009006AD74F6F09006AC740AF09006ADE00F
:10B1D000FE900AC8E0C39EFFC3EE9EFD9006ACE061
:10B1E000C39EFBA205920CC20D1246C69006ADE0AE
:10B1F0002F900AC8F0900ACDF0E4FF12BA11A20510
:10B20000E433FF12EEA4229006BF7401F0E4F0A331
:10B21000F0A3F0A304F012B3EEBF01139006BF74C5
:10B2200001F0900A7DE030E2069006C07401F01251
:10B23000B3EEBF0305E49006C2F0900CECE06005AD
:10B24000E49006C2F09006BFE0FF1269CE9006C0FF
:10B25000E0FF1268859006C1E0FF12687E9006C28A
:10B26000E0FF12686212B3EEBF030B7F0112688C1D
:10B270007F01126A6F22E4FF12688CE4FF126A6F8A
:10B28000228B488A49894A121B4FFF12D0899006A7
:10B29000FAEFF0E4A3F0A37463F0EF60089006FA0D
:10B2A000E0640E7050202E289006FAE0B40E21A320
:10B2B0007401F0A37428F07F0412E970AB48AA4926
:10B2C000A94A121B4FC39FFF9006FBE02F121BB72A
:10B2D000AB48AA49A94A121B4FFF9006FBE0FEEFBC
:10B2E000C39E400AA3E0FDEFD39D50028001C340FE
:10B2F00004EE121BB79006FAE0FF22900A0CE0540D
:10B30000CFF0900BE8E064016062900BE9E0640D1F
:10B31000605A12B9A89006C0EFF02456FFE4340337
:10B32000FE1227D69006BFEFF07FF67E001227D6DA
:10B33000900A01EFF09006BFE0FF541F24F6900A38
:10B340000FF09006C0E064296022EF54C0FF900621
:10B35000BFF0BF4009900A0CE04420F0800E900638
:10B36000BFE0B48007900A0CE04410F0900A01E0BE
:10B37000FF12924322757407C21D7F06126A7D3048
:10B380001C6B12F241C3EF947CEE9403500B7F7C54
:10B390007E0312E8B77574052212F241C3EF94C818
:10B3A000EE9403500B7FC87E0312E8B77574052234
:10B3B00012F241C3EF94FCEE9403500B7FFC7E032A
:10B3C00012E8B775740522900BBDE054FDF07F02C2
:10B3D000126A7D12F241C3EF94E4EE940650087FA6
:10B3E000E47E0612E3C62212F24112E3C622E49082
:10B3F00006EBF012F29BEF7006900A78E0600612FE
:10B40000F29BEF603E126548EF121F20B42B01B48F
:10B410003302B42B03B43304B42B05B43306B42B7A
:10B4200007B43308B43B0A0000B45F9006EB740124
:10B43000F0802C9006EB7402F080249006EB7403ED
:10B44000F0801C900A78E024FE24FD500C24047047
:10B450000E9006EB7403F080069006EB7402F090F9
:10B4600006EBE0FF22120B68900A7A7403F078A6CC
:10B47000E6FF125FF412F25A7F0112DECDE4900C67
:10B48000ECF0C2197F011268B6120B6E501CC3900B
:10B490000C99E09430900C98E0942A5009900B8716
:10B4A000E0C394284035120B7422C3900B61E094E2
:10B4B00030900B60E0942A5009900B87E0C39428E9
:10B4C0004006900B877401F0900B87E064016003E5
:10B4D000E014F0900B87E0FF12E0C822900AC1E070
:10B4E0009006AFF012BD429006B0EFF0900AC0E0B7
:10B4F0006F702D30CA2AE5BA20E425900AC2E054C4
:10B50000EFF0900ACAE004F0E4900ACCF0900ACA86
:10B51000E064087036F09006B0E09006AFF0802B43
:10B520009006B0E0900AC0F0900AC2E04410F0909B
:10B530000ACCE004F0E4900ACAF0900ACCE0B40827
:10B540000AE4F0900ACBE09006AFF0C2CA9006AFD2
:10B55000E0FF22900A0B7409F012BC7BEF121F204F
:10B56000B5A700B5AF01B5B702B59F03B5BF04B528
:10B57000A705B5AF06B58207B5AF0AB5AF0B00009A
:10B58000B5C5900A13E0D3940A5005E004F0803565
:10B59000E4900A13F0900A11E0FF12C03E8026905A
:10B5A0000A0B7404F0801E900A0B7401F080169050
:10B5B0000A0B7403F0800E900A0B7402F080069060
:10B5C0000A0B7406F012EE7122900AC2E020E367C3
:10B5D000900D3CE07061900B9DE030E135E4900A05
:10B5E000CCF0900ACAF0A3E0FF900AC1E06F600CB3
:10B5F00012C205C20C7F027E0A120B5C12F29BEF94
:10B600006401603312F29BEF6402602B7F0212BA76
:10B610001122900ACBE0FF900AC1E06F601912F28C
:10B620009BEF640E6011900ACBE0FF12C205C20CC2
:10B630007F027E0A120B5C22900A09E0121F20B6DC
:10B640006400B67001B69702B66403B68F04B6778D
:10B6500006B67F07B68708B68F09B6770BB67F0C9C
:10B660000000B69DE49006B1F07F011262FC802DCF
:10B67000E49006B1F080269006B17403F0801E902D
:10B6800006B17404F080169006B17401F0800E903B
:10B6900006B17402F080069006B17402F09006B113
:10B6A000E0FF12CB87228F368D37D209853636855B
:10B6B0003737125BB5EF64016014125BB5EF700EA3
:10B6C000125BB5EF64016048125BB5EF7042E5377D
:10B6D00024FE601714601B14601F1460231460277D
:10B6E0002406702AAF361262FC8025AF3612617EC6
:10B6F000801EAF3612615A8017AF36126307801072
:10B70000AF361261A28009AF361261968002C2097B
:10B71000A20922E49006B0F0A3E52CF0E4A3F0E542
:10B720002D908337939006B3F0E52D90833D939051
:10B7300006B4F09006B3E0FB9006B0E0D39B502F28
:10B740009006B2E070299006B1E0FF9006B4E0FDEB
:10B75000A207920CD20D1246C69006B1EFF012D994
:10B7600076E4339006B2F09006B0E004F080C49026
:10B7700006B2E060079006B1E0FF8002AF2C221213
:10B78000B9A89006AEEFF06429605EE02456FFE4AD
:10B790003403FE1227D6EF543F9006ADF0900A090D
:10B7A000E0602114601E24FA601224FC600714601B
:10B7B0000B24067017E49006ACF080169006AC746B
:10B7C00040F0800E9006AC7480F080069006AC7459
:10B7D000C0F09006AEE02456FFE43403FE9006ACC1
:10B7E000E0FDA3E04DFD124FE4228F2C1269DC90A6
:10B7F0000A76E0549FFFF0E52CC43354604FF022EA
:10B800008F35853535ED14602414603D24FD604B83
:10B8100024057056E535B4010A7F011263287F01C3
:10B82000026333E4FF126328E4FF026333E535B4B7
:10B83000010AE4FF12680E7F07026815900CF5E01C
:10B84000FF1268157F0102680EE535B401057F0718
:10B85000026807900CF1E0FF026807E535B40105C6
:10B860007F0102633EE4FF12633E228E2C8F2D8DFA
:10B870002E8B2FE52E1313543F7E00252DFFEE3522
:10B880002CFE9006B3F0A3EFF0E52E5403906AE18E
:10B89000939006B2F01227D69006B1EFF0A3E0F431
:10B8A0005F9006B1F0E52E540325E0FFC374069FB8
:10B8B000FFE52FC8EFC8088002C333D8FCFF90060D
:10B8C000B1E02FF09006B3E0FEA3E0FF9006B1E0F8
:10B8D000FD124FE42212F2419006AEEEF0A3EFF01B
:10B8E000900BBDE054FEF03006229006AEE475F0F9
:10B8F00001121C52D39006AFE094A09006AEE094E3
:10B900003740297437F0A374A0F080209006AE74FD
:10B91000FFF5F0121C52C39006AFE094C49006AE3F
:10B92000E0940250077402F0A374C4F0900BBDE0E1
:10B9300054F7F09006AEE0FEA3E0FF12A0BC227F19
:10B94000201266F47F201266FB7F20126702E4FF5C
:10B950001266ED7F3A1266D87F3A1266DF7F3A129E
:10B9600066E67F20126B817F1A7E001227D6EF5485
:10B970003FFF1266BC7F1C7E001227D6EF543FFFAC
:10B980001266CA7F1B7E001227D6EF543FFF126655
:10B99000C37F1D7E001227D6EF543FFF1266A01210
:10B9A000F07F7F02126A29229006C17429F0900963
:10B9B000B5E0121F20B9D100BA0501B9F902B9F3F7
:10B9C00003B9FF04B9ED0AB9ED0CB9ED100000BAE6
:10B9D0000B12F2A1EFC39400403112F2A1EFD39405
:10B9E00028502812F2A19006C1EFF0801E9006C1E7
:10B9F000E004F09006C1E004F09006C1E004F0908D
:10BA000006C1E004F09006C1E004F09006C1E0FF3A
:10BA100022E49006C1F0900AC2E054D0F0900ACE21
:10BA2000EFF024FD602C047035900B9DE030E114A4
:10BA30009006C17401F0E4900ACCF0900AC2E04490
:10BA400004F0802DE4900ACEF0900AC2E04401F0A8
:10BA5000801F900AC2E04408F04410F08013EF7099
:10BA600009900AC2E04401F08007900AC2E0440253
:10BA7000F09006C1E0FF12F11B227FC07E01122769
:10BA8000D68F2DE52DC394004009E52DD394635046
:10BA9000028001C34003E4F52D7FA07E3712E8B792
:10BAA000AF2D12DA783003079009C4E04420F01279
:10BAB00087CB9009C4E0FF30E6089009B37401F029
:10BAC0008005E49009B3F0EF30E6089009B4740102
:10BAD000F08005E49009B4F0EF20E605AF2C12E306
:10BAE0003222EF1470397F0112BA119006C074052A
:10BAF000F0900B9DE030E203D38001C34008900A30
:10BB0000CBE09006C0F09006C0E0FF900AC1E06F65
:10BB1000603712C205C20C7F027E0A120B5C227FC4
:10BB20000212BA11900B9DE030E103D38001C340B3
:10BB300018900ACBE0FF900AC1E06F600C12C205BA
:10BB4000C20C7F027E0A120B5C228D2E12DBA08FAC
:10BB50002F12F2FB5022E52F75F007A424A3F582E3
:10BB6000E43446F583E582252EF582E43583F583BA
:10BB7000E4939006ACF08033E52F75F007A42480A1
:10BB8000F582E43446F583E582252EF582E435839B
:10BB9000F583E4939006ACF0E52FB4040EE0B40214
:10BBA0000A12F28E4005E49006ACF09006ACE0FF7D
:10BBB000229006BC7401F0A374BFF012F2A1EFC092
:10BBC000E012F29BCDEFCDD0E0FF12D0459006BE43
:10BBD000EFF012E89C501A12F29BBF0E2B9006BC9D
:10BBE0007401F0A3746EF012F2A19006BEEFF08023
:10BBF000179006BEE0FF12D089EF700C9006BEE0F1
:10BC0000FD7FC07E01124FE49006BCE0FEA3E0FF82
:10BC1000A3E0FD124FE422300131EFFD900B60E410
:10BC20008DF0121C52D3900B61E09430900B60E0C9
:10BC3000942A403B3019067C2A7D3080047C227D8A
:10BC40002E900B60ECF0A3EDF08024C3900B61E02C
:10BC50009FFF900B60E09400FEF0A3EFF0C3942EE2
:10BC6000EE9422500A900B60742AF0A37430F09086
:10BC70000B60E0FEA3E0FF12DD6F229006B07407B8
:10BC8000F0125BB5EF64016006125BB5EF600690E1
:10BC90000D01E0FF22900D19E0FF6029640460258A
:10BCA000EFB401089006B07408F0802D900D01E00B
:10BCB000FE6003B40507E49006B0F0801C9006B067
:10BCC0007401F08014EFB404089006B07407F0809B
:10BCD00008900D01E09006B0F09006B0E0FF227FE2
:10BCE0000112692D12F197D227900A7A7402F07826
:10BCF000A6E6FF125FF478A6E6FF7DC87C00125628
:10BD0000E078A6E6FF7D0812001678A6E6FF125836
:10BD10007E900CEC7401F0900BBDE054F7F0C2A3E0
:10BD2000900B5B7401F0900BB8E0FFB45604D21A8C
:10BD30008006EFB45502C21AC20B7401FFFE120C4A
:10BD40000422E5BA540F9006B3F0E0604AE490068E
:10BD5000B1F09006B1E0FFC394085043EF90834BDD
:10BD6000939006B2F0900B9DE030E209EF90834390
:10BD7000939006B2F09006B2E0FF540FFEA3E06E7F
:10BD8000700DEF54F0FFC4540F9006B2F080109085
:10BD900006B1E004F080BB900AC9E09006B2F090D2
:10BDA00006B2E0FF228F31853131853232E531D361
:10BDB000940D400375310D125BB5EF6401601412F0
:10BDC0005BB5EF700E125BB5EF64016033125BB5CB
:10BDD000EF702DE531B40C10900CEEE0700204F021
:10BDE000E4FDFF129EBC8013900CEEE0B4010CE465
:10BDF000FD7F07129EBCE4900CEEF0AF3112C3132E
:10BE0000900CF7E531F022E49006ACF0A304F012B8
:10BE10006550EF5401FF900A7BE0FE25E04FF09063
:10BE20000A7AE024FE601214601614602424047060
:10BE3000269006AC7402F0801EE49006ADF08017E8
:10BE4000900A7BE0540F640F600DE49006ADF08023
:10BE5000069006AC7403F09006ACE0FF1268BD904B
:10BE600006ADE0FF1268A822900A0DE030E20D90C6
:10BE70000BE8E064057050120BA4504BA222500254
:10BE80008001C34042900BE8E0B4040C9009E7E065
:10BE90007003D38001C3502F900A0CE054FDF0C210
:10BEA0000812EF66900A0CE020E00312F1ECE4FDCA
:10BEB000FF12DF4E900AE0E06006900AEBE06007B8
:10BEC0007D01E4FF12DF4E22E49006ACF012F29BFB
:10BED000EF7053900A0AE0FFB402089006AC7401B8
:10BEE000F08010EF700D900A0BE0B402069006ACE3
:10BEF0007401F09006ACE06005E4FF1267879006DD
:10BF0000ACE060047F0180027F0012678012EA7457
:10BF100050067E007F0380047E007F021227D6EF4A
:10BF2000543FFF12668B228F38E4F539900B9DE069
:10BF300030E212753906900BA1E030E6057539053F
:10BF40008003753906E53864046008E538600464E8
:10BF500003702FE538B404047D0080027D017F85E5
:10BF60007E0312DC5D8F39E538B40416900B9DE03A
:10BF700030E20F900BA1E030E605753905800375BE
:10BF80003906AF392212F29B9006ADEFF0900BE824
:10BF9000E0B40107900A7DE054FEF0900A7DE0FFD6
:10BFA00030E03E20E13B12E2C350369006ADE0FFA8
:10BFB0007006900A78E06003EF602612F29BBF04DF
:10BFC0000312F33C12B3EE9006ACEFF0900A7EE061
:10BFD0006F600E9006ACE0900A7EF012EF7612F3DE
:10BFE0003D228E328F338B34EDC3137E002533FF19
:10BFF000EE3532FE9006C0F0A3EFF0ED5401906AEA
:10C00000E5939006BFF01227D69006BEEFF0A3E0AE
:10C01000FEF45F9006BEF0EEB4F00BE534C454F0CD
:10C02000FFE02FF080079006BEE02534F09006C0B8
:10C03000E0FEA3E0FF9006BEE0FD124FE422900A6E
:10C040000AEFF0A3F0121F20C08B00C06101C0688E
:10C0500002C06F03C07604C07D06C084070000C024
:10C0600096E4FF12AF73802E7F0212D21F80277FCB
:10C070000112AF7380207F0312D21F80197F041238
:10C08000D21F80127F0F12D21F800B7F0912AF7355
:10C09000900A0B7408F012EE71229006AF7401F052
:10C0A000FB7A0679AF12B2819006B0EFF09009BA30
:10C0B000F06005E49006AFF09006AFE09009BBF0A9
:10C0C00078C67C097D017B017A0979BA7E007F02FE
:10C0D000121B079006AF7401F09009BC740EF0A318
:10C0E0007401F078C87C09FDFB7A0979BC7E007F79
:10C0F00002121B0722E4FF1269427D067FAE7E001A
:10C1000012D74EE433FF12693BE4FF1269347F011A
:10C1100012692DE4FF126926E4FF12691FE4FF1281
:10C1200069187F011269117D0F7FAE7E0012D74E14
:10C13000E433FF12695E7D077FAE7E0012D74EE4C6
:10C1400033FF1269577F01126950E4FF12694922D7
:10C150008E308F3112D5885051900B81E530F0A38D
:10C16000E531F0900B85741FF0A3E04401F012F16B
:10C1700097900BBDE054F7F012C62D900B81E0FEB6
:10C18000A3E0FF12E8B7900B86E05401FF3333338E
:10C1900054F8FF900BBDE054F74FF0900A7DE04457
:10C1A00001F0E4FF12DECD12F0F4221264A090063A
:10C1B000ADEFF0900A6AE06F703D900A82E004F003
:10C1C000E0640A703FF09006AEF0900A81E0FF90C4
:10C1D00006ADE0C39F4004A37401F0900A83E0FF22
:10C1E0009006AEE06F601DE0900A83F024FF920895
:10C1F00012E30D12AA6422E4900A82F09006ADE0E8
:10C20000900A6AF022900AC1EFF0900AC9F0900AF1
:10C21000C2E0FF30E22D20E42A900B9DE030E215D1
:10C22000900AC1E0701D900BE8E0FF12BF27900A52
:10C23000C1EFF0800E900AC1E07008900ACBE09048
:10C240000AC1F01209825008900AC1E0900ACBF0AE
:10C25000900AC1E0FF12DEF89009E7740AF022901C
:10C260000AC2E0FF30E351900A40E030E31F900B38
:10C27000E9E0B40418900BD9E020E011EF20E60DBE
:10C280004440900AC2F0C20AD20B129F81900BE97F
:10C29000E06405600E900BD9E020E007900A40E0D2
:10C2A00020E315900AC2E030E60ED20AD20B129FAC
:10C2B00081900AC2E054BFF02212F287505112F36B
:10C2C000279006ACEFF0C394144006E0D394EB4003
:10C2D0002B9006ACE0FE75F00AA475F01984FFEE11
:10C2E000D394EB400E74FF9E75F00AA475F0198488
:10C2F000F404FF12C87CD21DE4F574229006ACE071
:10C30000C3947F50047F0480027FFC12C87C227596
:10C310007403228F33853434853535125BB5EF6471
:10C32000016014125BB5EF700E125BB5EF64016033
:10C330003B125BB5EF7035E4F534F535E533601845
:10C3400024FC5002800AE53390601E93F534800887
:10C35000E53390601E93F535AF3412636AAF351242
:10C3600061F67F011263DBE4FF1263DB22C20890F7
:10C370000BE8E0B40503A20822EF14601614602352
:10C3800014602414603024047039120B9E5034D28F
:10C39000088030900B9FE030E629120B9E5024D28B
:10C3A000088020D208801C900B9FE0FF30E31430FF
:10C3B000E611D208800D900B9FE0FF30E20530E5DA
:10C3C00002D208A208228F368D378B3812CEF49015
:10C3D00006BC121F17E536547FFF7E009006BFEEA5
:10C3E000F0A3EFF0EE7037EF602914601714702E91
:10C3F0009006BC121F0E900001E537121BC9E538EC
:10C40000121BB7229006BC121F0E900001E53712D6
:10C410001BC9229006BC121F0EE538121BB72290D2
:10C4200006BB7423F0A3748CF03008319006BA7404
:10C4300005F07F011267BF7F011267E2900BBDE03C
:10C4400054F7F09006BBE0FEA3E0FF12CC67900B20
:10C450005DE04401F0900B5C7406F08012900BBD1F
:10C46000E04408F0E4FF1267E29006BA7407F09027
:10C4700006BAE0FF126A6122E4FB7D017F0E120B17
:10C48000207F0112692D12F16B900A7A7402F0D2AA
:10C4900027E4FF12DB0E12E3EB12E3A1C23B900B89
:10C4A000877401F0900CEC7403F0900BBDE054F72E
:10C4B000F0C2A312EF36120B26120B2C7F3C12E2B5
:10C4C00007C21CE4FF12673A7FC47E0212E3C62251
:10C4D0008F307F0312CEF4900001121B689006B4D7
:10C4E000F0E530D3940340047F0480027F0090067F
:10C4F000B5EFF0E530B40C037403F09006B5E0FF3F
:10C5000012BF279006B5EFF0E530D39403500890A2
:10C5100009B5E094034003120BB09006B4E0FDA30C
:10C52000E0FBAF30120BB6228F2C8B2D8A2E892F79
:10C530009006B274FFF0E4A3F09006B3E0FFC39559
:10C54000305036AB2DAA2EA92F75F002EFA4F5823C
:10C5500085F083121B68652C7017EF75F002A42913
:10C56000F9EA35F0FA900001121B689006B2F080EB
:10C57000089006B3E004F080C09006B2E0FF22907D
:10C580000A09E0FF900A24E06F6042900A0CE0FE86
:10C5900020E60330E732EF24FC600824FB6004242B
:10C5A000077020900B9DE030E30BEE30E607D208D9
:10C5B00012AD408018900A0CE030E711D20312EC63
:10C5C0003F800A12D0CD8005C20312EC3F900A09C9
:10C5D000E0900A24F022900A09E024FC600824FB81
:10C5E00060042407702A9006E67402F0900B9DE028
:10C5F00030E30F900A0CE030E6089006E67404F091
:10C600008025900A0CE030E71EE49006E6F08017E3
:10C610009006E67403F0900A0CE0FF20E70330E692
:10C62000069006E67401F09006E6E0FF22900A7894
:10C63000E064017036C3900B82E094E4900B81E0DB
:10C640009406500E900BBDE04402F07F06126A7D06
:10C65000800C900BBDE054FDF07F02126A7D7F01DB
:10C6600012673AD21C7F0212678722900BBDE054FA
:10C67000FDF07F02126A7DE4FF12673AC21C7F035D
:10C6800012678722A20A920A125BB5EF6401601456
:10C69000125BB5EF700E125BB5EF6401603B125B8D
:10C6A000B5EF7035300A197F011263287F011263DC
:10C6B000337F011263497F011263547F0102633E9D
:10C6C000E4FF126328E4FF126333E4FF126349E4DA
:10C6D000FF126354E4FF12633E227F0112692D12A0
:10C6E000F16B900A7A7402F0D227900CEC14F012DD
:10C6F000F241900B81EEF0A3EFF0900BBDE054F708
:10C70000F0C2A312EF367F3C12E207900A78E0B441
:10C7100001117F5A12E207900B81E0FEA3E0FF12A5
:10C72000E72222900B81E0FEA3E0FF12E3C6221273
:10C73000E74112E621900BEAE030E02C12C09A7F2C
:10C74000037E0012CEF4121B4FFF9006ADE4F0A35F
:10C75000EFF07F0312CEF4900001121B68FB9006ED
:10C76000AEE0FD7F05120B2078B87C097D017B01CE
:10C770007A0979BA7E007F02121B0712F29B900998
:10C78000B2EFF022900CECE024FE6030047048120E
:10C79000CC1D500712DD9C12A77222301B39900A63
:10C7A00078E0B401097FC47E0212E72280077FC4CB
:10C7B0007E0212E3C6900CEC7402F02212CC1D40F3
:10C7C0001012F241C3900B82E09F900B81E09E50CB
:10C7D0000612DD9C12A77222ED131313541F2FFFB4
:10C7E000E43EFE787AF608EFF6ED54077878F6081E
:10C7F0007601E6FD18E6FCEDC8ECC8088002C333FC
:10C80000D8FC7879F61227D67878EFF608E6FEF4A9
:10C810005F18F6A213E4338EF0A426F6787AE6FECB
:10C8200008E6FF7878E6FD124FE4227F0112692DB9
:10C8300012F197900A7A7402F07F0E12DB0ED22763
:10C8400078A6E6FF125FF478A6E6FF7DC87C0012AA
:10C8500056E078A6E6FF7D0812001678A6E6FF12DD
:10C86000587E900CEC7403F0900BBDE054F7F0C2CE
:10C87000A312EF367F2E7E2212EF26228F2C12F289
:10C8800041AD2CED3395E0FCEF2DFFEE3CFE900624
:10C89000ADF0A3EFF0D394A0EE9437400E9006AD28
:10C8A0007437F0A374A0F0D21B8016C39006AEE0DC
:10C8B00094C49006ADE0940250077402F0A374C4CF
:10C8C000F09006ADE0FEA3E0FF12A0BC227F037E45
:10C8D0000012CEF4121B4F64037041126550EF60DA
:10C8E0003BE4752FFFF52EF52DF52CAF2FAE2EADB9
:10C8F0002DAC2CEC4D4E4F601374FFFBFAF9F8127F
:10C900001D648F2F8E2E8D2D8C2C80DF126548EFAD
:10C91000700A7F011268B6E4FF1268B622E490063E
:10C92000FAF0900B9FE0FE30E305EF64026009EE41
:10C9300030E232EF6403702D74017E00C8EFC80846
:10C940008005C333CE33CED8F9FF9009BEE0FDE4B5
:10C95000EF5D7003D38001C340047F0180027F003C
:10C960009006FAEFF09006FAE024FF221265389064
:10C9700006BFEFF0E4A3F0900A7DE030E2339006CA
:10C98000BFE0FF64086010EF24FD6003047019909D
:10C9900006C07401F08011126548EF24FE600304A4
:10C9A00070069006C07401F03008069006C074034B
:10C9B000F09006C0E0FF1266A722201B0512F01DB2
:10C9C000500412A8A32212CC1D503C12DD9C900BE7
:10C9D00087E0FF7B017A0B798112CD45900B87E0D0
:10C9E000FF120B7A900B87E0FF12EF16900B87E097
:10C9F000FF12D199900B87E0FF12ED69900B87E051
:10CA0000FF120B8012F0DA22900A01E0FF900BB8BF
:10CA1000E0FE64106004EEB45603C38001D39213A9
:10CA2000754664E4F547125C56900A01EFF01292E5
:10CA300043900A0CE030E01D900BB8E0B4101620D3
:10CA40002E1312D635C20C7F407E0E120B5C7F0176
:10CA50007E02120BDA22A22250028001C340437FE1
:10CA60001A7E001227D6EF543FFF1266BC7F1C7E51
:10CA7000001227D69006BFEFF07FEB7E001227D67C
:10CA8000EF540FFFBF030C7FB47E071227D690062A
:10CA9000BFEFF09006BFE0543FFF1266CAE4FF12FA
:10CAA00065F1229006C3E4F0A374B6F012F2A190EF
:10CAB00006C5EFF0E4A3F012F29BEF1460161460C9
:10CAC0000D24FE600F04701F9006C6E004F090066F
:10CAD000C6E004F09006C6E075F006A424D4FF90EA
:10CAE00006C3E4F0A3EFF09006C3E0FEA3E0FF224C
:10CAF00012EAF2900D23E0FF12F262E4FF12D21F5D
:10CB0000E4FDFF128E0AD20812EF66E4FDFF12DF89
:10CB10004E125BB5EF64016014125BB5EF700E123C
:10CB20005BB5EF64016014125BB5EF700E7D01E43C
:10CB3000FF128E0A7D01E4FF12DF4E227F78125130
:10CB4000C87878E6FF9006B1E4F0A3EFF0E0FE08C5
:10CB5000E67C002400FFEC3EFE9006B1F0A3EFF06F
:10CB6000C3900A26E09F900A25E09E4015900A2770
:10CB7000E0FEA3E0FFD39006B2E09F9006B1E09EF6
:10CB80004003D38001C3228F2C900D24E52CF0129A
:10CB90005BB5EF64016006125BB5EF6017E4FF124E
:10CBA000CBD2EF702CE52C6003B40103752C07AFDA
:10CBB0002C02DDF4125BB5EF64016015125BB5EF7A
:10CBC000700FE52C6003B40103752C07AF2C12DD48
:10CBD000F422E49006B2F0EF7013900D08E07004B8
:10CBE0007E0180027E009006B2EEF0802ABF011323
:10CBF000900D1AE070047E0180027E009006B2EE75
:10CC0000F08014BF0211900D1BE070047F018002C0
:10CC10007F009006B2EFF09006B2E0FF22E57412BA
:10CC20001F20CC5200CC5701CC5C02CC6103CC3E1F
:10CC300004CC4305CC4806CC4D070000CC6412B3AD
:10CC4000758021757406801C757407801712F1AD0C
:10CC5000801212D716800D12EE4D800812C2B980D4
:10CC60000312E865A21D22CBEFCBCAEECA900C9846
:10CC7000EAF0A3EBF07C007D05121BFDEF24D6FB50
:10CC8000E43EFA30190F787876D80876C00876C076
:10CC9000087609800D7878769808764008768008BE
:10CCA0007609787CEAF608EBF67D787F0612EBCB06
:10CCB000228F2CA2019201852D2DE52C30E207D286
:10CCC00001E4F52D8022E52C30E307D201752D011A
:10CCD0008016E52C30E407D201752D02800AE52C80
:10CCE00030E105C201E4F52DA2019202125CDCAF35
:10CCF0002D1263D1900CF3E52CF0228F36900CF0BE
:10CD0000E536F0853737125BB5EF64016006125BDC
:10CD1000B5EF601DE536905D3793FF641360251213
:10CD2000614E7F011262D0E4FF1262837F010262D2
:10CD300083125BB5EF6401600B125BB5EF7005AF5A
:10CD40003612DAAB228F308B318A328933EF75F0AD
:10CD500002A424C1FFE5F03401FE121C68FDACF012
:10CD600012ED2DE53024BCFFE43402FEAB31AA32D3
:10CD7000A933900004121B68FD124FE4900B86E06B
:10CD800013B39213AD307F9A7E0212C7D822E4FF0C
:10CD90001269F17D257FAE7E0012D74EE433FF127B
:10CDA00069EAE4FF1258407D2F7FAE7E0012D74E15
:10CDB000E433FF1269E37D017F3A7E0012DC5DEF10
:10CDC0005403FF1269DC7D1D7FAE7E0012D74EE456
:10CDD00033FF1269D52212F29BEFC39401403E1239
:10CDE000F29BEFD394035035126590EF602112CB84
:10CDF0003C501C9009C5E07024FF12677212F29B30
:10CE0000BF02057F021268389009C57401F02290B4
:10CE100009C5E06003128353E49009C5F0228F3600
:10CE2000D208853636ED601D24FD602E2402703157
:10CE3000900CF5E536F0126530EF64076025AF36EB
:10CE4000126815801E900CF1E536F0126528EF642B
:10CE5000076010AF361268078009AF3612681C8071
:10CE600002C208A208227D2B7FAE7E0012D74EE4BC
:10CE700033FF1269C77D057FAE7E0012D74EE433C3
:10CE8000FF1269C0E4FF1269B97D2C7FAE7E0012EB
:10CE9000D74EE433FF1269B2E4FF1269AB7F01128F
:10CEA00069A4E4FF1265F1E4FF1265F8228F348D66
:10CEB0003512D45B40347F0312CEF4900001121B74
:10CEC00068FDEDC0E07F037E0012CEF4121B4FFB25
:10CED000D0E0FD7F8212C3C67B01AD347F0112C357
:10CEE000C6AB357D01E4FF12C3C6AB34AD357F055B
:10CEF000120B20228F397B017A0979BA9006C11270
:10CF00001F177A0979C69006C4121F1712E89C50A1
:10CF1000167B017A0979BC9006C1121F177A09792C
:10CF2000C89006C4121F17E53930E7089006C412EE
:10CF30001F0E80069006C1121F0E2212F1D8E49037
:10CF40000AC7F0900AC1F0900B9DE030E203D38055
:10CF500001C3400C900AC1E0FD7F857E03124FE4BF
:10CF6000900B9DE030E20D900BE8E0FF12BF2790A0
:10CF70000AC1EFF0900AC1E0FF900ACBF012DEF890
:10CF8000228F2C852C2C125BB5EF64016014125B90
:10CF9000B5EF700E125BB5EF64016029125BB5EF5F
:10CFA00070237410252CF52CD36480949F40057554
:10CFB0002C1F800CC3E52C648094805003E4F52C76
:10CFC000AF2C125E642212E89C5034120C0AEF64FB
:10CFD00009702C7F02FE120C105024D20C7F027EAE
:10CFE00000120B5CD20C7F027E05120B5C7401FFF9
:10CFF000FE120C105009D20C7401FFFE120B5C22C1
:10D000008F2C852C2C125BB5EF64016014125BB57C
:10D01000EF700E125BB5EF64016029125BB5EF7023
:10D02000237410252CF52CD36480949F4005752C17
:10D030001F800CC3E52C648094805003E4F52CAF72
:10D040002C125F8B228F468D479006F9E546F0E55E
:10D05000476030FF12D785EF24639006F9F0E5476B
:10D06000B40E20E546C394014009E546D394285008
:10D07000028001C34003754601E54614FF9006F99E
:10D08000E02FF09006F9E0FF22E49006FDF0A37493
:10D0900063F0C3EF9463A3F0EFD394634029900B44
:10D0A0009BE030E6157F0E12D7859006FFE0C39F08
:10D0B00040089006FD740EF0800D9006FFE0FF1210
:10D0C000D86E9006FDEFF09006FDE0FF22900A0C6E
:10D0D000E04480F0900B9DE030E307900A0CE044C0
:10D0E00040F09006B37401F0A3F012C5D6EF7009BA
:10D0F0009006B37402F0E4A3F09006B3E0FF12BD13
:10D10000A59006B4E0FD7F5E7E0012DC5D12620E2B
:10D1100022EF3395E0900BBF8FF0121C52D3900B8F
:10D12000C0E094A0900BBFE0943740077437F0A3A1
:10D1300074A0F0C3900BC0E094C4900BBFE09402C5
:10D1400050077402F0A374C4F0900BBFE0FEA3E09C
:10D15000FF12A0BC22CDEFCDCCEECC900BBEE06494
:10D1600003601BD3ED94A8EC941B40037F0422D3EF
:10D17000ED94D4EC940940037F02227F0122D3ED89
:10D1800094F4EC941A40037F0822D3ED9464EC9459
:10D190000940037F02227F01228F2C7F837E0012B1
:10D1A000CEF4121B4F9006B0F07B01AD2C7F011224
:10D1B000C3C67F0312CEF478B87C097D017E007F60
:10D1C00002121B079006B0E0FF600D640E60097B41
:10D1D00001AD2C7F8112C3C612BBB1228F2E12F279
:10D1E0009B9009B2EFF0900BBDE04420F09009C491
:10D1F000E04440F09009B47401F09009C2E52EF0CB
:10D2000012F2A19009C3EFF078B87C097D017B018F
:10D210007A0979C27E007F02121B0712F02B228F3F
:10D2200034AD05853434E4900D0EF0900D01E534F5
:10D23000F0B404047D018002E4FD900D23E0FF12B0
:10D24000E410AF3412CCFB125BB5EF640160061240
:10D250005BB5EF600C78AA760178A9760178AB7699
:10D2600001229009B0E0B4021A12F29BEF6008901C
:10D270000A7A7404F08006900A7A7402F07F011230
:10D2800068D2229009B0E0B4031912F29BEF600853
:10D29000900A7A7404F08006900A7A7403F0E4FF2E
:10D2A0001268D222900B9CE030E4047F0180027F60
:10D2B00000BF0130E4900B0EF07F0112F2DD12F29C
:10D2C0009BEF700B9006CF04F0A37455F0800A908A
:10D2D00006CF7401F0A37460F09006CFE0FEA3E0E7
:10D2E000FF12D9AA227F037E0012CEF4121B4F70C8
:10D2F000099009C4E0547FF080079009C4E044809D
:10D30000F09009C4E054BFF0900BE8E0700490097D
:10D31000B4F07F0312CEF478B87C097D017E007FE3
:10D3200002121B072212E89C503A900BD6E030E024
:10D3300013D20C7F837E00120B5CD20C7F827E05A1
:10D34000120B5C22C20C7F027E00120B5CC20C7FAF
:10D35000027E05120B5C7F027E00120BDA7F027EDA
:10D3600005120BDA22EF75F002A4246DFFE5F0340C
:10D3700001FE12E16B9006C1EEF0A3EFF0C3942E14
:10D38000EE9422400CD3E094309006C1E0942A4001
:10D390000A9006C17422F0A3742EF09006C1E0FE3C
:10D3A000A3E0FF228D34E5345403906AE1939006A4
:10D3B000CEF0E5341313543F2FFFE43EFE1227D680
:10D3C0009006CEE05FA3F0E534540325E0FFC3747C
:10D3D000069FFFE0FEC8EFC8088002C313D8FCFF19
:10D3E00022900BA0E030E43512E2C3502B126548C6
:10D3F000BF0221126568BF011BE49006ACF0900AE1
:10D4000083E060199006ACE0900A83F024FF920854
:10D4100012E30D2212C1AB22D20812E30D228F3289
:10D420008D3312F29B9009B2EFF0AF3312D54DADB0
:10D4300033AF3212CEAD12D2E512BBB112F02B9047
:10D440000D3CE06015E533D394004009E533247EBC
:10D45000FF120B8622AF32120B86228F368D37E4F5
:10D460009006BCF07F03FE12CEF4121B4F6537709E
:10D47000209006BC04F0E5376003B40E147F03125D
:10D48000CEF4900001121B6865366005E49006BC7E
:10D49000F09006BCE024FF22900B85E0FF70033083
:10D4A0000532EFB43E0320052BA205920CC20D7B82
:10D4B0003EE4FD1246C6900B85EFF0A205920612DF
:10D4C000B8D512F241900B81EEF0A3EFF0900B86ED
:10D4D000E054FEF0228F2D8D2EAF2E12D5FC90063B
:10D4E000B0EFF0AF2E12E9709006B1EFF0A3F0901C
:10D4F00006B0E0FB9006B2E0D39B50129006B1E07C
:10D50000FDA208920CD20DAF2D1246C68F2DAF2D65
:10D5100022900D3CE06007900A0CE054CFF0900A96
:10D520000BE0B4081D900A0AE0700C7F0912AF737B
:10D53000900A0B7409F022900A0AE0FFA3F012C0CF
:10D540003E22900A0BE0B4090312B553228F3490A7
:10D550000BE8E07032900BB9E0640160169008E9C6
:10D56000E0D39400500D900BB8E0FF64206004EF0E
:10D57000B421147F037E0012CEF4121B4F65346079
:10D58000069009B5E534F022900BE8E064016007ED
:10D59000900BE9E0B40D16C3EF942EEE9422400BED
:10D5A000D3EF9430EE942A50028001C322C3EF944B
:10D5B000C4EE9402400BD3EF94A0EE943750028057
:10D5C00001C3228E458F468D478B488A49894AABD5
:10D5D00048AA49A94A121B4FFDAF46AE45124FE477
:10D5E00050190546E546700205457401254AF54A7D
:10D5F000E43549F5491547E54770D4228F2F900649
:10D60000B37463F012D66E9006B3E02FF0202E1F95
:10D61000900B9BE030E618E52F6403600BE52F6468
:10D62000046005E52FB405079006B3E02427F090C9
:10D6300006B3E0FF22900A0CE0FF20E00F20E10398
:10D6400012EFFD900A0CE04401F08011900A0CE00A
:10D6500020E10312F1EC900A0CE054FEF0900A0C69
:10D66000E01392137D107FAE7E0012C7D822E490A3
:10D6700006B4F0A304F0EF908337939006B6F090D1
:10D6800006B6E0FE9006B5E0FFD39E501312D976A1
:10D6900050069006B4E004F09006B5E004F080DF98
:10D6A0009006B4E0FF227F027E001227D6900BB8CE
:10D6B000E0B45603C38001D3921375463FE4F547A7
:10D6C000125C569006AFEFF0FD7F027E00124FE431
:10D6D00012EA7440089006AFE0FF12668B227F03C7
:10D6E0007E001227D6900BB8E0B45603C38001D356
:10D6F000921375463FE4F547125C569006EDEFF045
:10D70000FD7F037E00124FE412EA7450089006ED8C
:10D71000E0FF12668B22900BBDE04401F012F2870D
:10D72000502612F241BE020ABFC407201D047574C0
:10D730000222900BBDE0FFC31330E0077F6012C8E8
:10D740007C80057F5012C87CC21D75740122ED13C8
:10D750001313541F2FFFE43EFE787AF608EFF6ED20
:10D7600054077878F6087601E6FD18E6FCEDC8EC7B
:10D77000C8088002C333D8FC7879F61227D67879A6
:10D78000E65F24FF22CDEFCDE4900700F012D976BA
:10D79000501F9007007401F0900700E0FFC3941140
:10D7A000500F12D86EEF6D6008900700E004F08013
:10D7B000E7900700E075F01184AFF02278BA7C069C
:10D7C0007D017B017A0979BA7E007F02121B073046
:10D7D000081378BA7C067D017B017A0979BC7E004A
:10D7E0007F02121B079006BBE0FF9006BAE0FD1215
:10D7F000D04522744C2FF582E4340BF583E0FF22F0
:10D80000A2099209125BB5EF64016006125BB5EFE5
:10D81000601D3009077F011262E68005E4FF126295
:10D82000E6900CF0E0B4040EA209920A02DDC8A250
:10D8300009920A12DDC82212F307EF7030900D1919
:10D84000F0900D01E0FF12E8ED4022900D01740709
:10D85000F0E478ACF622E4900D19F078ACF6229062
:10D860000D017407F0E4900D19F078ACF622CEEFBC
:10D87000CEE4900701F0A304F0900702E0FFC39408
:10D8800011501612D9765009900701E004F06E602D
:10D8900008900702E004F080E0900702E075F011C4
:10D8A00084AFF022E49006BFF0900A0AE0FFB401D2
:10D8B000089006BF7401F08010EF700D900A0BE025
:10D8C000B401069006BF7401F09006BFE060047FCB
:10D8D0000180027F001267562212F29B9006BFEF72
:10D8E000F064016005E064027023900D3CE0701D5F
:10D8F0009006BFE0B401099009C4E05403FF800A18
:10D900009009C4E0FF13135403FF12BAE2228E47BA
:10D910008F488D498B4A8A4B894CAF48AE471227B6
:10D92000D6AB4AAA4BA94CEF121BB77401254CF594
:10D930004CE4354BF54B0548E54870020547D549A1
:10D94000D9228E2E8F2F8D308B3112DC5D9006B157
:10D95000EFF0AD31AF2FAE2E12DC5DCBEFCBAD30A3
:10D96000AF2FAE2E12BFE29006B1E0FBAD31AF2F6C
:10D97000AE2E12BFE222EF602C64016028BF0207C6
:10D98000900B9FE020E61EBF0307900B9FE020E571
:10D9900014EF6409600FEF640A600ABF0E0A900B6F
:10D9A0009BE030E603D38001C3228E368F37E490AC
:10D9B00006D1F09006D1E0FFC3940B50207E00E525
:10D9C000372FFFEE3536FE1227D6CDEFCD9006D19C
:10D9D000E0FF12E1929006D1E004F080D622900B95
:10D9E0009CE030E4047F0180027F00BF0123E4FF5C
:10D9F00012F2DDE49006AFF09006AFE0FF9062AF68
:10DA000093FD12E1929006AFE004F0E0C3940B4066
:10DA1000E7221264A09006BFEFF0900BA0E030E484
:10DA200023E4900A82F0A374FFF0C20812E30D9081
:10DA30000A81E0FF9006BFE0C39F4005D20812E3D1
:10DA40000D12AA64228F2C20190F900C98E0FFA3CE
:10DA5000E0900B60CFF0A3EFF0E52C75F002A4246A
:10DA60006DFFE5F03401FE900B60E0FCA3E0FD12D9
:10DA7000ED2DAF2C12F32322EF75F002A424C1FF89
:10DA8000E5F03401FE12E16B9006AEEEF0A3EFF08C
:10DA900012D588400A9006AE7402F0A374C4F090C8
:10DAA00006AEE0FEA3E0FF12E8B7228F38853939D1
:10DAB000853838C208126445D208126445E53890AA
:10DAC000643C93FF640860031267B8E538B403054B
:10DAD0007539018003E4F539AF390267D48E348F8C
:10DAE000358C368D371227D69006B2EFF0AF37AEB1
:10DAF000361227D69006B3EFF0FDAF35AE34124F95
:10DB0000E49006B2E0FDAF37AE36124FE4228F2D1F
:10DB100012D976502912EF9412F29B9009B2EFF0CD
:10DB20007F0312CEF4900001121B68FFAD2D12CEC0
:10DB3000AD12D2E5900BBDE054BFF012835322C268
:10DB400027900A7A7403F078A6E6FF125FF4E49057
:10DB50000CECF0C218900C98E0FEA3E0FF12CC672A
:10DB60007F0112DECD900BBDE054F7F012D32522D9
:10DB7000900A76E05402FFC313600512E7BA8003EF
:10DB800012EBE312CAA3EF2405FFE43EFE900A76EF
:10DB9000E05402FDC31324FF92137D0212C7D82262
:10DBA000E49006ADF0EF30E7037401F0EF30E606E5
:10DBB0009006AD7402F0EF30E5069006AD7403F008
:10DBC000EF30E0069006AD7404F09006ADE0FF2261
:10DBD0008E308F318D328B3312D74E9206AD33AFEC
:10DBE00031AE3012D74E9213AD32AF31AE3012C7D4
:10DBF000D8A2069213AD33AF31AE3012C7D822BFD0
:10DC000001047F0280027F039006B7EFF0E4F52E57
:10DC10007D71122CB55005752E02800F9006B7E06D
:10DC2000FF7D2F122CB55003752E01AF2E22AC07AD
:10DC3000EDD3941F50079006B8ECF0801AC3743FE0
:10DC40009DFFE49400FEAD047C00121BEB7D1F12CF
:10DC50001BFD9006B8EFF09006B8E0FF22ED5401EE
:10DC6000906AE5939006C5F0EDC3132FFFE43EFEE6
:10DC70001227D69006C5E0FE5FA3F0EEB4F006E0F2
:10DC8000FFC4540FF09006C6E0FF22126568EF54FF
:10DC900001FF900A80E0FE25E04FF05407FF900658
:10DCA000B2F0BF0406E4900A79F0229006B2E0B424
:10DCB0000306900A797401F022300519E4FF126717
:10DCC000727D027F0112DF4EE4FF12682A7D017F20
:10DCD0000112DF4E221283537D02E4FF12DF4E7DDC
:10DCE00001E4FF12DF4E227D1A7FAE7E0012D74E76
:10DCF000500E7F9F7E031227D6900A01EFF0800C12
:10DD00007FF67E001227D6900A01EFF0900A01E01C
:10DD1000FF1292432212E89C5027C20B7F027E0022
:10DD2000120C04C20B7F037E00120C04120C16C2EC
:10DD30000B7F027E05120C04C20B7401FFFE120C55
:10DD40000422900BBDE054FEF012F3279006ACEFD6
:10DD5000F0C394034018E0FFD394FD5011EFC39437
:10DD60007F50067F0112D111227FFF12D11122CBE9
:10DD7000EFCBCAEECA900C98EAF0A3EBF07C007DE2
:10DD800005121BFDEF24D6FBE43EFA787BF6CFEBC1
:10DD9000CF08EFF67D7B7F0212EBCB2212F241908F
:10DDA0000B81EEF0A3EFF0900B85741FF0A3E0441D
:10DDB00001F0900CECE0B4030E301C067F0112E77A
:10DDC0000322E4FF12E70322300A0AE4FF1267E9A4
:10DDD0007F020267C6900CF0E0B40407E4FF12670C
:10DDE000C680057F011267C6900CF4E060057F01D4
:10DDF0001267E9228F34853434125BB5EF64016019
:10DE000014125BB5EF700E125BB5EF640160101277
:10DE10005BB5EF700AE5349064B093FF1261722233
:10DE20008F2E852E2E125BB5EF64016014125BB548
:10DE3000EF700E125BB5EF64016010125BB5EF700E
:10DE40000AE52E9065B093FF12623E228E308F312C
:10DE50008C328D330531E5317002053014FF053306
:10DE6000E5337002053214FD12DADDAD33AC32AFAA
:10DE700031AE3012DADD228F31900A7CE531F025A7
:10DE8000E024C2F582E43482F583E493FF12698FC3
:10DE9000E53125E024C3F582E43482F583E493F58B
:10DEA000A5227D017F387E0012DC5DEF5403FF1256
:10DEB00068A17D017F397E0012DC5DEF5403FF1203
:10DEC000689AE4FF126893E4FF12688C22900A0DAE
:10DED000E04408F0900A0B7408F0E4900A13F0EFA5
:10DEE000600B900A0E7411F0E4900A14F0900A127C
:10DEF0007403F0900A09F022900AC6E0FE6F6018E1
:10DF0000EEF46014EFF0900AC1E0FF12E37CCDEF75
:10DF1000CDE4FB7F06120B20900AC6E0B4FF037429
:10DF2000F0F022E4FD7F24FE12DC5D900AC3EFF0E6
:10DF30007D017F217E0012DC5D900AC4EFF0E4FDDC
:10DF40007F21FE12DC5DEFF404900AC5F022BF01D0
:10DF500013900CFEE0FEED906AED93FCEE4C900CFD
:10DF6000FEF08012900CFEE0FEED906AED93F4FC62
:10DF7000EE5C900CFEF002B80012E68412F30DE4A1
:10DF8000900A0DF0900A0CF07F0812CCB1C2131267
:10DF90009DF27D397FAE7E0012D74E5005D213120E
:10DFA0009DF222900BE8E0B40505120BA4401D90F1
:10DFB0000A0CE04402F0D20812EF6612EFFDE4FD15
:10DFC0007F0112DF4E7D017F0112DF4E221264E0DD
:10DFD000900BB8E0B45603C38001D3921375463F4B
:10DFE000E4F547125C561266841264E0CDEFCD7FF3
:10DFF000047E00124FE42212F287500D900BBDE018
:10E00000FFC41313540330E013126558EF601090EF
:10E010000BBDE0FFC41313540330E003D38001C3EE
:10E0200022900D10EFF0125BB5EF64016014125BEB
:10E03000B5EF700E125BB5EF6401600E125BB5EFC9
:10E040007008900D10E0FF12E53122900D22EFF0E4
:10E05000125BB5EF64016014125BB5EF700E125BDA
:10E06000B5EF6401600E125BB5EF7008900D22E011
:10E07000FF12E55522AE05EEC3941F40079006B887
:10E08000EFF08015EFFD7C00AF067E00121BEB7DEC
:10E090001F121BFD9006B8EFF09006B8E0FF22E4D7
:10E0A000FF126A22E4FF126A1BE4FF126A14E4FF03
:10E0B000126A06E4FF1269FF7D2E7FAE7E0012D742
:10E0C0004EE433FF1269F8228F31E49006BBF01260
:10E0D000E89C500B9006BB740EF0E49009C4F0AFBE
:10E0E0003112EB83500A9006BBE0FDAF3112D41E13
:10E0F0002212DFA312F10112F2E3D20812F0557FCF
:10E100000712C03E7F6E7E011227D612EDA5E4FDF8
:10E11000FF128E0A7F0D124A7922900BE8E064010B
:10E120006007900BE9E0B40D19900B5DE0FF30E063
:10E1300011900B5CE014F0E07008EF54FEA3F012B5
:10E14000F1B8228F2C852C2CE52C906B5893FF1264
:10E1500067F7E52C906B5A93FF1267F0E4FF1267A4
:10E160009CE4FF1267E2E4FF0267BF8E458F461210
:10E1700027D6EF7F00FEEFC0E0EEC0E0E5462401C9
:10E18000FFE43545FE1227D6EFFDD0E0FED0E04D8E
:10E19000FF22744C2FF582E4340BF583EDF0787890
:10E1A000F67B788F507D017F4012454312626250AA
:10E1B00007900C61E04440F0228F3012EC56EFC023
:10E1C000E012EBFACEEFCED0E0FFC3EE9F04900654
:10E1D000B2F0AF3012D66E9006B2E02FF0E0FF2220
:10E1E0008F2C852C2C125BB5EF64016014125BB58B
:10E1F000EF700E125BB5EF6401600B125BB5EF7050
:10E2000005AF2C12449B228F2D78A6E6FF125FF4F7
:10E2100078A6E6FFE52DFD7C001256E078A6E6FF25
:10E220007D0812001678A6E6FF12587E227F027E35
:10E230000A120C105013900AC1E0FF6405600AEF47
:10E240006007A204920512B18AC20C7F027E0A12F4
:10E250000B5C228F3412EF5640012212E50D900B19
:10E2600087E534F0900B897401F0FB7A0B7981AF6C
:10E270003412B082120472D3228F317B78853150F0
:10E280007D027F40124E0E126262500A900C61E0D5
:10E290004440F07FFF2274782531F8E6FF22900A8F
:10E2A0007DE030E10D12EF7612BEC8900A7DE05499
:10E2B000FDF0900A77E030E003D38001C340031201
:10E2C000D3E122126550BF0103D38001C392131220
:10E2D000F29BEF7010900A7BE0540FFFBF0F03D347
:10E2E0008001C39213A21322E4FD7FDA7E0412DCC4
:10E2F0005D900A81EFF0E4FF12683FC20812E30D5F
:10E30000900BA0E030E405D20812E30D229006C085
:10E310007401F0900A7DE054FBF030080CE49006A4
:10E32000C0F0900A7DE04404F09006C0E0FF125770
:10E3300022228F307B007A00793012B2819006BAA7
:10E34000EFF06004E0B40E06AF3012E0C822900691
:10E35000BAE0FF12ED5522900A0BE024FE60111482
:10E36000601424FD601024057011E4FF1267B822C8
:10E370007F011267B8227F031267B8229006E6EF8A
:10E38000F0900B9DE030E203D38001C3400D900676
:10E39000E6E0D394004004E02406F09006E6E0FFB7
:10E3A00022900BE8E0FF12BF27900AC1EFF0900B1C
:10E3B0009DE030E108900ACBE0900AC1F0900ACDD0
:10E3C000E0900AC8F022E4F574C3EF94C4EE94021E
:10E3D0004017D3EF94A0EE9437500E900BBDE0445D
:10E3E00001F0C21B12A0BCD322C322900BBDE0FFE0
:10E3F000C413540730E0187FA07E3712E8B7900BA3
:10E40000BDE054DFF0900B897404F0900B88F0228B
:10E41000853636EF25E02DF5369060EE93FF1267D6
:10E4200095E5369060F293FF1267CDE5369060F681
:10E4300093FF0267DB900A08E0FF900BB8E0B45648
:10E4400003C38001D39213754664E4F547125C560A
:10E45000900A08EFF012E98A22900A02E0FF900B7E
:10E46000B8E0B45603C38001D39213754664E4F553
:10E4700047125C56900A02EFF012E9BE22900A039E
:10E48000E0FF900BB8E0B45603C38001D39213753C
:10E490004664E4F547125C56900A03EFF012E9D89F
:10E4A00022900A04E0FF900BB8E0B45603C3800149
:10E4B000D39213754664E4F547125C56900A04EF54
:10E4C000F012E9F222900A05E0FF900BB8E0B45692
:10E4D00003C38001D39213754664E4F547125C567A
:10E4E000900A05EFF012EA0C22900A10E0FF900B60
:10E4F000B8E0B45603C38001D39213754664E4F5C3
:10E5000047125C56900A10EFF012EA262278A6E62F
:10E51000FF125FF478A6E6FF7D287C001256E078B3
:10E52000A6E6FF7D0712001678A6E6FF12587ED3F6
:10E53000228F36125BB5EF64016014125BB5EF7089
:10E540000E125BB5EF6401600B125BB5EF7005AFA7
:10E5500036124C0B228F36125BB5EF640160141239
:10E560005BB5EF700E125BB5EF6401600B125BB52B
:10E57000EF7005AF36124BC82212F29B9006BFEF28
:10E58000F064046011E0B401109009BEE020E103E2
:10E59000D38001C34003D38001C322900A78E0FFF7
:10E5A000900BB8E0B45603D38001C3920CD20D7B1C
:10E5B00004E4FD1246C612E70312F0F42230191EDD
:10E5C000C3900C99E09430900C98E0942A500C90F1
:10E5D0000B87E0942850041289912212B465227F9F
:10E5E0008312CEF4900001121B68FFEFC0E07F831E
:10E5F0007E0012CEF4121B4FFDD0E0FF12D41E227B
:10E600007F8312CEF4900001121B68FFEFC0E07F01
:10E61000837E0012CEF4121B4FFDD0E0FF12D045D6
:10E6200022E49009B0F09009BEF0A3F09009C4F084
:10E63000900BBDE04420F0E4FF126981E49009C131
:10E64000F02212E89C501B120C0ABF0915D20C7F55
:10E65000827E00120B5CD20C7F827E05120B5C1254
:10E660000BE022900BBDE0FD1313543F30E0057E1C
:10E67000027F6022EDC31330E0057E027F1E227E02
:10E68000027F6E227454E4900D19F0900D0F7412F5
:10E69000F0900D0E7410F0900D177401F0E4FF125D
:10E6A000BDA502F340900BBCE060197F027E0A1208
:10E6B0000C105007A204920512A2DBC20C7F027E4E
:10E6C0000A120B5C2290044FE02405F582E4340525
:10E6D000F583E0FF9006B3F012C4D0120BAAE490C9
:10E6E0000AABF0227F07126A6112A9CF9009B5E048
:10E6F000B40408E4FD7F04128E0A22E4FD7F0112B7
:10E700008E0A228F3412F29BEF600412F21422E57B
:10E7100034C394054003E4F534AF3412F00F12EF24
:10E72000DF228E2C8F2DC21B900BBDE04402F0D255
:10E730001C7F0112673A757404AF2DAE2C12E8B736
:10E740002212E79C900BBEEFF012F33F900BBDE05E
:10E7500054FBF07F02126A7D7FC47E0212E8B7226A
:10E760007D607F0E125A147D14E4FF1244F0900A6B
:10E770007FEFF07D0E120016E4900A6EF022900AF0
:10E7800006EFF0D3946440037432F0900A06E090F0
:10E7900082CA93FF9006C9F012E04B229006AF7434
:10E7A00003F0900B9BE030E70B9006AF7401F02074
:10E7B0002E02E4F09006AFE0FF22900B9CE030E4E4
:10E7C000097D207F0312EE298005E4FF1269F19094
:10E7D0000A76E054FDF02212E8D212E6219009B642
:10E7E00074FFF09009AFF07FBD7E071227D6900925
:10E7F000B5EFF02230080DD20912ED18900A0CE0A6
:10E800004404F022C20912ED18900A0CE054FBF007
:10E8100022E4FD7F3CFE12DC5DEF5403FF1266B57F
:10E820007D017F227E0012DC5D1266AE22900A70AE
:10E83000E0B401047F0180027F00EF640160099071
:10E840000A6E7401F01290E122CBEDCBEF6404600C
:10E8500003EF7010EF70047D0180027D007F857EE4
:10E860000312BFE22212F287500475740222E5738C
:10E87000D394044004757401227F0412C87C05738C
:10E8800022E4FF12585F7F0112696C7D017F257EB3
:10E890000012DC5DEF540FFF12696522900B9BE0C4
:10E8A00030E612900BE8E064016007900BE9E0B4F9
:10E8B0000D03D38001C3228E358F3612D5885010B8
:10E8C000900BBDE04401F0AF36AE3512A0BCD322B0
:10E8D000C32212EFD0E4900B89F07D5F7F07125ABC
:10E8E000147D287F801244F078A6EFF622C202122F
:10E8F0005BB5EF6401600E125BB5EF7008900CF62B
:10E90000E024FF9202A20222E4FF12676BE4FF12EE
:10E9100067647D287FAE7E0012D74EE433FF126716
:10E9200048227F0112684DE4FF126854E4FD7F2500
:10E93000FE12DC5DEF540FFF126846227D047FAEAD
:10E940007E0012D74EE433FF1268EE7F011268E7B3
:10E950007F031268E022900B877401F0900BBF04D4
:10E96000F0A374C4F0900C987422F0A3742EF022DB
:10E97000E49006FDF0BF040C7F0E12D785EF2463F0
:10E980009006FDF09006FDE0FF22900A08EFF0D31C
:10E99000946440037432F0900A08E09082CA93FFB6
:10E9A00012EEB522900A07EFF0D39464400374325C
:10E9B000F0900A07E09082CA93FF12E02122900AA9
:10E9C00002EFF0D3946440037432F0900A02E090B6
:10E9D00082CA93FF12496322900A03EFF0D3946432
:10E9E00040037432F0900A03E09082CA93FF124908
:10E9F0001C22900A04EFF0D3946440037432F09028
:10EA00000A04E09082CA93FF1248D522900A05EFCB
:10EA1000F0D3946440037432F0900A05E09082CA07
:10EA200093FF12488E22900A10EFF0D394644003B3
:10EA30007432F0900A10E09082CA93FF1248472285
:10EA40007D267FAE7E0012D74EE433FF126A4CE47F
:10EA5000FF126A45E4FF126A3E22900B9CE030E40C
:10EA6000047F0180027F00BF0109E4900B0EF0A338
:10EA700074FFF022900A78E0B40111C3900B82E099
:10EA800094E4900B81E0940650028001C322900B25
:10EA9000B7E0FFD201900BBBE07009EF60066403A2
:10EAA0006002C201A20122900A0BE0FF6408600F1D
:10EAB000EF6409600A12EA745003D2A322C2A322AF
:10EAC0007FD27E041227D68F2C7F7B1251C8787B91
:10EAD000E6D3952C500122C3228F2C852C2C125B5F
:10EAE000B5EF64016006125BB5EF6005AF2C125EF6
:10EAF0005422E4FF1267E9125BB5EF64016006126D
:10EB00005BB5EF6005E4FF12635F22CDEFCD900AA5
:10EB100071EDF0D3946440037432F0E4FB7F14127F
:10EB20000B1A22CDEFCD900A72EDF0D3946440031E
:10EB30007432F0E4FB7F15120B1A22CDEFCD900A50
:10EB400073EDF0D3946440037432F0E4FB7F16124B
:10EB50000B1A22CDEFCD900A74EDF0D394644003EC
:10EB60007432F0E4FB7F17120B1A227FEC7E001246
:10EB700027D69006ADEFF012EF859006ADEFF012BC
:10EB80006B7E228F3212EC56E532C39F400B12EBA4
:10EB9000FAE532D39F50028001C322900A09E02493
:10EBA000FC600824FB60042407700412EDCD2212DF
:10EBB000EFA32212E89C5012900905E0FF12ED41EC
:10EBC0007D0E12D045900B5EEFF022CBEDCBCDEF5A
:10EBD000CD7FC21245921262625007900C61E044F0
:10EBE00002F022900B9CE030E4087D207F0312EEBF
:10EBF0009322900A76E04402F0229006BC7463F0FF
:10EC000012E89C50069006BC7428F09006BCE0FF09
:10EC100022900A0FE0C36480948A500BE004F090C5
:10EC20000A01E0FF12924322900A0FE0D36480941D
:10EC300076400BE014F0900A01E0FF12924322307C
:10EC40000310900B9DE030E305C20812AD4012D0D6
:10EC5000CD2212EF0622E49006EFF012E89C500657
:10EC60009006EF7401F09006EFE0FF22900BB8E001
:10EC7000B4560412EC1122900BB8E0B4550312EC18
:10EC80002822900A0CE06410FFF0900A097402F048
:10EC9000EF30E4037401F022E4900AC2F0900AC954
:10ECA000F0A3F0900ACCF012DF2312CF3B2278A71A
:10ECB000E6B4010F7F011299AC12F307EF600478FC
:10ECC000A776FA22E4FF126787E4FF1267797F02D2
:10ECD0001267727F0112678E227F0112690A7F011B
:10ECE000126903E4FF1268FCE4FF126B8422E4FF64
:10ECF00012699DE4FF126996E4FF12698FE4FF1226
:10ED0000697A22900CECE014600A14600714700712
:10ED100012E5BD2212EE3B22AF07A209923E303E21
:10ED200007900D17E0FF8002E4FF02EFEE9006BEB1
:10ED3000ECF0A3EDF07B017A0679BE7D0212D5C31B
:10ED4000229006ECEFF07B017A0679EC12B281900A
:10ED500006ECE0FF228F317F0312CEF49000011207
:10ED60001B68FFAD3112D41E22EFC39429500DEF62
:10ED70002456FFE43403FE7DCA124FE422900B9C1C
:10ED8000E030E4047F0180027F00BF010312EA5AF1
:10ED9000227F217E031227D6900CEDEFF0C3940C56
:10EDA0004002E4F022900B87EFF012D3659006BF8B
:10EDB000EEF0A3EFF012CC6722900BE8E0B401096B
:10EDC00012F2E37F0712C03E2212F2E922900A0CEF
:10EDD000E020E606D20812AD4022C20812AD402261
:10EDE000900A0CE020E206D20812E7F422C20812D0
:10EDF000E7F42212F08C12E7BA12F0A612F0C0E487
:10EE0000FF12B7EA22A203920812EF66A203E433CC
:10EE1000FF7D0112DF4E22CDEFCD7F227E0312DC7B
:10EE20005DBF0103D38001C3228F368D3712D7F324
:10EE3000E537F45FFDAF3612E1922230180412DBA1
:10EE40003F221289917F027E05120BDA22E4F573CC
:10EE500012F2875004757402227F1012C87C22902F
:10EE60000D07EFF012F07112F32F12F06312F32B73
:10EE70002212D8A412EAA712E357900A7DE04402B6
:10EE8000F02212F2A1CDEFCD7F227E0312DC5D12C3
:10EE9000E703228F368D3712D7F3E5374FFDAF36B4
:10EEA00012E19222EF60047D0080027D01E4FB7F8D
:10EEB00007120B2022900D1CEFF012F07112F32FAD
:10EEC00012F06302F32BE4FF1266BCE4FF1266CA81
:10EED0007F011265F122E4FF1268CBE4FF1268C4DF
:10EEE000E4FF1268B6227F0112660D7F01126606EA
:10EEF0007F01126A682212EBFAEFD3946340047F19
:10EF00000380027F0222900A0CE0547FF054BFF08D
:10EF1000E4FF12BDA522CDEFCD900A78E0FB7F2261
:10EF20007E0312BFE22212CC67900B5B7401F0905B
:10EF30000B87F0D21922E4FF1268B67F0112676BCB
:10EF4000E4FF1268A822E4FF1268B6E4FF12676BC0
:10EF50007F011268A822EFC394004008EFD39463A6
:10EF600050028001C322A208E433900D16F024FF62
:10EF7000920912D8002212AA6412B20712E57992FD
:10EF80000812C96C22EFD3946440027F64EF908230
:10EF90005D93FF229009B0E0600812CA56E4900920
:10EFA000B0F022900A0CE020E70412D0CD2212EF3C
:10EFB0000622900B9DE030E30412EB9B2212EFA39C
:10EFC00022C21CE4FF12673A7FC47E0212E3C6220B
:10EFD000900BBDE054FEF07D5F7F02125A142212A6
:10EFE000C62D900B81E0FEA3E0FF12E8B722900C43
:10EFF000F4EFF0EF906AE793FF12621A22C2A022A8
:10F00000A209E433900D12F024FF920A02C6849004
:10F010000A78EFF07F0112687712EF7622900B8763
:10F02000E0C394634003D38001C322E49009BFF09E
:10F030009009B004F01285A722CBEDCBCDEFCD7FA8
:10F04000227E0312BFE222900CEDEFF0FD7F217EC5
:10F0500003124FE422A20892137D187FAE7E0012A5
:10F06000C7D822900D07E0FF900D1CE0FD12E0755F
:10F0700022900D07E0FF900D1CE0FD12DC2E227F98
:10F08000011269D5900A76E04404F022E4FF126987
:10F09000D5900A76E054FBF0227F011269C0900AF5
:10F0A00076E04408F022E4FF1269C0900A76E0544A
:10F0B000F7F0227F011269C7900A76E04410F0222F
:10F0C000E4FF1269C7900A76E054EFF0227D637F77
:10F0D00008125A14E4900CECF022900CEC7405F039
:10F0E00090097C7401F022900CEC7403F0900B8773
:10F0F000E004F022900A78E0906B0F93FF12C03E7C
:10F10000227FC07E011227D6900B5FEFF0228F2C5A
:10F11000E4FF12BA11AF2C12C20522900B9DE03011
:10F12000E105EF24FF92C92275FE554387108FFF3A
:10F1300075FE0A22900BB874FFF0A37405F0227FCD
:10F14000011269507F01126A7622CDEFCDE4FB7F78
:10F1500006120B1A22E4FF126725E4FF12671E2233
:10F160007F01126A37E4FF126A302212F197900A87
:10F170007DE054FEF022900A0DE04420F012F333BB
:10F1800022900A0DE054DFF012F33622900A0DE0CF
:10F190004404F012DFA32212DFA3900A0DE054F71B
:10F1A000F0227F02126A5AE4FF126A532275740435
:10F1B00012F2875002D21D22E4FF1262837F0112F5
:10F1C000628322C203A23F9203C23FA20322E490C1
:10F1D0000C60F0A3F0A3F022E4900A80F0900A798A
:10F1E000F0221287CB128B2812CDD622900A0DE086
:10F1F00020E402D2A0227D187FAE7E0012D74E22DC
:10F20000129D2212AE5D12C25F22E4FF1299AC7809
:10F21000A776FA227F0812687712EF7622CDEFCD1B
:10F220007F0712E19222CDEFCD7F0912E192229069
:10F230000CEDE0FF120BEC2212BF27900ACBEFF08F
:10F2400022900BBFE0FEA3E0FF229009C4E05480AF
:10F25000F022900A0DE054FBF022900BBDE054FE2A
:10F26000F022900D23EFF002E1437FAC1262C50261
:10F27000F31212F134124A3522900CEC7404F0228D
:10F28000900AC6740AF022126550EF24FF22900DF6
:10F290000EE0A2E622E4900CECF0229009B8E0FF28
:10F2A000229009B9E0FF227F07120BE6227F0812A5
:10F2B0000BE6227F09120BE6227F0A120BE6227F61
:10F2C0000B120BE6227F0C120BE6227F0D120BE6CF
:10F2D000227F0E120BE6227F0F120BE622900B0DFF
:10F2E000EFF022D20812C41F22C20812C41F2290BB
:10F2F0000D0EE0FF22900D17EFF022900D0EE0337F
:10F3000022900CF7E0FF22900CEFE0FF22E4FF02D6
:10F31000E1E07FA70262C512EE822212F3172212E9
:10F32000ED9122120B7A221265A02212444622127B
:10F3300043F122C28422D2842222222222222222A9
:10F3400022FFFFFFFFFFFFFFFFFFFFFFFFFFFFFFAA
:10F35000FFFFFFFFFFFFFFFFFFFFFFFFFFFFFFFFBD
:10F36000FFFFFFFFFFFFFFFFFFFFFFFFFFFFFFFFAD
:10F37000FFFFFFFFFFFFFFFFFFFFFFFFFFFFFFFF9D
:10F38000FFFFFFFFFFFFFFFFFFFFFFFFFFFFFFFF8D
:020000040001F9
:100000004D61696E005069637475726500536F7558
:100010006E6400466561747572657300496E737431
:10002000616C6C004D6F6465005043004844004DA6
:100030006F7265202E2E2E004272696768746E659D
:10004000737300436F6C6F757200436F6E747261EF
:1000500073740053686172706E65737300436F6EE2
:1000600074726173742B00436F6C6F7572205465EA
:100070006D7000436F6F6C005761726D004E6F7250
:100080006D616C004175746F5069632E426F6F73C0
:1000900074657200547265626C650042617373002E
:1000A00042616C616E63650044656C746120566FDB
:1000B0006C756D650041564C0053415000496E63AC
:1000C000722E537572726F756E6400446F6C627934
:1000D000205669727475616C0054696D65720043D5
:1000E00068696C64204C6F636B00343A3300457868
:1000F00070616E6420343A3300436F6D70726573C3
:10010000732031363A39005A6F6F6D2031343A39E5
:10011000005A6F6F6D2031363A3900537562746939
:10012000746C65205A6F6F6D00537570657220573F
:10013000696465005769646573637265656E00463E
:10014000756C6C73637265656E00504950004C5459
:1001500049004C54492044454D4F004C616E677531
:1001600061676500456E676C69736800436F756E03
:10017000747279004175746F2053746F7265004D0D
:10018000616E75616C2053746F7265004575726F96
:100190007065004672616E636500554B005765736C
:1001A00074204575726F70650045617374204575E4
:1001B000726F7065004E616D6500536F7274005010
:1001C0006C6561736520576169742E2E2E00457130
:1001D00075616C697A65720031323020485A003599
:1001E000303020485A003135303020485A00352010
:1001F0004B485A003130204B485A0054696D650015
:1002000053746172742054696D650053746F70206B
:1002100054696D6500536C656570004F6E636500D1
:100220004461696C7900416374697661746500505A
:10023000726F6772616D00545600464D20526164C2
:10024000696F0053746F72653F0053746F72656419
:100250000053656C6563740053797374656D005366
:1002600065617263680050726F6772616D204E6FD6
:100270002E0046696E652054756E65004672657184
:1002800075656E63790053637265656E20536176A0
:100290006572004D6F6E6F0053746572656F004438
:1002A00075616C2049004475616C204949004E69B4
:1002B00063616D204D6F6E6F004E6963616D2053F9
:1002C000746572656F004E6963616D204475616C81
:1002D0002049004E6963616D204475616C20494975
:1002E000005370617469616C0052696368004E610B
:1002F000747572616C00536F667400566F69636544
:10030000004D757369630054686561747265004DD2
:10031000756C74696D6564696100506572736F6EA8
:10032000616C004372797374616C20436C65617217
:1003300000436C6173736963616C004A617A7A008F
:10034000506F7000526F636B00436C6561722041A7
:100350006C6C004C6F636B656400436C6561726527
:100360006400436C656172203F00566F6C756D656B
:1003700000D20053746F7265004F6E004F666600C6
:10038000476F6F64627965005456205377697463D0
:1003900068696E67204F6666004368616E67696EC4
:1003A0006720546F00696E0053656300486F746581
:1003B0006C20536574757000486F74656C204D6FC8
:1003C0006465004F6E204368616E6E656C00436823
:1003D000616E6E656C20426C616E6B6564004B658E
:1003E00079626F617264204C6F636B004D6178209D
:1003F000566F6C756D65004F6E20566F6C756D6530
:100400000041757820566F6C756D65004F53442020
:10041000446973706C6179004D6F6E69746F7220FE
:100420004F75740049434F4E4E204D6F6465004137
:10043000637469766520436F6E74726F6C004469F3
:1004400073706C6179204F6E00446973706C6179D0
:1004500020416C6C004C696768742053656E736F43
:1004600072004D656469756D004175746F00004ED2
:100470005453430050414C00534543414D004247C3
:10048000004900444B004D004C4C00455854004579
:1004900058543100455854320041560045583100F7
:1004A00045583200000041004200434800440044E7
:1004B0004B0045004600464900474200475200496C
:1004C000524C004C004E004E4C0050005300435A1A
:1004D000004800485200504C00524F005255530003
:1004E000534B00534C4F005452005955002E2E2EA2
:1004F00000456E676C6973680044616E736B004EF3
:10050000656465726C616E64730053756F6D69002C
:100510004672616EE961697300446575747363685E
:100520000045BABAB676B8B9B0004974616C696171
:100530006E6F004E6F72736B00506F7274756775DB
:10054000FB7300457370610A6F6C005376656E73C0
:100550006B61004872766174736B69000165736B3F
:1005600079004D616779617200506F6C736B69003F
:10057000526F6D616E6100507963BAB8B900536C07
:100580006F76656E736B7D00536C6F76656E736B03
:10059000690054FE726B0D65005365727669636580
:1005A0000000436C656172004C6F616465640053C8
:1005B000414D0053444D0043534D00436F6D7061F6
:1005C0006972204D6F646500434F444553004F509E
:1005D000005033432D31004E4F542054554E454466
:1005E00000434F00425200485500425300554E4BC5
:1005F0004E4F574E00455252004F7074696F6E73E4
:100600000054756E657200576869746520546F6E8A
:10061000650047656F6D6574727900417564696F37
:10062000004E564D20456469746F72005343204E4E
:10063000564D20456469746F720054657374205080
:1006400061747465726E004F5031004F5032004F2C
:100650005033004F5034004F5035004F5036004F4C
:100660005037004F5038004946504C4C00414743EA
:1006700000434C00334420434F4D46494C544552AF
:1006800000414743204C27004E6F726D616C205231
:100690006564004E6F726D616C20477265656E0017
:1006A0004E6F726D616C20426C75650044656C74B0
:1006B0006120436F6F6C205265640044656C746107
:1006C00020436F6F6C20477265656E0044656C74E3
:1006D0006120436F6F6C20426C75650044656C74DB
:1006E00061205761726D205265640044656C7461CD
:1006F000205761726D20477265656E0044656C74A9
:1007000061205761726D20426C756500486F726997
:100710007A6F6E74616C00566572746963616C0007
:100720004850004842004853480045575700455735
:10073000500045575400554350004C435000565309
:100740004C0056414D0056534300565348005653F3
:100750000053424C0041462D4D004132540051534C
:100760005300464D490049463100494632004E6922
:1007700063616D20416C69676E6D656E7400444302
:10078000584F20416C69676E6D656E740044424538
:10079000004144520056414C0053746172743F0052
:1007A000496E2070726F677265737300446F6E6577
:1007B000004661696C6564000080008005800D80E2
:1007C00013801C80248029802C802F8038804380D7
:1007D0004A8053805D806780738078807D808480CC
:1007E00094809B80A080A880B580B980BD80CB809C
:1007F000D980DF80EA80EE80F981078111811B8139
:10080000298134813F814A814E8152815B8164819B
:100810006C8174817F818C8193819A819D81A98172
:10082000B581BA81BF81CE81D881DF81E681EE8139
:10083000F481FB8200820B8215821B822082268239
:100840002F8237823A8243824A82518258825F8263
:10085000668272827C828682938298829F82A6823E
:10086000AE82B982C682D382E182E982EE82F682CA
:10087000FB83018307830F831A83238331833B83A5
:1008800040834483498353835A8362836A83718399
:10089000738379837C83808388839983A583A883EA
:1008A000AC83B883C383CE83DE83EC83F784018477
:1008B0000C84188424842F843E8449845584628463
:1008C00069846E846F84748478847E848184838454
:1008D000868488848B848F84948499849C84A08467
:1008E000A484A684A884AA84AD84AF84B284B4848A
:1008F000B684B984BC848184BF84C384C584C7841E
:10090000CA84CC84CE84D184D384D684D984DC8434
:10091000E084E384E784EA84ED84F184F984FF854C
:100920000A851085198521852A8533853985438572
:100930004B8553855C8562856985708577857E8565
:10094000888592859985A185A285A885AF85B3857F
:10095000B785BB85C885CE85D185D785E185E485FA
:10096000E785EA85ED85F585F98601860786128695
:100970001B8621862C863A8647864B864F86538671
:1009800057865B865F86638667866D86718674860A
:10099000818688869386A086AC86BB86CC86DC86DC
:1009A000EB86FC870C8717872087238726872A8773
:1009B0002E87328736873A873E87428746874A871F
:1009C0004E87518755875A875E87628766876A8711
:1009D0006E877E878D87918795879987A087AC875B
:1009E000B187B8936B47466567686C6D110F102629
:1009F000171285868788898A8B8C4F5051525354A1
:100A0000555618204C200020522020000C520C5823
:100A10000C5E0C640C6A0C700C760C7C0C820C88DE
:100A20000C8E0C940C9A0CA00CA60CAC0CB20CB84E
:100A30000CBE0CC40CCA0000000007FF7FFF0100C1
:100A40004081058068F70018000000180000031FAF
:100A500055050000C0B700000000000150810001F2
:100A6000508100015081000150810001000000010F
:100A70000000000100000000C0B700000214000DDB
:100A80004E00001710010D4E00002405010D4E0010
:100A90000B002902905B0101020C000D4E01011BAD
:100AA0000C010D4E02020216000D4E02021D0A013B
:100AB0000D4E03030110000D4E0606040C000D4EF2
:100AC0000606022502905B01020222000D4E0A0A70
:100AD000022602905B0B0B022502905B00002403B0
:100AE000010D4E020A021A000D4E0309061D029066
:100AF0005B01090512000D4E0109190F000D4E0092
:100B0000000220000D4E00000227000D4E030402DB
:100B100022000D4E03090227000D4E0000022100A5
:100B20000D4E01010218000D4E0606022502905BD3
:100B300002020207000D4E0402010F0000000F0028
:100B40000F0F0B00000F0B05000F0F000F0F0F0012
:100B500000000F0000000F000F0F0000000F0F003B
:100B60000F000F0F0F0F0F4D487A00000602050906
:100B7000060F000602050906520301090705030DC9
:100B8000010203060504FF0D0006020500000D002A
:100B900006020509090F0D0D0D0F520F0D840D846E
:100BA0000D8A0D840D90010D28010B5E8D8E8F90A6
:100BB000930807090000020C02070112ED8E92044F
:100BC000900BB8E09006ADF0300403028E5AD204C8
:100BD00030272390044FE075F003A42455F582E4F8
:100BE0003404F583121F0E900003121C93AAF0F92F
:100BF000121F73028E5A9006ADE0121F208D050F52
:100C00008C24108C24118C1C208C1C218C1C388C66
:100C1000AE508CAE518C2C5200008D1712E86B92A6
:100C200004028E5A12F0D09204028E5A900BBCE04D
:100C30006065900526E0705F90044EE06401601FDF
:100C4000120CEE90044EE0B40B10900AE0E07047F6
:100C5000D207FD7F0112D518803D12DCA580381225
:100C6000E0671209E25030900CA1E0B40110D20705
:100C7000E4FD7F0C12D518E490094CF08019900C1B
:100C8000A2E0B40112D20C7FA17E1712BFC1D20C18
:100C90007FA17E0B12BFC1900526E0FF64016008B2
:100CA000EF64026003028E5A12EEE7028E5A12EBD4
:100CB00051EF64347030900BBCE0700C900BBAE0D4
:100CC000D394055003028E5A9009E6E07013900603
:100CD000ADE013920512A1E89009E67402F0028ECD
:100CE0005AC204028E5A900BBCE0700C900BBAE012
:100CF000D394055003028E5A9006ADE0139205126C
:100D0000A1E8028E5A900BBCE07003028E5A120CBE
:100D1000F412E067028E5A900BB9E0FF640260089B
:100D2000EF64016003028E2FEF64027049900BBCE8
:100D3000E0FE7009900BBAE0D39405401B90044F7D
:100D4000E075F003A42455F582E43404F583121F02
:100D50000E121B4F6401702FEE601B90044FE07564
:100D6000F003A42455F582E43404F583121F0E1217
:100D70001B4F64016011EF64016003028E5A900BF7
:100D8000BCE07003028E5AEFB4012990044FE07565
:100D9000F003A42455F582E43404F583121F0E12E7
:100DA0001B4FFF64046005EF64077069900BB9E0A6
:100DB00064017061900BBCE0FF6002C21E301E1225
:100DC000EF6003028E5A900BBAE0D3940540030201
:100DD0008E5A90044FE075F003A42455F582E43454
:100DE00004F583121F0E121B4FB40502D21E12E32C
:100DF00085506790044FE075F003A42455F582E414
:100E00003404F583121F0E900003121C93AAF0F90C
:100E1000121F738045900BB9E06401703D900BE8A0
:100E2000E0640460359006ADE0FF12DAB1802B90EB
:100E30000BB8E06422702112E79CBF0717120CFA6E
:100E4000EFD39463400E900BE8E07008120D00128F
:100E5000DCA58006C2048002C20412D5C5A2042209
:100E6000E49006AEF0900526E0707A12093AEF6041
:100E70002812093AEF640E602090044FE075F003E9
:100E8000A42455F582E43404F583121F0E121B4F7F
:100E9000B40906120934120CD012093490052CE062
:100EA000FEC3EF9E900527F0900BD6E030E01012C5
:100EB0000CD6500BD20C7F837E0012BFC18017D29C
:100EC0000C7F027E0012BFC1120CD65009C20C7FEB
:100ED000027E0512BFC1E490052AF0900528F0902B
:100EE000052604F022900526E0B4010B900BB8E033
:100EF000B4550412EEE722900526E0B40603D38031
:100F000001C3500302905A90044FE075F003A424EB
:100F100055F582E43404F583121F0E121B4FB408FA
:100F2000089006AE7405F080069006AE7402F0904C
:100F30000BB9E06402600302905A90052AE0FF902A
:100F40000BB8E0B45603D38001C3920CC20D7BFFF3
:100F5000E4FD1246C690052AEFF0E4A3F0EFD39427
:100F600000406B9006AEE0FF90052AE0FED39F5054
:100F70005D90044FE075F003A42455F582E4340439
:100F8000F583121F0E121B4F6408703590052674EE
:100F900002F0900528E0FF900527E0C39F75F0035D
:100FA000A424D5F582E43404F583121F0EEE7E00EE
:100FB00024FFF582EE34FFF583121B68FF12E52E45
:100FC000229005267403F090052A7401F02253C77D
:100FD000BF9005267401F0E490052AF090044FE0DC
:100FE00075F003A42455F582E43404F583121F0E32
:100FF000121B4F64087063900528E0FF900527E0FE
:10100000C39F75F003A424D5F582E43404F583125C
:101010001F0E7E0A7FF0124C4E120CD65008120999
:1010200034120CDC8015120934EFC0E012093ACDFD
:10103000EFCDD0E0FF120940120CDC900BD6E0306F
:10104000E00F120CD6500AD20C7F837E0012BFC173
:1010500022D20C7F027E0012BFC122900BF0E0FE74
:10106000A3E08EF0121F46910B0001911600029131
:101070002C00039121000491420101914D02019243
:101080000803019158050291630701916E080191CF
:10109000790A0191840A02918F0A03919A0A0491B4
:1010A000A50A0691B00A0792290A0992290A0A920A
:1010B000290A0B92290A0C92290A0D92290A0E92EA
:1010C000290A0F91BB0B0191C60C0191D10C029121
:1010D000DC0C0391E70D0191F20E0191FD0F0292DC
:1010E000131601921E1701913718029234190392B8
:1010F0003F19049229190592291906922919079274
:101100002919089229190900009249900BF274ECF0
:10111000F0A374FFF022900BF274DDF0A374F6F0EC
:1011200022900BF274DCF0A37460F022900BF27446
:10113000EAF0A37448F022900BF274F2F0A374DC8E
:10114000F022900BF274F1F0A374FBF022900BF2FA
:1011500074CFF0A37479F022900BF27419F0A37499
:101160008AF022900BF27419F0A37490F022900B85
:10117000F274F2F0A37404F022900BF274F2F0A374
:10118000740DF022900BF274F0F0A374ECF0229046
:101190000BF274ECF0A37430F022900BF274F2F0C6
:1011A000A37416F022900BF274F2F0A374DEF02216
:1011B000900BF274F2F0A374DFF022900BF274192A
:1011C000F0A37496F022900BF274F2F0A3741FF067
:1011D00022900BF274CDF0A374D7F022900BF2742E
:1011E000F2F0A37428F022900BF274F2F0A374D200
:1011F000F022900BF27419F0A37484F022900BF299
:1012000074F2F0A374E0F022900BF2740DF0A3746A
:1012100054F022900BF27419F0A3749CF022900BFE
:10122000F27419F0A374A2F022900BF274CCF0A324
:101230007421F022900BF27419F0A374A8F022909C
:101240000BF274F2F0A37431F022900BB7E0700847
:101250001209825003029429900BE9E0FF640470A4
:1012600003029429EF64057003029429120CD650EE
:1012700003029429900BB9E06401601B900BB8E065
:10128000FF640F6012EF642E600DEF64526008EF90
:10129000640D6003029426900914E0C39407400390
:1012A00002937DE49006ACF09006ACE0FFC3940797
:1012B0005048900914E0FEEF75F007A4246BF58206
:1012C000E4348BF583E5822EF582E43583F583E4FF
:1012D00093FE900BB8E0FDEE6D6017900915E0FEEF
:1012E0007401C8EFC8088002C333D8FCF45E9009CB
:1012F00015F09006ACE004F080AE900915E0FF54C4
:101300007F601A900914E004F0EF30E208900916AB
:101310007414F0800B900916740CF0800312F14ADB
:10132000E49006ACF09006ACE0FFC39407504E90FA
:101330000914E0FEEF75F007A4246BF582E4348B0A
:10134000F583E5822EF582E43583F583E493B4FFDB
:101350002474017E00C8EFC8088005C333CE33CEA5
:10136000D8F9FF900915E0FDE4EF5D6008900914DD
:101370007407F080089006ACE004F080A89009148F
:10138000E064076003029429900BE8E0B4040D9038
:101390000915E0547F64406003029429900915E028
:1013A000540F600312E5AC900915E0547F121F2022
:1013B00093C90193D60293F00493E30893FA10942F
:1013C0001220941A40000094221209E25003120DD8
:1013D000BA120DC0804C1209E25003120DBA120D60
:1013E000C6803F1209E25003120DBA120DCC8032B2
:1013F0001209E2402D120DD28028900BAAE0D3945E
:1014000000401F120DD87F01120988E4900BA9F04B
:10141000801012098E120DDE8008E4FBFD7F181289
:101420000B1A12F14A2212F14A228F309006B2743E
:10143000E0F0A37405F0C20890044DE02530FF9061
:101440000454E0FEC3EF9EFF7D0212F1AB9004490D
:10145000E030E51190044FE065306009900BA5E0A5
:10146000FF12F1A022900452E0FFE530C39F400339
:1014700002951790044FE065307014900449E030F5
:10148000E4069006B274D3F0900449E01392083059
:10149000080C7D057F0712F24312E417800912F24F
:1014A00078900BA27403F09006B2E0FF12EBC17FBC
:1014B0002012EBC19006B3E0900BA4F0E53075F07C
:1014C00003A42455F582E43404F583121F0E900022
:1014D00002121B68FF12F25C90044FE06530703717
:1014E000E53075F003A42455F582E43404F5831245
:1014F0001F0E121B4F9006B1F06405600AE0FF64F6
:10150000086004EFB40910900BA4E0FFC374149FAB
:10151000FF12EE2C12F29A90044FE075F003A4240F
:1015200055F582E43404F583121F0E121B4F24F884
:10153000600D14600A1470030295E92405705F9031
:101540000BA4E0FFC374169FFF12EE2C90044FE033
:101550006530700312F278900454E0FFC3E5309FC9
:101560009006B1F09006B37416F0900BA4F09004BE
:101570004FE075F003A42455F582E43404F583129A
:101580001F0E121B4FB4050D90044DE0FFC3740AEB
:101590009F900529F09006B1E0FF12D0AA22900496
:1015A0004FE065306007900449E030E33690045224
:1015B000E0FFE530C39F5007AF3012B7778024902B
:1015C000044EE0B4080A3043079087F8E020E7F9BA
:1015D00090044DE02530FF900454E0FEC3EF9EFFE1
:1015E00012F1A012EEAB12F0DE22900452E0FF9056
:1015F000044FE0C39F4003EF14F0900C6EE0448072
:10160000F0E4900C6DF0A3E0548FF012B9989004C0
:101610004FE0FF7B017A04795412E709900527E037
:10162000FF7B017A05792812E70912EE8390044FB7
:10163000E0FF75F003A42455F582E43404F5831229
:101640001F0E121B4F24F8700302971B1470030225
:10165000971B24046003029732900449E020E6328D
:10166000C21F90044EE09006B0F0EF75F003A42482
:1016700055F582E43404F583121F0E900001121B0D
:101680006890044EF012DA1D9006B0E090044EF01F
:101690008005E4900453F0900453E0FF9006AFF00F
:1016A00090044DE0FEC3740A9EFEEFD39E40207F5F
:1016B0000812C1EF90044DE0FFC374099F75F00359
:1016C000A424D5F582E43404F583121F17806390B7
:1016D000044DE0FFC3740A9FFF9006AFE0C39F5024
:1016E0005190044DE0FFC3740A9FFF9006AFE0C322
:1016F0009F503F3040047F0080027F9312C1EF90E3
:1017000006AFE075F003A424D5F582E43404F58334
:10171000121F179006AFE004F080C6900526E0FF88
:10172000600864016004EFB4030890044FE0FF1206
:10173000B05A120D24502C900454E09006AFF09053
:10174000044DE0FFC3740A9FFF900454E02FFE9005
:1017500006AFE0FFC39E500B12942A9006AFE00440
:10176000F080DC120D244012900CECE0B4050890DF
:10177000097CE064046003120D2A90044EE090049A
:1017800050F090044FE0900451F0C2402212E02E3D
:10179000500E90044AE0FEA3E054FD4420FF800870
:1017A00090044AE0FEA3E0FF12EE6E7F0112F29475
:1017B000E49006B2F07BFF7A577901900A71E0F568
:1017C00035E4FF12F1169006B2E0FFE4FD12EFC01F
:1017D0009006B2E004F0E0FF7BFF7A577906900AAA
:1017E00072E0F53512F1169006B2E0FF7D0112EFBE
:1017F000C09006B2E004F0E0FF7BFF7A57790B90CF
:101800000A73E0F53512F1169006B2E0FF7D021280
:10181000EFC09006B2E004F0900BE8E06404702C96
:10182000120F94EF704A9006B2E0FF7BFF7A57796F
:1018300010900A74E0F53512F1169006B2E0FF7DC3
:101840000312EFC09006B2E004F080249006B2E0EC
:10185000FF7BFF7A577910900A74E0F53512F11684
:101860009006B2E0FF7D0312EFC09006B2E004F0F4
:101870009006B2E0FF7BFF7A57791512F19590063A
:10188000B2E075F005A42485F582E43404F583E024
:10189000547FF0900A75E090571F93FF12C1EF90AC
:1018A00006B2E0FF75F005A42487F582E43404F560
:1018B00083121F177D0512EFC0900A75E0FF900696
:1018C000B2E02415F582E43405F583EFF09006B21A
:1018D000E004F0E0FF7BFF7A5C790612DEB9900647
:1018E000B2E0FF12C4069006B2E0FF7D0812EFC01E
:1018F0009006B2E004F0E0FF12F01E22301F131237
:10190000093AEF600D12093AEF640E6005E4FF1228
:1019100010007F2D12F294E49006B2F012093AEF13
:10192000704B9006B2E0FF7BFF7A5C791512F1955F
:101930009006B2E0FF75F005A42485F582E4340436
:10194000F583E0547FF012E9AF9006B2E0FFE4FDCA
:1019500012EFC0900A78E0FF9006B2E02415F582FD
:10196000E43405F583EFF09006B2E004F09006B29F
:10197000E0FF7BFF7A6379B312F195301F56900434
:101980004FE075F003A42455F582E43404F5831286
:101990001F0E121B4F6404703B120CD65011900C9A
:1019A00098E0FFA3E09006B3CFF0A3EFF08015120C
:1019B0000C4CEEC4F854F0C8689006B3F0EFC45471
:1019C0000F48A3F09006B3E0FEA3E0FF9006B2E05C
:1019D000FD129A589006B2E0FF7D0312EFC0900608
:1019E000B2E004F0E0FF7BFF7A5C790B12F1959096
:1019F00006B2E0FF7D0412EFC09006B2E004F012E0
:101A00000CD64028900B85E0FF12E6238F35900618
:101A1000B2E0FF7BFF7A6379B812F1169006B2E06C
:101A2000FF7D0512EFC09006B2E004F09006B2E030
:101A3000FF7BFF7A5C790612F1959006B2E0FF1207
:101A4000C4069006B2E0FF7D0612EFC09006B2E039
:101A500004F0E0FF12F01E228E308F318D3290099B
:101A600003E530F0A3E531F0E49008F7F03041737E
:101A700090044FE06532706B12B8E98B548A558937
:101A8000567B017A0879F71252C0120CD65011E435
:101A90009008FCF09008FAE0A3F09008FA742EF099
:101AA000754EFF754F8B7550677B017A0879F71279
:101AB000560A9008E9E0FF90044FE0FE75F005A497
:101AC0002486F582E43404F583EFF07B017A08790B
:101AD000F7EE75F005A42487F582E43404F583124B
:101AE0001F1722900BE8E0B40129900C98E0FAA3AC
:101AF000E0FB7C007D64FFCEEACE121BFD8E308FB2
:101B0000317C007D64CFEBCFCEEACE121BFD900678
:101B1000B5EDF07B017A0879F7AD31AC301257E3BF
:101B2000120CD6504C7B017A0879F77D2E1254089E
:101B300090044EE0B409167B017A0879F79006B557
:101B4000E075F00A84FD7C001257E380249006B50E
:101B5000E0C3940A500B7B017A0879F77D30125468
:101B6000087B017A0879F79006B5E0FD7C001257F2
:101B7000E3754EFF754F8B7550677B017A0879F7D7
:101B800012560AE53275F005A42486F582E4340481
:101B9000F583E4F07B017A0879F7E53275F005A466
:101BA0002487F582E43404F583121F1722E490069B
:101BB000B2F07F0412F2941209E240559006B2E0AE
:101BC000FF7BFF7A5079F912F1959006B2E0FFE4BD
:101BD000FD12EFC0900D27E0FF120FB89006B2E0A3
:101BE0002415F582E43405F583EFF0900D27E0909D
:101BF000512393FF12C1EF9006B2E075F005A424C3
:101C000087F582E43404F583121F179006B2E004CE
:101C1000F0120CD6404E9006B2E0FF7BFF7A50796E
:101C2000FE12F195900CEDE090511793FF12C1EF69
:101C30009006B2E0FF75F005A42487F582E4340431
:101C4000F583121F177D0112EFC0900CEDE0FF909D
:101C500006B2E02415F582E43405F583EFF0900632
:101C6000B2E004F09006B2E0FF7BFF7A51790312F4
:101C7000F1959006B2E0FF900B87E0FD7C0012EE3C
:101C8000979006B2E0FF75F005A42485F582E43450
:101C900004F583E04480F07D0412EFC09006B2E0CA
:101CA00004F0E0FF7BFF7A51790812F1959006B2BB
:101CB000E0FF7D0512EFC09006B2E004F0E0FF7B8C
:101CC000FF7A51790D12DEB99006B2E0FF7D06125F
:101CD000EFC09006B2E004F0E0FF7BFF7A5179128A
:101CE00012DEB99006B2E0FF7D0712EFC09006B297
:101CF000E004F0E0FF12F01E228B2C8A2D892E12B8
:101D00001B4F24CE6069046003029E31782CE47579
:101D1000F001121EFE121B4F900962F0782CE47540
:101D2000F001121EFE121B4F900963F0782CE4752F
:101D3000F001121EFE121B4F900964F0782CE4751E
:101D4000F001121EFE121B4F900965F0782CE4750D
:101D5000F001121EFE121B4F900966F0782CE475FC
:101D6000F001121EFE121B4F900967F0029E31789F
:101D70002CE475F001121EFE121B4F900968F078DA
:101D80002CE475F001121EFE121B4F900969F078C9
:101D90002CE475F001121EFE121B4F90096AF078B8
:101DA0002CE475F001121EFE121B4F90096BF078A7
:101DB0002CE475F001121EFE121B4F90096CF07896
:101DC0002CE475F001121EFE121B4F90096DF0906D
:101DD0000969E0FFC394304058EFD39439505290D2
:101DE000096BE0FEC394304048EED394395042A3CF
:101DF000E0FDC39430403AEDD394395034EE540FA3
:101E000075F00AA4FEED540F2EFEEF540F75F0642A
:101E1000A42EFF7E009006ACEEF0A3EFF0D3900C62
:101E200091E09F900C90E09E4007900C60E0440190
:101E3000F0900CA2E0B40109D20C7FA17E1712BF72
:101E4000C1228F2CE52C24F99006AEF0E52C24F964
:101E500024FD4003029EF924FD500A24FD400302A4
:101E60009EF9029F87900BB8E06456703F9006AED3
:101E7000E0246EF582E43409F583E0C394FF502C2E
:101E80009006AEE0FF246EF582E43409F583E004A9
:101E9000F0746E2FF582E43409F583E0FD7B02AF28
:101EA0002C120B1A900977E04404F022900BB8E052
:101EB00064556003029F879006AEE0246EF582E4CD
:101EC0003409F583E0D394005003029F879006AE57
:101ED000E0FF246EF582E43409F583E014F0746EBB
:101EE0002FF582E43409F583E0FD7B02AF2C120B61
:101EF0001A900977E04404F022900BB8E064567021
:101F0000419006AEE0246EF582E43409F583E0C327
:101F1000648094B2502C9006AEE0FF246EF582E40B
:101F20003409F583E004F0746E2FF582E43409F58A
:101F300083E0FD7B02AF2C120B1A900977E044047A
:101F4000F022900BB8E06455703D9006AEE0FF249F
:101F50006EF582E43409F583E0D36480944E402723
:101F6000746E2FF582E43409F583E014F09009775C
:101F7000E04404F0746E2FF582E43409F583E0FD4B
:101F80007B02AF2C120B1A228F398D3A8B3B7A00D1
:101F9000793E783E7C007D007BFF7A6B798A7E00FB
:101FA0007F02121B07900D2B7480F012E970E47809
:101FB0005DF27851F2E539D3943040047F308002ED
:101FC000AF397852EFF2E53AD3941040047F108095
:101FD00002AF3A7850EFF2E53B601D900ABBE05447
:101FE0003FFF900ABDE0543F6F60287852E22F54C3
:101FF0003FF09087F4F0801B900AB4E0543FFF90CC
:102000000AB6E0543F6F600B7852E22F543FF090D5
:1020100087E1F0900D2BE0F53C753D00E53D242077
:10202000FFE4353CCDEFCDFC7852E2FF7850E28FF3
:10203000F0A4FFAEF08D828C837420F0A3E4F074E2
:10204000022DFDE43CFCEF1F70011E144E70E6F5FE
:102050003A7850E2FFE53AC39F5007AF3FCDEFCD4E
:1020600080027D0012A0B17002053C7850E2FFE5CD
:102070003AC39F5007AF3ECDEFCD80027D0012A046
:10208000B17002053CAE3EAF3F7852E2FD7C00EEFF
:102090005403FACBEFCBEE54FCFEEB2DFDEC3A549F
:1020A000034EF53EEDF53F053AE53AC3941040A1E5
:1020B00022AF3DAE3C12E5D4053DE53D228F341202
:1020C0000934EFC0E012093ACDEFCDD0E0FF12099C
:1020D000409006BFEFF0E4A3F07B017A0679BFA33E
:1020E000121F1778C57C067D017BFF7A8B79A67E4F
:1020F000007F06121B07900917E534F090044EE0AC
:1021000024F670197B017A0A79E49006C1121F1730
:102110009009187402F09006C014F080297B017AAF
:102120000D79289006C1121F179009187401F0123A
:102130000CD650127B017A0B795E9006C1121F17E4
:102140009009187404F0900917E014700302A1D8E4
:1021500014601B14700302A1D82403600302A1E7DA
:102160009006C1121F0E121B4F900905F022E49039
:1021700006C4F0120934EFC0E012093ACDEFCDD019
:10218000E0FF1209409006C4E075F003A424C5F5F1
:1021900082E43406F583121F0EEF121BB79006C4BB
:1021A000E004F0E0C3940240CA9006C0E06401601D
:1021B00017120934EFC0E012093ACDEFCDD0E0FF9D
:1021C000120940900905EFF0900905E0FF9006C163
:1021D000121F0EEF121BB722900905E0FF9006C1F7
:1021E000121F0EEF121BB722900526E01460411457
:1021F000700302A2CD14606C2403600302A3049058
:10220000044FE0FF900452E014FBA205500280014D
:10221000C3920CD20DE4FD1246C690044FEFF0E4D9
:10222000900528F012EF5820200302A304C22022B8
:102230007F0F12E8CE400302A304900527E0FF9031
:10224000052DE014FBA20550028001C3920CD20DB3
:10225000E4FD1246C6900527EFF090052CE02FFF15
:10226000120D0622900527E0FF9006AEF090052D96
:10227000E014FBA20550028001C3920CD20DE4FDD4
:102280001246C6900527EFF090052CE02FFF120DA7
:102290000C900BD6E030E010120CD6500BD20C7F15
:1022A000837E0012BFC18017D20C7F027E0012BF56
:1022B000C1120CD65009C20C7F027E0512BFC1901C
:1022C00006AEE0FF900527E0FD120D1222A2059256
:1022D000067F2412DF78900528E0FE900527E0C3F2
:1022E0009E75F003A424D5F582E43404F583121F0F
:1022F0000E90052AE07C0024FFF582EC34FFF58384
:10230000EF121BC9229006AE7407F0A374FFF012FF
:10231000E79CBF120A9006AE740FF0A374FFF09012
:102320000BB9E0FF64027050900BB8E0B4562C90EB
:10233000095FE475F001121C529006AEE0FCA3E0C8
:10234000FDD3900960E09DEC6480F890095FE06443
:1023500080984020ECF0A3EDF0801990095F74FFA5
:10236000F5F0121C52C390095FE064809480500421
:10237000E4F0A3F0C2418078EF64017073126AA5A3
:10238000EF600302A41D9008E8E0FF9008E9E0C3B5
:102390009F4003D38001C3500312EF58900BB8E065
:1023A000FD7F0412E1119008E8E0FF9008E9E0C326
:1023B0009F4003D38001C350379008EAE0FEA3E0BA
:1023C000FF90095FEEF0A3EFF0C39006AFE09FEE41
:1023D0006480F89006AEE0648098501212EF589036
:1023E00008EAE0FFA3E090095FCFF0A3EFF0C2415D
:1023F00012E79CBF121720411490095FE0FF33954C
:10240000E0CDEFCDA3E0FB7F10120B1A2290095F05
:10241000E0FEA3E0FF1227D6900961EFF022900BB7
:10242000A27401F0D240900806E0121F20A44600DA
:10243000A47501A47D02A49303A4A704A4BA05A5CE
:102440000E060000A52D7BFF7A29790D12EDEAE436
:102450009006E6F09006E6E0FFC3940C400302A568
:102460002DEF24A2FF7E001227D612F1239006E65C
:10247000E004F080DF7F3512F12302A52D7F3612B4
:10248000F123120ECE50047F0080027F2A12F13D0C
:1024900002A52D7F3712F123120ED4EF9029DD9380
:1024A000FF12F13D02A52D7F3812F123900A09E0B9
:1024B0009029E193FF12F13D80737F3912F123E4FB
:1024C0009006E6F09006E6E0FFC39403505FEF90BD
:1024D00029F293FF12F13D9006E6E02478F582E4BC
:1024E0003409F583E0FF7E00C21375480175490683
:1024F000754AE77D0312E4D47B017A0679E712EE90
:10250000007F2012F1239006E6E004F080B67F30D1
:1025100012F1237F0D12F13D900A0CE030E2047FAE
:102520000780027F0812F13D7F2012F123900807F7
:10253000E04401F0C240228F428D438B4412E8AD4B
:10254000AD43AF4212D855400302A6339007FDE0D9
:102550009006E4F09007FEE09006E5F0E4900806AF
:10256000F09006E4E0FFA3E0C39FFE900806E0FDC4
:10257000D39E400302A633ED2FFF9007FFE0FD122C
:10258000F1ABE5446401600302A611900804E0FF8A
:10259000A3E0FD12F243E49007D3F090080774F82B
:1025A000F0E4A3F0900802E0FEA3E0FF4E607BCAD7
:1025B000EECAC9EFC9121F73AD43AF42120D4250AC
:1025C000259007D3E070028001C34017900801E016
:1025D000FF900807E030E0047D0080027D0112AC2E
:1025E000D6800312E88CAD43AF42120D42403B90BF
:1025F0000806E070079009E5E030E0079009E5E0A3
:1026000030E107AD43AF42120D48E49009E5F08098
:1026100019E5447015900800E004FF12EEBF900821
:1026200006E07006FDAF42120D48900806E004F087
:1026300002A56112EDA5D322120D727E0A7F2C1223
:102640000D78400302A730E49006F8F09006F8E019
:10265000FFC394135022742C2FF582E4340AF583BF
:10266000E0FFC394204006EFD3947F40037420F032
:102670009006F8E004F080D4E49006F8F09006F8B4
:10268000E0F9C394145030E9FFC374149FFFE4943D
:1026900000FE742B2FF582740A3EF583E0642060FF
:1026A0000E742C2FF582740A3EF583E4F0800890B6
:1026B00006F8E004F080C6E9FFC374149FFFE494B9
:1026C00000FE742C2FF582740A3EF583E0B42002DC
:1026D000E4F0E49006F8F09006F8E0FFC39413509D
:1026E0004F742C2FF582E4340AF583E064206038BF
:1026F000E49006F9F09006F8E0FFC39413502974B3
:102700002C2FF582E4340AF583E0FF9006F9E024EB
:102710002CF582E4340AF583EFF09006F9E004F03A
:102720009006F8E004F080CD9006F8E004F080A771
:102730007B017A0A792C22745C900AAFE054F3F0A2
:102740009087E4F054FC900AAFF09087E4F0EF1229
:102750001F20A77E00A77101A79202A7BD03A7A40F
:1027600004A7CA05A7E006A7F607A811080000A855
:102770002F12B50E900BF7E012B48302B52712B5F5
:102780000E900BF5E012B51E543F242312B48F02B5
:10279000B52E12B46D12B4FE12B4D512B4BA53A150
:1027A000BF02B52712B4DE43A12012B51D12B491A9
:1027B00012B49A53B5FE12F2BE53A1BF2212B46DE9
:1027C00012B49A12B52753A1BF2212B46D12B4C32A
:1027D000900BC512B4B712F2C453B5FE43A1402208
:1027E00012B4DE43A120900BF512B47E12B49A12FB
:1027F000B52E53A1BF2212B4DE43A120900BF512D7
:10280000B47E12B4FE12B4D512B4BA53A1BF02B54D
:102810002E12B4DE53A1DF12B51D12B49112B4C34F
:10282000900BC512B4B753B5FE12F2C443A14022B7
:10283000E49006B2F07BFF7A56799BFF12DEB990E6
:1028400006B2E0FFE4FD12EFC09006B2E004F0E053
:10285000FF7BFF7A5679A012DEB99006B2E0FF7DC9
:102860000112EFC09006B2E004F0900B9FE030E65A
:102870001E9006B2E0FF7BFF7A5679A512DEB99072
:1028800006B2E0FF7D0212EFC09006B2E004F090C5
:102890000B9FE030E51E9006B2E0FF7BFF7A567991
:1028A000AA12DEB99006B2E0FF7D0312EFC09006D7
:1028B000B2E004F0900B9EE030E71E9006B2E0FF1D
:1028C0007BFF7A5679AF12DEB99006B2E0FF7D0940
:1028D00012EFC09006B2E004F09006B2E0FF7BFF7A
:1028E0007A5679B412DEB99006B2E0FF7D0A12EF93
:1028F000C09006B2E004F0900B9BE030E61E90061C
:10290000B2E0FF7BFF7A5679B912DEB99006B2E0E9
:10291000FF7D0E12EFC09006B2E004F09006B2E028
:10292000FF12F01E228B4B8A4C894D9006EFEEF081
:10293000A3EFF0121B4F9006F1F0900001121B68FC
:1029400024FF9214900002121B6824FF9215900637
:10295000F1E0FFF582758300E4121BC9EF149006C5
:10296000EDF09006EDE0C364809480404B9006EF5C
:10297000E0FEA3E0FF7C007D0A121BFDED2430FF8A
:10298000AB4BAA4CA94D9006EDE0FD3395E08D824E
:10299000F583EF121BC99006EFE0FEA3E0FF7C0079
:1029A0007D0A121BFD9006EFEEF0A3EFF04E6008DB
:1029B0009006EDE014F080AA9006EDE0D3648094D8
:1029C000804053A37420F030151BAB4BAA4CA94D8B
:1029D0009006EDE014FFF03395E08F82F583742DBF
:1029E000121BC980093014069006EE7430F0900670
:1029F000EDE0D364809480401DA3E0FFAB4BAA4C74
:102A0000A94D9006EDE014F0FD3395E08D82F5833D
:102A1000EF121BC980D822EF14605014700302AA71
:102A2000D62402600302AB07900BE9E06403600365
:102A300002AB0790044EE06409600302AB0720205C
:102A40000302AB07900905E0FF120E08EFC0E01289
:102A50000934CEEFCED0E0FFEE6F700302AB0790EB
:102A60000905E0FF120E08120CD022C220E49004E7
:102A70004FF0D226120CD6500812E79CEF64096082
:102A800019900BD6E020E012C20C7F407E0012BFEE
:102A9000C1C20C7F407E0112BFC1D20512DD727F20
:102AA0000312A0BD90044FE09006ACF09006ACE09D
:102AB000FF75F003A42455F582E43404F583121F56
:102AC0000E121B4F640460089006ACE004F080DC3A
:102AD00090044FEFF022900BE9E06403702990041A
:102AE0004EE0B4092290044FE075F003A42455F59C
:102AF00082E43404F583121F0E121B4FB4040890B5
:102B00000CECE07002D226228F328D33E532B40411
:102B100008900C6C7405F08031900C6C7414F0907B
:102B20000BA4E0FFC374149FFF9006B7F012EE2CC5
:102B30007FD112EBC1E532B4030B7BFF7A8A7903B4
:102B400012E22080057F0312EE2CE53214601A1485
:102B5000601E14601414601F24FD60142407703F6D
:102B6000C209AF3312CEA98036AF3312F0B4802F32
:102B7000AF3312EF468028900BE8E0B4010D900CC3
:102B800098E0FEA3E0FF12EC158014120C4CEEC48A
:102B9000F854F0C868FEEFC4540F48FF12EC15E576
:102BA000326404604AE53264076032900BA4E0FFAF
:102BB000C374209FFF12EE2CE532B4030B7BFF7A27
:102BC0008A790712E2208022AF33EF3395E0FEC20C
:102BD000097D0312E1497F0112EE2C800D900BA4B8
:102BE000E0FFC374239FFF12EE2C7FD012EBC122B3
:102BF000E49006ADF07F01FE1227D6BFAA14900B19
:102C0000AAE06409600C12104EC20C7F837E191278
:102C1000BFC19006ADE0700302ACD57F01120E0873
:102C20009006ADEFF0120CFA9006ADEFF07F0112B6
:102C30000CE29006ADEFF07D017C00E4FFFE121087
:102C4000547B017D017F017E0012105A7B017D01C2
:102C50007F017E001210607B017D017F017E0012EA
:102C600010667D017F017E0012106C7F01121072D0
:102C70007F0112DB8C12EDBC7F0112E3E712F04BF7
:102C800012EBA512F2E27B017A0679AC7D0112E328
:102C90002112F17112EF9E12F2D67B017A0679AC05
:102CA0007D35124E4B7F057E0012EFD07B017A06F8
:102CB00079AE12574378327C007D007B017A067929
:102CC000AE7E007F03121B07125A2EE4FF1210780B
:102CD0007FFF12107E228F458D467B017A0779D3C4
:102CE0001254D59006E6EFF0E546B40109900800CD
:102CF000E024FEFF8005900800E0FF9006E7EFF07B
:102D0000E4A3F074D32FF582E43407F583E4F09064
:102D100006E6E0FED39F4005A3E0FF8003CFEECFA1
:102D20009006E6EFF0E545604024FE602804704917
:102D30009006E6E0FF900800E0C39F9006E8F0E50B
:102D400046B40105E014FF80059006E8E0FF900618
:102D5000E8EFF080249006E6E0FF900800E0C39FD3
:102D6000FFC3139006E8F08010E546B401047F012C
:102D700080027F009006E8EFF0E546B4011F9087DF
:102D8000F8E020E7F99006E8E0FF12EE2C900BA4A3
:102D9000E0FF7B017A0779D312E353801A9006E8AB
:102DA000E0FF12EE2C900BA4E014F012F2787B01FD
:102DB0007A0779D312E22012E88C22E490095FF0BE
:102DC000A3F0FFFE1227D6900961EFF0900977E09B
:102DD0004410F07FC512F294E49006B2F0201F0375
:102DE00002AE94E0FF7BFF7A29791012F1959006EC
:102DF000B2E0FF12D2319006B2E004F0E0FF7BFFB8
:102E00007A29791512F1959006B2E004F0E0FF7B83
:102E1000FF7A29791A12F1959006B2E004F0E0FFEA
:102E20007BFF7A29791F12F1959006B2E004F0E059
:102E3000FF7BFF7A29792412F1959006B2E004F025
:102E4000E0FF7BFF7A29792912F1959006B2E00420
:102E5000F0E0FF7BFF7A29792E12F1959006B2E01F
:102E600004F0302E13E0FF7BFF7A297933D2081269
:102E7000F00F9006B2E004F09006B2E0FF7BFF7A1C
:102E8000297938900D3EE024FF920812F00F900649
:102E9000B2E004F09006B2E0FF12F01E227F0A7E3C
:102EA0000012EE6E7F2C12F294E49006B2F07BFFDB
:102EB0007A5C792EFF12DEB99006B2E0FF75F0055C
:102EC000A42485F582E43404F583E0547FF0900B6C
:102ED00087E014FD7C0012EE979006B2E0FFE4FD5F
:102EE00012EFC09006B2E004F0120CD6501090061B
:102EF000B2E0FF7BFF7A5C793812DEB9800E900673
:102F0000B2E0FF7BFF7A5C793312DEB9120C4CEE33
:102F1000C4F854F0C8689006B3F0EFC4540F48A347
:102F2000F0900CECE0602B120CD65011900C98E055
:102F3000FFA3E09006B3CFF0A3EFF08015120C4C86
:102F4000EEC4F854F0C8689006B3F0EFC4540F48CC
:102F5000A3F09006B3E0FEA3E0FF9006B2E0FD12FE
:102F60009A589006B2E004F0E0FF7BFF7A5C793D6E
:102F700012DEB99006B2E004F0E0FF12F01E228FDC
:102F8000477B007A0079471208A49006F9EFF060B9
:102F900005E0F9B40E1A302E0302B0579006F9E09E
:102FA000640E600302B05774C82547F54702B05756
:102FB000E9B4050675478C02B057E9B406067547B3
:102FC0008E02B057E9B4090675478D02B057E9B4CF
:102FD000070675478F02B057E9B40805754790801A
:102FE00076E9B40A05754788806DCFE9CF120DAE3A
:102FF000501C900B9FE0FF30E30F30E20C9006F97D
:10300000E0B40205754789804E7547878049900670
:10301000F9E0B401077F02120DB4500E7F01120DCA
:10302000B4400C9006F9E0B40205E49006F9F09083
:1030300006F9E0908BAC932472600F146011146059
:10304000132403701275477E800D75477F800875C5
:1030500047808003754781AF4722EF75F003A424B2
:1030600055F582E43404F583121F0E900001121B03
:1030700068600D14700DE4FF120CE290052DEFF066
:1030800012F1F2E49006B1F09006B1E0FFC39406AD
:10309000400302B131900528E0FEEF2EFFA3E0FED1
:1030A000EFD39E400302B12812EB51EF6433600668
:1030B00012EB51BF34289006B1E075F006A4242E1F
:1030C000F9740535F0FA7B01900528E0FF9006B110
:1030D000E02FFF90052CE02FFF12C9DA8013900635
:1030E000B1E075F006A4242EF582E43405F583E4FE
:1030F000F09006B1E0FF75F006A42433F582E434C5
:1031000005F583E4F0EF75F006A4242EF974053577
:10311000F0FA7B019006B1E075F003A424D5F582A6
:10312000E43404F583121F179006B1E004F002B0F6
:1031300088227F0212F294E4F5307BFF7A5079C244
:10314000AF3012DEB9E4FDAF3012EFC005307BFFC7
:103150007A5079E0900A08E024CEF535AF3012F1CC
:10316000167D01AF3012EFC00530900BE8E064012E
:10317000601A7BFF7A5079EF900A0FE0F535AF3097
:1031800012F1167D02AF3012EFC005307BFF7A508E
:1031900079E5900A0CE0A2E29208AF3012F00F7DC0
:1031A00003AF3012EFC005307BFF7A5079EAAF30C1
:1031B00012F195120D66EF9050F493FF12C1EFE5F6
:1031C0003075F005A42487F582E43404F583121FDA
:1031D000177D04AF3012EFC0120D6674152530F55F
:1031E00082E43405F583EFF005307BFF7A5C7906E5
:1031F000AF3012DEB9AF3012C4067D07AF3012EF28
:10320000C00530AF3012F01E22900BA27401F0D234
:1032100040900806E014605D04600302B2CF900D98
:103220003CE0B401097BFF7A29790712EDEA900DA1
:103230003CE060047F2780027F3012F130E490068A
:10324000E6F09006E6E0FFC39405400302B2CF1219
:103250000EC87E00C213754801754906754AE77DA0
:103260000312E4D47B017A0679E712EDEA9006E6D0
:10327000E004F080CD900D3CE0B401097BFF7A2999
:10328000790A12EDEA7F2812F1307F2012F123E44F
:103290009006E6F09006E6E0FFC394075031EF2475
:1032A00011FF7E001227D67E00D2137548017549A2
:1032B00006754AE77D0312E4D47B017A0679E712AA
:1032C000EDEA7F2012F1239006E6E004F080C5903D
:1032D0000807E04401F0C240228E3C8F3DE53C905F
:1032E00006C5F0C20FC210D21175410175420675B4
:1032F00043C775441B7B017A08792B1253AEE490C7
:1033000006C6F09006C6E0FFC3941B506F9006C53A
:10331000E0FEEF6E605E7B02E4FD12DA67505590CE
:1033200006C5E0FFA3E0FD12BAEC5048200E0E9057
:1033300006C6E0FDAF3DAE3C12D80650339006C63F
:10334000E0FF24C7F582E43406F583E06004E4F08E
:10335000D20F740D2FF582E43408F583E060157404
:10336000C72FF582E43406F5837440F0D210800450
:10337000C21180089006C6E004F080873011212039
:103380001003300F1B75410175420875432B7544BE
:103390001B7B017A0679C71253AE30100312EC4B37
:1033A000A21122C2139006EBEFF0900BE8E0B401FB
:1033B00008120E089006EBEFF09006EBE0FF120FFC
:1033C000D0E49006E9F09006E9E0FFC394054003DD
:1033D00002B45874F02FF582E4340AF583E09006C5
:1033E000EAF064206069E0F9C39461401AE9D3947B
:1033F0007A5014E924E0FE74F02FF582E4340AF5E3
:1034000083EEF0D2138048E964276043E9644060AA
:103410003E742BD3995005E9942F4033743AD399D5
:103420005005E9943B40287430D3995005E994390C
:10343000401D7441D3995005E9945A40129006E911
:10344000E024F0F582E4340AF5837420F0D213907E
:1034500006E9E004F002B3C63013089006EBE0FF83
:10346000120CDC12D4637B017A0A79F022900ABC38
:10347000E04401F09087FFF053A1DF900BF7E025C7
:10348000E02405900ABBF09087F2F0543F242854C2
:103490003F900ABDF09087F4F022900BC6E0547F75
:1034A000900AB7F09087E2F0900BC7E0900AB4F072
:1034B0009087E0F0900BC8E0543F900AB6F09087F8
:1034C000E1F022900BC3E0547F900AB7F09087E2BE
:1034D000F0900BC4E0900AB4F09087E0F022900ADC
:1034E000BCE04401F09087FFF022E0900AADF0903C
:1034F00087F1F0543F900AB0F09087E3F022900BF0
:10350000C6E0547F900AB7F09087E2F0E422900A78
:10351000BCE054FEF09087FFF053A1DF22E4900A54
:10352000BBF09087F2F02212F2BE53B5FE2212F2E7
:10353000C443B5012212EB51EF6434600B12EB511E
:10354000EF6433600302B5F7900BB8E024E06074D9
:1035500014607114602F24D0607C241A600302B5BB
:10356000E1900526E0B4010B12EB51BF3405D20601
:1035700002B5F7900526E0FF64036005EF64027072
:1035800076D2068072900526E06401702512EB5118
:10359000EF6434600812EB51EF6433705A120CFA86
:1035A000EFD39463405112093AEF640E6049D2069A
:1035B0008045900526E0FF64036005EF64027037E4
:1035C000D2068033900526E0FF64036005EF6402B5
:1035D0007025D2068021900526E0B4021AD206801A
:1035E00016900BB9E0B4010F900526E0FF6403606C
:1035F00004EFB40202D206A206227F3612F294E44D
:103600009006B2F07BFF7A5079C7900A02E024CE90
:10361000F535E4FF12F1169006B2E0FFE4FD12EF7B
:10362000C09006B2E004F0E0FF7BFF7A5079CC90C6
:103630000A03E024CEF53512F1169006B2E0FF7DC4
:103640000112EFC09006B2E004F0E0FF7BFF7A5079
:1036500079D1900A04E024CEF53512F1169006B225
:10366000E0FF7D0212EFC09006B2E004F0E0FF7BC5
:10367000FF7A5079D6900A05E024CEF53512F1167E
:103680009006B2E0FF7D0312EFC09006B2E004F0B6
:10369000E0FF7BFF7A5079DB900A10E024CEF5350D
:1036A00012F1169006B2E0FF7D0412EFC09006B250
:1036B000E004F0E0FF12F01E22E4FF12F294E49026
:1036C00006B2F07BFF7A29793DFF12DEB99006B28F
:1036D000E0FF12CB3C9006B2E004F0E0FF7BFF7A03
:1036E00029794212DEB99006B2E0FF12CB3C900677
:1036F000B2E004F0E0FF7BFF7A29794712DEB9904F
:1037000006B2E0FF12CB3C9006B2E004F0E0FF7B93
:10371000FF7A29794C12DEB99006B2E0FF12CB3C59
:103720009006B2E004F0E0FF7BFF7A29795112DEC7
:10373000B99006B2E0FF12CB3C9006B2E004F0E094
:10374000FF7BFF7A29795612DEB99006B2E0FF12AC
:10375000CB3C9006B2E004F0E0FF7BFF7A29795B76
:1037600012DEB99006B2E0FF12CB3C9006B2E00444
:10377000F0E0FF12F01E228F31EF75F005A42485D2
:10378000F582E43404F583E020E74FEF75F003A4FD
:103790002455F582E43404F583121F0E121B4F14D6
:1037A000602514602914601114601524FD6026043E
:1037B0007028AF3112D9D38021AF3112D61A801AB6
:1037C000AF3112C48A8013AF3112D170800CAF3187
:1037D00012D6C28005AF3112D56F90044FE075F05C
:1037E00003A42455F582E43404F583121F0E121B42
:1037F0004F6405603CE53175F005A42485F582E44D
:103800003404F583E030E529900C6C7423F0900BC0
:10381000A4E0FFC374239FFF12EE2C900BA4E0FFE3
:10382000900C6CE0C39FFF9006B4F012EE2C12F2E5
:103830009A228F30900A6EE060317F6B12C1EFE503
:103840003075F005A42487F582E43404F583121F53
:1038500017E53075F005A42485F582E43404F5837A
:10386000E054DFF090094B7401F022900A7074016B
:10387000F0900A6FE0B401197F6C12C1EFE530756A
:10388000F005A42487F582E43404F583121F178021
:103890004E7F6D12C1EFE53075F005A42487F582E7
:1038A000E43404F583121F1790094BE06401601C97
:1038B0007F6A12C1EFE53075F005A42487F582E434
:1038C0003404F583121F17E4900A70F0E53075F0A8
:1038D00005A42485F582E43404F583E04420F0E473
:1038E00090094BF0900A6FF0229008EAE0FFA3E005
:1038F0009006B7CFF0A3EFF09008E8E09006B9F09B
:10390000E024ECF582E43408F583E4F09006B6F0A8
:103910009008E9E0FF9008E8E0C39FFF9006B6E05A
:10392000C39F501A9006B9E014F024ECF582E434F9
:1039300008F583742DF09006B6E004F080D2E49090
:1039400006B6F09008E9E0FF9006B6E0C39F50414C
:10395000A3E0FAA3E0FB7C007D0AFFCEEACE121BB7
:10396000FDED2430FFA3E014F024ECF582E43408EC
:10397000F583EFF07C007D0ACFEBCFCEEACE121BB1
:10398000FD9006B7EEF0A3EFF09006B6E004F080ED
:10399000B27B017A0879EC22120D3C90052CEFF0F5
:1039A000E4FF120CE290052DEFF090044FE075F06B
:1039B00003A42455F582E43404F583121F0E121B70
:1039C0004F24F8602014705B900526E0B40303D305
:1039D0008001C3406C12093490052CE0FEC3EF9EB9
:1039E000900527F022120CD6501AE4FF120CE29038
:1039F000052DEFF012093490052CE0FEC3EF9E90E8
:103A00000527F022120934EFC0E012093ACDEFCDBC
:103A1000D0E0FF12094090052CE0FEC3EF9E900518
:103A200027F022120934EFC0E012093ACDEFCDD0D1
:103A3000E0FF12094090052CE0FEC3EF9E900527A1
:103A4000F022EF121F20BA7300BA6801BA6802BAF6
:103A50006503BA7B04BA8305BA7006BA7307BA8ED7
:103A6000080000BA9412F16412EC6612F157802437
:103A700012F16412E75312EBDD801912EC6612F1B9
:103A800064801112E75312F15712EBF9800612E726
:103A90005312EBF9900AB37454F09087F5F0900A42
:103AA000B17421F09087F6F0E4900AB5F09087F7B2
:103AB000F0900AB904F09087F8F0900AAE7405F01F
:103AC0009087FCF0E4900AB2F09087FDF0900ABA7B
:103AD000F09087FEF0900ABCE0548F4420F090876D
:103AE000FFF0C228E4900C73F002F28D8F3ECFED10
:103AF000CFC212C2137D0112D855921378EA7C0608
:103B00007D017B017A0779FD7E007F07121B077D0F
:103B100001AF3E12D855821392133013739007FFF2
:103B2000E0FF9006E2F09007FDE09006E3F09008D9
:103B300000E02FFF9006E4F09007FEE09006E5F02D
:103B40009006ECE0FE9006E6F09006EAE09006E7CC
:103B5000F09006EDE02E9006E8F09006EBE090067F
:103B6000E9F0D212EED39F50259006E5E0FF9006D3
:103B7000E7E09F50199006E2E0FF9006E8E0C39F5F
:103B8000400C9006E3E0FF9006E9E09F5002C2126D
:103B9000A21222E4FF12F294E49006B2F0900BE835
:103BA000E06401601E9006B2E0FF7BFF7A5C791A48
:103BB00012DEB99006B2E0FFE4FD12EFC09006B24B
:103BC000E004F09006B2E0FF7BFF7A5C791F12DE22
:103BD000B99006B2E0FF7D0112EFC09006B2E0049A
:103BE000F0E0FF7BFF7A5C792412DEB99006B2E048
:103BF000FF7D0212EFC09006B2E004F0900BE8E007
:103C00006404602A12093AEF600612093ABF0E1ED8
:103C10009006B2E0FF7BFF7A5C792912DEB990064C
:103C2000B2E0FF7D0312EFC09006B2E004F0900610
:103C3000B2E0FF12F01E22900BB9E0B4021B12EFAB
:103C400058D24190044FE075F005A42485F582E434
:103C50003404F583E054DFF022900BB9E064017086
:103C600075126AA5EF706F9008E8E0FF9008E9E030
:103C7000C39F4003D38001C3500312EF58900BB889
:103C8000E0FD7F0312E1119008E8E0FF9008E9E011
